:020000040800F2
:1000000000090020250500081D1A0008ED19000848
:10001000091A0008ED190008011A00082705000850
:10002000270500082705000827050008993500085E
:10003000270500082705000827050008AD3A000835
:1000400027050008270500082705000827050008E0
:100050002705000827050008DD37000809380008D3
:1000600035380008613800088D3800082705000879
:1000700027050008270500082705000827050008B0
:100080002705000827050008270500083D2A000865
:10009000A92A0008FD2A0008512B0008B9380008D9
:1000A0002705000827050008270500082705000880
:1000B0002705000827050008270500082705000870
:1000C0002705000827050008270500082705000860
:1000D0002705000827050008270500082705000850
:1000E0002139000827050008270500082705000812
:1000F0002705000827050008270500082705000830
:10010000270500082705000827050008270500081F
:10011000270500082705000827050008270500080F
:1001200027050008270500082705000827050008FF
:1001300027050008270500082705000827050008EF
:1001400027050008270500082705000827050008DF
:1001500027050008270500082705000827050008CF
:100160004FF0FF0C1CEAD0521EBF1CEAD15392EA9A
:100170000C0F93EA0C0F6FD01A4480EA010C400276
:1001800018BF5FEA41211ED04FF0006343EA5010D0
:1001900043EA5111A0FB01310CF00040B1F5000F12
:1001A0003EBF490041EAD3715B0040EA010062F1C1
:1001B0007F02FD2A1DD8B3F1004F40EBC25008BFAB
:1001C00020F00100704790F0000F0CF0004C08BFC9
:1001D00049024CEA502040EA51207F3AC2BFD2F196
:1001E000FF0340EAC250704740F400004FF00003A4
:1001F000013A5DDC12F1190FDCBF00F000407047DE
:10020000C2F10002410021FA02F1C2F1200200FA1B
:1002100002FC5FEA310040F1000053EA4C0308BFE2
:1002200020EADC70704792F0000F00F0004C02BF33
:10023000400010F4000F013AF9D040EA0C0093F0AE
:10024000000F01F0004C02BF490011F4000F013B08
:10025000F9D041EA0C018FE70CEAD15392EA0C0F76
:1002600018BF93EA0C0F0AD030F0004C18BF31F0E1
:10027000004CD8D180EA010000F00040704790F0B7
:10028000000F17BF90F0004F084691F0000F91F05B
:10029000004F14D092EA0C0F01D142020FD193EA21
:1002A0000C0F03D14B0218BF084608D180EA0100A9
:1002B00000F0004040F0FE4040F40000704740F085
:1002C000FE4040F44000704780F0004002E000BF74
:1002D00081F0004142001FBF5FEA410392EA030F31
:1002E0007FEA226C7FEA236C6AD04FEA1262D2EB7B
:1002F0001363C1BFD218414048404140B8BF5B4280
:10030000192B88BF704710F0004F40F4000020F018
:100310007F4018BF404211F0004F41F4000121F02E
:100320007F4118BF494292EA030F3FD0A2F1010278
:1003300041FA03FC10EB0C00C3F1200301FA03F1B6
:1003400000F0004302D5494260EB4000B0F5000FD9
:1003500013D3B0F1807F06D340084FEA310102F198
:100360000102FE2A51D2B1F1004F40EBC25008BF4A
:1003700020F0010040EA03007047490040EB000014
:10038000013A28BFB0F5000FEDD2B0FA80FCACF115
:10039000080CB2EB0C0200FA0CF0AABF00EBC25042
:1003A00052421843BCBFD0401843704792F0000F30
:1003B00081F4000106BF80F400000132013BB5E783
:1003C0004FEA41037FEA226C18BF7FEA236C21D0F9
:1003D00092EA030F04D092F0000F08BF084670475E
:1003E00090EA010F1CBF0020704712F07F4F04D12C
:1003F000400028BF40F00040704712F100723CBF3F
:1004000000F50000704700F0004343F0FE4040F468
:10041000000070477FEA226216BF08467FEA236326
:100420000146420206BF5FEA412390EA010F40F411
:10043000800070474FF0000304E000BF10F000435D
:1004400048BF40425FEA000C08BF704743F0964344
:1004500001464FF000001CE050EA010208BF70475F
:100460004FF000030AE000BF50EA010208BF7047E6
:1004700011F0004302D5404261EB41015FEA010CFB
:1004800002BF84460146002043F0B64308BFA3F1F3
:100490008053A3F50003BCFA8CF2083AA3EBC253D5
:1004A00010DB01FA02FC634400FA02FCC2F12002F4
:1004B000BCF1004F20FA02F243EB020008BF20F02B
:1004C0000100704702F1200201FA02FCC2F1200291
:1004D00050EA4C0021FA02F243EB020008BF20EA86
:1004E000DC70704742000ED2B2F1FE4F0BD34FF0DA
:1004F0009E03B3EB126209D44FEA002343F000439A
:1005000023FA02F070474FF00000704712F1610FBC
:1005100001D1420202D14FF0FF3070474FF000008E
:10052000704700BF02E000F000F8FEE772B6264810
:1005300080F30888254880F3098825482549086004
:10054000022080F31488BFF36F8F03F075F803F077
:10055000D9F84FF0553020491B4A91423CBF41F831
:10056000040BFAE71D49194A91423CBF41F8040BBC
:10057000FAE71B491B4A1C4B9A423EBF51F8040B39
:1005800042F8040BF8E700201849194A91423CBF91
:1005900041F8040BFAE703F053F803F0B5F8154CF3
:1005A000154DAC4203DA54F8041B8847F9E700F014
:1005B0003FF8124C124DAC4203DA54F8041B884742
:1005C000F9E703F03BB8000000090020001100200B
:1005D0000000000808ED00E00001002000090020F4
:1005E000C03B000800110020241100202811002029
:1005F000D4250020600100086001000860010008A7
:10060000600100082DE9F04FC1F80CD0C3689D4689
:10061000BDE8F08F002383F311882846A04700200F
:1006200002F036FDFEE702F0CFFC00DFFEE700003F
:10063000F8B500F03BFE02F04DFF074602F098FFD0
:10064000064600283ED12B4B9F423BD001339F42B0
:100650003BD0294B27F0FF029A4239D1F8B200F083
:10066000FFFB354642F2107400F000FC08B1002494
:10067000254601F041F978B30024032000F042F848
:10068000254636B11D4B9F4203D0002402F068FF7F
:100690002546002002F028FF194B9B6813F0400309
:1006A0001FD00DB100F044F800F042FC01F0B8F9A1
:1006B0000546C4B101F0B4F9401BA04213D900F0C3
:1006C00037F8F3E735460024CEE704460125CBE7AB
:1006D00005464FF47A74C7E7B4F57A7F08BF012561
:1006E000CFE71C46E0E700F0D5FC012002F0D6FC85
:1006F000DFE700BF010007B0000008B0263A09B0EC
:10070000000C0140084B187003280CD8DFE800F0FB
:1007100008050208022000F025BE022000F01ABEE3
:100720000022024B5A607047281100202C11002033
:1007300038B501F0E1F830B103221F4B1A700022E6
:100740001E4B5A6038BD1E4B1E4A19680131F9D044
:1007500004339342F9D11C4C194DD4F80424AA4215
:10076000F0D31A4B9B6803F1006303F5C8439A4228
:10077000E8D202F0C9FE02F0DBFE002000F0B0FD7E
:100780000220FFF7BFFF124BDA690022DA61D96954
:1007900099699A619B6972B64FF0E023C3F8085DCE
:1007A0003021D4F80034D4F8042481F311889D4614
:1007B00083F308881047C5E7281100202C1100207A
:1007C0000064000820640008006000080011002098
:1007D0000010024049F26900084A136899B21B0CE4
:1007E00000FB013344F250611360054B186882B27C
:1007F000000C01FB0200186080B27047201100203D
:100800001C11002010B504460021102200F0C6FD86
:10081000034B03CB206061601868A06010BD00BF6F
:10082000E8F7FF1FF0B5ADF5517D6EAC4FF4C47223
:1008300007460D462046002100F0B0FD01F0F0F81B
:100840004FF47A72B0FBF2F0244B186093E8070083
:10085000022384E807000DF5ED702382FFF7D2FF35
:1008600045F204031E4906A8238403F057F9232305
:100870000DF2EB2284F832310DF1380C06AB1E4636
:1008800003CE664510605160334602F10802F6D18E
:100890003188B3780FAE1180937031460122204623
:1008A00000F0C8FD00230393AB7E80B2029305F1F4
:1008B000190301930123CDE904600093384605A391
:1008C000D3E90023E97E01F0FFFB0DF5517DF0BD7A
:1008D000AFF300809E6AC421818A46EE3411002065
:1008E0002C3B00082DE9F041264D80462B7A0C4622
:1008F000DAB0FBB9204627A900F0C2FE074600285F
:1009000036D19DF89D60C82E32D801464FF4FA7258
:10091000284600F043FD32460DF19E0105F1090025
:1009200000F02AFD9DF89C302E4477722B720BB993
:10093000E37E2B728122002106AD27A800F02EFD58
:100940000122294627A800F0E1FE00230393A37E9D
:1009500080B2029304F1190301932823CDE90450D6
:100960000093404605A3D3E90023E17E01F0ACFBF0
:100970005AB0BDE8F08100BFAFF30080264172722B
:10098000DF25D7B77C210020F0B54FF48A7500240D
:10099000234EF1B005FB006596F8D830D8222146E9
:1009A00085F8DC3085F8E8403AA800F0F7FC06F15D
:1009B000090000F0EBFCD5F8E430C2B206AF8DF8C8
:1009C000F00006F109010DF1F100CDE93A3400F033
:1009D000D3FC394601223AA800F0CEFE80B2CDE920
:1009E000047008230127CDE9023706F1D8030193EB
:1009F0003023317A00930B4807A3D3E9002301F099
:100A000063FBA04206DD01F00BF8C5F8E0003846B4
:100A100071B0F0BD2046FBE778F6339F93CACD8DC9
:100A20007C2100204C210020F0B51E4E1E4F1F4D92
:100A300085B0304601F074FB044660B310220021FB
:100A4000684600F0ABFC4FF00003227B6068A168B1
:100A500062F303038DF8003002AB03C3019B2268ED
:100A6000384662F31C0301939DF800306A4643F058
:100A700020038DF800300023194602F0E1F9044606
:100A800020B9304601F050FB2C70D2E72B78072BB1
:100A900003D801332B7005B0F0BD024801F044FBD0
:100AA000F9E700BF4C210020A82300207523002077
:100AB00070B50D4614461E4601F062FA50B9022E7A
:100AC00010D1012C0ED112A3D3E900230120C5E9D6
:100AD000002307E0282C10D005D8012C09D0052CC4
:100AE0000FD0002070BD302CFBD10BA3D3E9002325
:100AF000ECE70BA3D3E90023E8E70BA3D3E900233A
:100B0000E4E70BA3D3E90023E0E700BFAFF30080E5
:100B1000401DA12026812A0B78F6339F93CACD8DE4
:100B20009E6AC421818A46EE26417272DF25D7B7BC
:100B3000F017304A39059E5638B505460E4C00214F
:100B4000013500F0EFFBA4F8F051B4F8F00100F02B
:100B5000D1FB78B1B4F8F00100F0DCFB014648B9F4
:100B6000B4F8F00100F0DEFBB4F8F0310133A4F882
:100B7000F031EAE738BD00BF7C2100202DE9F04FBD
:100B80008DB000AF04460D4601F0FAF9002848D1B7
:100B90002B7E022B1AD1EB8A012B17D100F040FFDC
:100BA0000646FFF717FE4FF4C873B0FBF3F202FBE3
:100BB0001303DFF88C829BB206F516763344C8F82F
:100BC0000030EB7E33B900229E4B1A703437BD469D
:100BD000BDE8F08F284607F11C0100F005FD002854
:100BE000F4D107F10C00FFF70DFEBD7F07F10C01FA
:100BF0002A4607F11F0002F061FF0028E3D10F2D04
:100C000008D8904B1D70D8F80030A3F51673C8F8BB
:100C10000030DBE7397F0029D8D0204601F0A8F961
:100C2000D4E7EB8A282B6BD010D8012B63D0052B8F
:100C3000CCD1BFF34F8F8449844BCA6802F4E06281
:100C40001343CB60BFF34F8F00BFFDE7302BBDD107
:100C50007F4CEA7E237A9A42B8D194F8DC206B7EEE
:100C60009A4240F0E480284604F1EA0100F0B8FD21
:100C700006460028AAD1012384F8E83000F0D0FE0F
:100C8000D4F8E030C01A192840F6B83338BF19201C
:100C9000984228BF1846FFF7CDFB6E49FFF760FA70
:100CA00005462068FFF7C6FB6B49FFF759FA014676
:100CB0002846FFF70FFBFFF715FC20604FF48A7200
:100CC00094F8D930606802FB03F562197B6092F8F2
:100CD000E83053B1D2F8E430E946834215D000231E
:100CE00082F8E830C2F8E030CD4663685B4A9B0A80
:100CF000013313816AE729462046FFF793FD65E734
:100D000029462046FFF7EEFD60E7B2F8EC803B6035
:100D100008F1030A4FEA9A0A4FEA8A02D11DC9086C
:100D2000A9EBC1039D46EB460021584600F036FB77
:100D300005F1EE0142465846214400F01DFB3B6898
:100D400013B9012000F0CCFA94F8D20000F0D2FAE6
:100D5000054630B9207200F0EDFA284600F0C0FADE
:100D6000C2E7D4F8D4303BB994F8D200B4F8F031EB
:100D7000834201D8FFF7E0FED4F8D43043449D42CB
:100D800008D294F8D200B4F8F0310130834201D88F
:100D9000FFF7D2FE594660685FFA8AF200F006FB60
:100DA00008B9CD468AE7636894F8D200434463608B
:100DB000D4F8D43008EB030AC4F8D4A000F09AFAAF
:100DC000824509D394F8D230D4F8D4000133401BC3
:100DD00084F8D230C4F8D400B8F1FF0F0FD8002542
:100DE000257200F0A7FA284600F07AFA00F084FD98
:100DF0001A4B188108B9FFF79BFCCD46E6E64FF485
:100E00008A727B6894F8D90002FB0343D3F8E4208C
:100E100083F8E86002F58072C3F8E060C3F8E4206C
:100E2000FFF7B2FDFFF700FE84F8D960B9E740F69E
:100E3000B8322368FA33934294BF23602260C5E638
:100E4000482100204521002000ED00E00400FA05C3
:100E50007C210020CDCCCC3D6666663F341100205D
:100E6000014B1870704700BF4011002030B54FF0A3
:100E70000054264B226885B09A4217D1637DABB1EE
:100E80000025234A23481370237DC9220372224977
:100E9000C0F8E450093000F06FFA2046E0222946FD
:100EA00000F07CFA0124204605B030BD02F06AFB58
:100EB000044608B90024F6E7184A194DD36943F0EF
:100EC0000073D361AA6D174B9A42F3D12B6E013B8D
:100ED0007E2BEFD8144A01AB07CA83E807001846F7
:100EE000032100F0D9FC6B6D83424FF00003E1D188
:100EF0002A6D8A4203BFAB652A6E054B1C4601BFB3
:100F00001A70EA6D094B1A60CDE700BF9AAD44C56F
:100F1000401100207C21002016000020001002401B
:100F2000006600405041A0B05866004018110020F3
:100F30002DE9F04385B000F0DFFC0223494C6371DA
:100F400000230293484B2081D3F800C0BCF57A7F80
:100F500012D3464F464BB7FBFCF59C458CBF0A238A
:100F60001123B5FBF3F603FB1652591EC8B2002A33
:100F70003ED002290B46F4D89DF80B303D495A1E4D
:100F80009DF80A303C48013B1B0443EA0253BDF87C
:100F90000820013A13434B6001F042FF0023019304
:100FA000364B374900934FF48052364B364800F0A9
:100FB000B5FF364B197811B1334800F0D9FF00F076
:100FC0002FFD0546FFF706FC4FF4C873B0FBF3F2A4
:100FD00002FB130305F516709BB218442C4B1860E6
:100FE00002F0C6FA08B10F23238105B0BDE8F083F3
:100FF000731EB3F5806FBFD24FF47A75C0EBC00E8D
:101000000EF103034FEAE30909FB0555C3F3C703D8
:10101000C11AC9B209F101088844B5FBF8F5B5F564
:10102000617F08D90EF1FF33C3F3C703C11A581EFD
:101030000F28C9B214D84A1E072A8CBF00220122E9
:10104000581800FB0660B7FBF0F7BC4594D1002AA6
:1010500092D0ADF808608DF80A308DF80B108BE750
:101060001346EDE73411002018110020005125022D
:101070003F420F0010110020A8230020B10A0008F1
:10108000441100207D0B00084C210020401100205D
:10109000482100202DE9F04F80A7D7E900670FF223
:1010A0000429D9E90089734D93B00DF1300AFFF797
:1010B000BBFC18220021504600F070F9DFF8B8B1EF
:1010C0006E4C002352461946584601F0E1FE014697
:1010D00050BB102208A800F061F9E36883F0100308
:1010E000E36000F09FFC0DF1240C0B4612A90246B0
:1010F00011E903008CE803009DF83410C1F30300EC
:10110000890649BF0E99BDF83810C1F31C0141F0A2
:10111000004158BFC1F30A018DF82C000891284600
:1011200008A901F0E1F9CCE7284600F029FF0446C0
:10113000002847D100F074FCDFF844B1DBF8003040
:1011400098423FD300F06CFC0790FFF743FB4FF44D
:10115000C873B0FBF3F101FB1300079A83B202F5E9
:1011600016701844CBF80000DFF818B18DF8204055
:101170009BF8001011B901238DF8203050460791DB
:10118000FFF740FB07990DF12100C1F11004E4B213
:10119000062C28BF06245144224600F0EDF808AB87
:1011A000039318230293384B013401930123E4B2D3
:1011B000009332463B462846049400F027FF002364
:1011C0008BF8003000F02CFC304A314C1368C31A05
:1011D000B3F57A7F30D3106000F024FC02460B4652
:1011E000284600F0ABFF284600F0CAFE20B3237A61
:1011F000DFF8A0B0002B14BF032302238BF80530C7
:1012000000F00EFC4FF47A73B0FBF3F00122CBF840
:1012100000005146584600F0BFF9182302931E4BB8
:1012200080B2019340F25513CDE903A000934246EA
:101230004B46284600F0EAFE237ABBB100F0F0FBF3
:1012400094F8E83073B9D4F8E03043B1C01A236899
:10125000FA2B38BFFA230533B0EB430F02D300203B
:10126000FFF792FB237A002B7FF41FAF13B0BDE88A
:10127000F08F00BF4C210020A8230020000801406F
:101280004821002045210020442100207023002017
:101290007C2100203411002074230020401DA12057
:1012A00026812A0BF1C6A7C1D068080F70B501F0DE
:1012B000CDFF0024084E094D3080286833888342D2
:1012C00008D901F0BFFF2B6804440133B4F5C84FBF
:1012D0002B60F2D370BD00BFA42300207823002030
:1012E00002F042B800F10060920000F5C84001F041
:1012F000E7BF0000054B1A68054B1B889B1A834209
:1013000002D9104401F09EBF0020704778230020CE
:10131000A4230020024B1B68184401F099BF00BFB2
:1013200078230020024B1B68184401F0A3BF00BFC4
:1013300078230020064991F8243033B10023082295
:10134000086A81F82430FFF7CDBF0120704700BF45
:101350007C230020022802BF1022014B1A61704733
:1013600000080140022802BF4FF48012014B1A61AD
:10137000704700BF00080140002310B5934203D01E
:10138000CC5CC4540133F9E710BD000003460246AB
:10139000D01A12F9011B0029FAD170470346024402
:1013A000934202D003F8011BFAE770472DE9F84396
:1013B0001F4D144695F824200746884652BBDFF897
:1013C00070909CB395F824302BB92022FF21484619
:1013D0002F62FFF7E3FF95F824004146C0F10802B1
:1013E000A24228BF224605EB8000D6B29200FFF74A
:1013F000C3FF95F82430A41B1E44F6B2082E1744F0
:101400009044E4B285F82460DBD1FFF793FF002815
:10141000D7D108E02B6A03EB82038342CFD0FFF7DA
:1014200089FF0028CBD10020BDE8F8830120FBE72D
:101430007C2300202DE9F3470D4604460021904609
:10144000284640F27912FFF7A9FF23462022002107
:10145000284600F0EBFF022220212846231D00F041
:10146000E5FF032222212846631D00F0DFFF03224F
:1014700025212846A31D00F0D9FF10222821284647
:1014800004F1080300F0D2FF08223821284604F1B5
:10149000100300F0CBFF08224021284604F111037D
:1014A00000F0C4FF08224821284604F1120300F08E
:1014B000BDFF20225021284604F1140300F0B6FF9E
:1014C00040227021284604F1180300F0AFFF0822E3
:1014D000B021284604F1200300F0A8FF0822B8211B
:1014E000284604F1210300F0A1FFC02604F12207E1
:1014F0003B46314608222846083600F097FFB6F5ED
:10150000A07F07F10107F3D194F8323031468DF80E
:101510000730082228460DF1070300F087FF002658
:1015200004F1330A9DF807304FEAC6099E4209F5D7
:10153000A47720D394F83231502B28BF50238DF854
:101540000730B8F1000F08D13946072228460DF1BF
:10155000070300F06BFF09F24F17002604F2331463
:101560009DF8073007EBC6019E420DD30731C8082E
:1015700002B0BDE8F0870AEB060308223946284688
:1015800000F054FF0136CDE7A3190822284600F0E9
:101590004DFF0136E4E7000038B50C460021054652
:1015A00021600346C4F803102046202200F03EFFCD
:1015B00020462B1D0222202100F038FF20466B1D03
:1015C0000322222100F032FF2046AB1D03222521F9
:1015D00000F02CFF20461022282105F1080300F01E
:1015E00025FF072038BD0000F7B5047F05460E46ED
:1015F0002CB1838A122B02D9012003B0F0BD002345
:10160000072219462846009600F0D2FD731C00936D
:10161000012200230721284600F0CAFDD4B9B31CDB
:101620000093052223460821284600F0C1FD0D2421
:10163000B378102BE0D83746B278BB1B934210D357
:101640002B7F0734A88AE408B3B9844294BF0020F2
:101650000120D2E7AB8A0824DB00083BDB08B3702B
:10166000E6E7FB1C2146009308220023284600F0F1
:101670009FFD08340137DFE7201A18BF0120BCE7BF
:10168000F7B5047F05460E462CB1838ACA2B02D9D2
:10169000012003B0F0BD0023082219462846009619
:1016A00000F086FD731CD4B908220093114623462E
:1016B000284600F07DFD10247378C82BE8D801235C
:1016C00072785F1C013B934210D32B7F0734A88AAA
:1016D000E408B3B9844294BF00200120D9E7AB8A63
:1016E0000824DB00083BDB087370E5E7F3192146AB
:1016F000009308220023284600F05AFD08343B4698
:10170000DEE7201A18BF0120C3E70000F7B50D4639
:1017100004460021164628468122FFF73FFE234655
:1017200008220021284600F081FE94F90120637808
:10173000002AB8BF7F238DF807309EB90722082101
:1017400028460DF1070300F071FE0F270026023432
:101750009DF8073007EBC6019E4205D30731C80844
:1017600003B0F0BD0827F1E7A3190822284600F0CE
:101770005DFE0136ECE70000F7B50E460546002198
:1017800014463046CE22FFF709FE2B4628220021C0
:10179000304600F04BFE2B7AC82B28BFC8238DF8AB
:1017A00007308CB90822282130460DF1070300F0DC
:1017B0003DFE30242F469DF807207B1B934205D326
:1017C000E01DC00803B0F0BD2824F3E7214607F16F
:1017D00009030822304600F029FE08340137EAE701
:1017E000F7B5047F05460E4634B1838AB3F5827F90
:1017F00002D9012003B0F0BD0123102200212846A8
:10180000009600F0D5FCDCB9B31C009309222346F6
:101810001021284600F0CCFC19247388B3F5807F92
:10182000E7D837467288BB1B934210D32B7F07340F
:10183000A88AE408B3B9844294BF00200120D9E704
:10184000AB8A1024DB00103BDB087380E5E73B1D0F
:101850002146009308220023284600F0A9FC083402
:101860000137DFE7201A18BF0120C3E730B5094D63
:101870000A4491420DD011F8013B5840082340F32F
:101880000004013B2C4013F0FF0384EA5000F6D122
:10189000EFE730BD2083B8ED4FF0FF33F7B500EB35
:1018A00081061946DFF848C0DFF848E0B0421BD097
:1018B00050F8042B01AF0192042217F8014B81EA82
:1018C000046108240D46DB184941013C002DBCBFD2
:1018D00083EA0C0381EA0E0114F0FF04F2D1013A0D
:1018E00012F0FF02E9D1E1E7D843C94303B0F0BDEC
:1018F0009336EAA9EBE1F042F7B56B46354A10683A
:1019000051686A4603C308233349344802F0E6F8B5
:10191000044690BB0A256B46314A106851686A46F6
:1019200003C308232F492D4802F0D8F804460028A5
:1019300047D00369B3F5CE3F43D8B0F86620B2F57F
:101940008A6F3ED1284A024402F15C018B4238D3AF
:101950005C3B224900209E1AFFF788FF074632466B
:10196000002004F16401FFF781FFA3689F4228D1A2
:10197000E368984208BF002523E00369B3F5CE3F32
:1019800026D8428BB2F58A6F20D1174A024402F161
:1019900010018B4218D3103B104900209D1AFFF70D
:1019A00065FF06462A46002004F11801FFF75EFF96
:1019B000A3689E4202D1E368984201D00D25AAE7B0
:1019C0000025284603B0F0BD1025A4E70C25A2E7AA
:1019D0000B25A0E7503B0008DC9B010000640008D9
:1019E000593B0008909B0100089CFFF7EFF3098327
:1019F000EFF30583014B9B6BFEE700BF00ED00E0BA
:101A000008B5FFF7F3FF0000EFF30983EFF3058359
:101A1000014B5B6BFEE700BF00ED00E0FEE700005E
:101A200001F008BD01F0B4BC2DE9F041456A15B9DB
:101A30004162BDE8F0814B68AC4623F06047C3F3D8
:101A40008A4616EA230638BF3E464FEAD37EC3F3E2
:101A500080782B465A68BEEBD27F22F060440AD0D1
:101A6000002A18DAA40CB44217D19D420FD10D60A0
:101A7000DEE71346EEE7A74207D102F08044C2F347
:101A8000807242450BD054B1EFE708D2EDE7CCF8B5
:101A900000100B60CDE7B44201D0B442E5D81A681B
:101AA0009C46002AE5D11960C3E700002DE9F04704
:101AB0004FF47F49089D01F007044FEAD5082244FE
:101AC00005F0070500EBD100944201D1BDE8F08795
:101AD00004F0070705F0070A57453E4638BF56464B
:101AE000111BC6F108068E4228BF0E46E108415C74
:101AF00008EBD50E13F80EC0B94029FA06F721FA03
:101B00000AF1FFB28CEA010147FA0AF739408CEA80
:101B1000010C03F80EC034443544D5E7082341F2E4
:101B2000210280EA012001B24000002980B203F1C5
:101B3000FF33B8BF504013F0FF03F4D170470000EB
:101B400038B50C468D18A54200D138BD14F8011BDC
:101B5000FFF7E4FFF7E700000346406848B102687A
:101B600099895A605A89013292B291425A8138BF9A
:101B70009A81704770B504460D4688B02022002136
:101B80006846FFF70BFC20460495FFF7E5FF024689
:101B900058B16B46054608AE1C4603CCB4422860DB
:101BA0006960234605F10805F6D1104608B070BDFE
:101BB000082817D909280CD00A280CD00B280CD0DB
:101BC0000C280CD00D280CD00E2814BF402030203B
:101BD00070470C2070471020704714207047182061
:101BE0007047202070470000082817D90C280CD90E
:101BF00010280CD914280CD918280CD920280CD955
:101C000030288CBF0F200E207047092070470A2013
:101C100070470B2070470C2070470D207047000064
:101C20002DE9F843078C0446072F1ED9D0E9029806
:101C300000254FF6FF73C5F12006A5F1200029FA13
:101C400005F108FA06F628FA00F031430143C9B25B
:101C50001846FFF763FF0835402D0346EBD13A469F
:101C6000E169BDE8F843FFF76BBF4FF6FF70BDE8D1
:101C7000F883000010B54B6823B9CA8A63F30902E0
:101C8000CA8210BD04691A681C600361C38A013BE3
:101C9000C3824A60EFE700002DE9F84F1D46CB8A6A
:101CA0000F46C3F309010529814692460B4630D001
:101CB0000020AAB207F11A049EB2042E1FFA80F87F
:101CC0000FD8904503F1010306D3FB8A0A4462F35F
:101CD00009030120FB821AE01AF800600130E65483
:101CE000EAE79045F1D21C23A1F1050BBBFBF3F20F
:101CF00003FB12BB7C681FFA8BF6002C45D14846CB
:101D0000FFF72AFF044638B978606FF00200BDE89B
:101D1000F88F4FF00008E6E70026066078604FF085
:101D2000000BADB2454510D90AEB0803221D13F88C
:101D3000011B08F101089155B1B21B291FFA88F85F
:101D40002BD0454506F10106F1D8FB8AC3F3090201
:101D5000154465F30903BCE71C46013292B22368BF
:101D6000002BF9D16B1F0B441C21B3FBF1F30133A2
:101D70009BB29A42D3D2BBF1000FD0D14846FFF7B5
:101D8000EBFE20B9C4F800B0BFE70122E7E7C0F8D6
:101D900000B05E4620600446C1E74545D5D94846B7
:101DA000FFF7DAFE08B92060AFE7C0F800B0002600
:101DB00020600446B6E700002DE9F74F1C465B693A
:101DC000074688460092002B00F0A480238C2BB19C
:101DD000E269002A00F09E80072B33D807F10C003F
:101DE000FFF7BAFE054628B96FF00205284603B092
:101DF000BDE8F08F14220021FFF7D0FA228CE169B0
:101E000005F10800FFF7B8FA208C48F000410130D6
:101E100080B2FFF7E9FEFFF7CBFE013880B22084E5
:101E2000013028746369228C1B782A4403F01F0355
:101E300063F03F031372384669602946FFF7F4FDEB
:101E40000125D3E7072202339BB20633B3FBF2F33B
:101E5000C18A828A9BB2521A92B29342C4D84FF07E
:101E600000094FF0800A4E464D4600F10C030193E5
:101E70000198FFF771FE83460028B5D01422002197
:101E8000FFF78CFA002E3BD10222009BABF8083002
:101E90000BF1080E1FFA82FC0CF10100BCF1060FD9
:101EA000218C80B201D88E422CD3FFF79DFEFFF724
:101EB0007FFE8E4208BF4FF0400A626901381278F7
:101EC00080B202F01F0242EA49120BEB00014AEA1B
:101ED000020A013048F0004281F808A08BF8100097
:101EE00059463846CBF80420FFF79EFD238C013578
:101EF000B3424FF0000A2DB289F00109B8D175E75D
:101F00000022C5E7E169895D01360EF80210B6B21C
:101F10000132BFE76FF0010568E70000F8B504463D
:101F200015460E46302200211F46FFF737FA069B62
:101F3000B5F5001F6360079B28BF4FF6FF72A362D1
:101F40004FF0000338BF6A09A760E66197B204F159
:101F500010009A4206D800230360A782E3822383FD
:101F6000E360F8BD0660013330462036F1E700003B
:101F700003781BB94BB2002BC8BF0170704700003B
:101F800000787047F8B50C46C969074611B9238C2B
:101F9000002B37D1257E1F2D34D8387828BB228CD2
:101FA000072A2CD8268A36F003032BD14FF6FF7070
:101FB000FFF7C6FD4FF6FF7220F001003602400425
:101FC00046EA0565400C45EA402523462946384641
:101FD000FFF7F2FE002807DD626913780133DBB2F8
:101FE0001F2B88BF00231370F8BD218A2D0645EAF8
:101FF000012505432046FFF713FE0246E5E76FF093
:102000000300F1E76FF00100EEE7000070B5044651
:102010001D4616468AB0282200216846FFF7BEF901
:10202000BDF838306946ADF810300F9B2046059357
:102030009DF84030CDE902658DF81830119B07936B
:10204000BDF84830ADF82030FFF79CFF0AB070BDF6
:102050002DE9F041D36905460C4616460BB9138CA1
:102060005BBB377E1F2F28D895F80080B8F1000F92
:1020700026D03046FFF7D4FD3378210241EAC33140
:1020800041EA0801338A41EA076141EA0341024615
:102090003346284641F08001FFF78EFE00280ADD16
:1020A0003378012B07D1726913780133DBB21F2B10
:1020B00088BF00231370BDE8F0816FF00100FAE7DC
:1020C0006FF00300F7E70000F0B504460D461E462A
:1020D00017468BB0282200216846FFF75FF99DF86C
:1020E0004C3029465A1E534253418DF800309DF81A
:1020F00040306A46ADF81030119B204605939DF89C
:102100004830CDE902768DF81830149B0793BDF85E
:102110005430ADF82030FFF79BFF0BB0F0BD00004E
:10212000406A00B104307047436A1A68426202692B
:102130001A600361C38A013BC38270472DE9F041F5
:10214000D0F8208014461D4641460027174E09B995
:10215000BDE8F081D1E90223A21A65EB03039642A0
:1021600077EB03031ED2036A8B420DD1FFF782FD8A
:10217000036A1B68036203690B60C38A0161016A19
:10218000013B8846C382E2E7FFF774FD0B68C8F89D
:10219000003003690B60C38A0161013BC382D8F838
:1021A0000010D4E788460968D1E700BF80841E008C
:1021B0002DE9F04F8BB00D4614469B468046DDF866
:1021C0005090002800F01A81B9F1000F00F016813C
:1021D000531E3F2B00F21281012A03D1BBF1000FE5
:1021E00040F00C810023CDE90833B8F81430B5EB8A
:1021F000C30F4FEAC30703D300200BB0BDE8F08F35
:102200002B199F42D8F80C3036BF7F1B2746FFB2F0
:102210001BB9D8F81030002B7BD0272D4ED8C5F134
:102220002806B7424FF0000334BF3E46F6B2009393
:1022300029463246D8F8080008ABFFF737FCA7EB71
:10224000060A35445FFA8AFA2821B8F8143003F1F7
:102250000053053BDB000493D8F80C300393039B39
:1022600013B1BAF1000F2CD1D8F8100040B1BAF177
:10227000000F05D05246009608AB691AFFF716FC0E
:1022800038B2002FB8D066070AD00AAB03EBD401EE
:1022900011F8083C624202F00702134101F8083CC1
:1022A000082C3DD9102C40F2B680202C40F2B8808A
:1022B000BBF1000F00F09D80082335E0BA460026F0
:1022C000C2E7049BE02B28BFE02306930B44AB42FC
:1022D000059315D95A1B924538BF5246039828BF1B
:1022E000D2B20096691A08AB04300792FFF7DEFB02
:1022F000079A1644AAEB020A1544F6B25FFA8AFA64
:10230000049B069A05999B1A0493039B1B680393ED
:10231000A5E700933A462946D8F8080008ABADE790
:10232000BBF1000F13D00123B4EBC30F6CD0082C0A
:1023300012D89DF82030621E23FA02F2D50706D586
:102340004FF0FF3202FA04F423438DF820309DF859
:10235000203089F8003050E7102C12D8BDF820301A
:10236000621E23FA02F2D10706D54FF0FF3202FABD
:1023700004F42343ADF82030BDF82030A9F8003034
:102380003BE7202C0FD80899631E21FA03F3DA07E4
:1023900005D54FF0FF3202FA04F40C430894089B71
:1023A000C9F8003029E7402C2BD0DDE90865611E13
:1023B000C4F12102A4F1210326FA01F105FA02F287
:1023C00025FA03F311431943CB0712D50122A4F1D7
:1023D0002003C4F1200102FA03F322FA01F1A24022
:1023E000524243EA010363EB430332432B43CDE9FB
:1023F0000823DDE90823C9E90023FEE66FF00100A8
:10240000FBE66FF00800F8E6082CA0D9102CB3D931
:10241000202CEED8C3E7BBF1000FADD0022383E739
:10242000BBF1000FBBD004237EE70000012A30B5CA
:10243000144638BF01220025402A28BF402285B01B
:10244000012CCDE9025517D81B788DF808305307B9
:102450000AD004AB03EBD20515F8083C544204F053
:102460000704A34005F8083C0346009102A8002198
:10247000FFF71CFB05B030BD082CE5D9102C03D8A4
:102480001B88ADF80830E2E7202C02D81B680293C5
:10249000DDE7D3E90045CDE90245D8E710B5CB68C3
:1024A0001BB98B600B618B8210BD04691A681C60BC
:1024B0000361C38A013BC382CA60F0E703064CBFD5
:1024C000C0F3C0300220704708B50246FFF7F6FFA0
:1024D000022806D15306C2F30F2001D100F00300F9
:1024E00008BDC2F30740FBE72DE9F04F93B0CDE9FB
:1024F00003230A6804461046FFF7E0FF02280CBFDA
:102500000026C2F30626002A0D46824680F2FD818F
:1025100012F0C04940F0F981097B002900F0F581F3
:10252000022803D02378B34240F0F281C2F304635F
:102530001046069302F07F030593FFF7C5FF059B46
:1025400000224FEA8348002348EA0A48294448EA1F
:102550004668CE78CDE90823F309834648EA0008A7
:10256000029367D0059B0246009320465346676856
:1025700008A9B847002800F0CE81276A4FB9414624
:1025800004F10C00FFF7F6FA074690B96FF002006D
:1025900054E03B6998450DD03F68002FF9D1414682
:1025A00004F10C00FFF7E6FA07460028EED0236A94
:1025B0003B60276297F817C006F01F08CCF3840C25
:1025C000ACEB08001FFA80FE0028B8BF0EF1200017
:1025D000A8EB0C031FFA83FEB8BF00B2002B0793D1
:1025E000BEBF0EF120031BB20793D7E9022152EAC6
:1025F000010338D04FF0000C039BDFF800E29A1A79
:10260000049B63EB010196457CEB01032BD36B7BB1
:1026100097F81AE0734519D1029B002B78D0012856
:1026200021DC7868F8B9DFF8D8C1944570EB010374
:1026300016D337E0276A27B96FF00C0013B0BDE856
:10264000F08F3B699845B5D03F68F4E76C489042FD
:102650007CEB010301D30020F0E7029B002BFAD0B2
:10266000079B0F2B17DCFA7DB30002F0030203F087
:102670007C031343FB7539462046FFF7FBFA6B7B5F
:10268000BB76029B3BB9FB7DC3F38402013262F34C
:102690008603FB75D0E76A7BBB7E9A42DBD1029B47
:1026A000002B35D0B309022B32D0039B1422BB6020
:1026B000049B0021FB600DA8FEF770FE039B2046E3
:1026C0000A93049BADF83EB00B932B1D0C932B7B10
:1026D0008DF840A0013BDBB2ADF83C30069B8DF895
:1026E00041808DF84230059B0AA98DF8433094F85B
:1026F0002C3083F001038DF84430A3689847FB7DAC
:10270000C3F38403013303F01F039B02FB82A2E7A0
:10271000FB7DC6F34012B2EBD31F40F0FF80C3F342
:102720008403434540F0FD80029A2B7BB609002AC2
:1027300052D016F0010665D1032B40F2F580039BC1
:102740003946BB60049B04F10C00FB60FB8A66F316
:102750000903FB822B7BAE1D033B3246DBB2FFF746
:102760009BFA00280CDA39462046FFF783FAFB7DF6
:10277000C3F38403013303F01F039B02FB8205E7CD
:10278000AB88DDE908843B834FF6FF73C9F1200075
:10279000A9F1200228FA09F104FA00F0014324FA11
:1027A00002F211431846C9B2FFF7B8F909F1080956
:1027B000B9F1400F0346E9D13146B8822A7B033A8A
:1027C000D2B2FFF7BDF9FB7DB882DA43C2F3C01283
:1027D00062F3C713FB753EE7A6B92E1D013B3246D7
:1027E0003946DBB204F10C00FFF756FA0028BADBD9
:1027F0002A7B3146013AB88AD2B2E2E780841E00D1
:1028000040420F00F98A013BC1F309010429DAB201
:102810005DD80023281D07F11B069A4208D910F83D
:1028200001CB013306F801C001310529DBB2F4D137
:10283000934228BF0023039938BF04330A910499B7
:1028400038BFDBB20B9107F11B010C91796838BFDF
:102850005B190D910E93FB8AADF83EB0C3F30903EB
:102860001A44069BADF83C208DF84230059B8DF84C
:1028700040A08DF8433094F82C308DF8418083F0DF
:1028800001038DF8443000237B602A7BB88A013A2B
:10289000291DFFF755F93B8BB882834203D12046AF
:1028A000A3680AA9984720460AA9FFF7F7FDFB7D10
:1028B000BA8AC3F38403013303F01F039B02FB8234
:1028C0003B8B9A420CBF00206FF01000B6E67B688D
:1028D000002BADD0052001E033461C301E68002ED1
:1028E000FAD1091A081D2E1D184401EB090CBCF180
:1028F0001B0F5FFA89F39BD89A4299D916F8013BCE
:1029000009F1010900F8013BEFE76FF0090095E6D6
:102910006FF00A0092E66FF00B008FE66FF00D008B
:102920008CE66FF00E0089E66FF00F0086E600BFC0
:10293000F0B53F4D3F4FEB6943F00073EB61EB693E
:102940003D4B9B6AD3F800623E4046F00106C3F857
:102950000062D3F800423C4044EA002444F0010401
:10296000C3F80042002955D000200646C3F81C02D7
:10297000C3F80402C3F80C02C3F8140203EBC0044A
:1029800001300E28C4F84062C4F84462F6D1002732
:102990004FF0010C9678148816F0010F18BFD3F889
:1029A00004E20CFA04F01CBF40EA0E0EC3F804E285
:1029B00016F0020F18BFD3F80CE203EBC4041CBFDF
:1029C00040EA0E0EC3F80CE2760748BFD3F8146253
:1029D00007F1010744BF0643C3F814625668B942C1
:1029E000C4F84062966802F10C02C4F84462D3F85D
:1029F0001C4240EA0400C3F81C02CBD1D3F80022E9
:102A000022F00102C3F80022EB6923F00073EB61AE
:102A1000EB69F0BD0122C3F84012C3F84412C3F8B9
:102A20000412C3F81412C3F80C22C3F81C22E5E701
:102A3000001002400000FFFFA8230020184A08B53C
:102A4000916A8B688B6013F0010104D013F00C0FB6
:102A500018BF4FF48031D80506D513F4406F14BF6A
:102A600041F4003141F00201D80306D513F4402FA0
:102A700014BF41F4802141F00401D3690BB108482F
:102A80009847302383F311880021064800F022FB89
:102A9000002383F31188BDE8084000F0ABBD00BF00
:102AA000A8230020B023002038B5124CA36ADD68AB
:102AB000AA0712D05A6922F002025A61A36913B11F
:102AC000012120469847302383F3118800210A48CA
:102AD00000F000FB002383F31188EB0606D51021DC
:102AE000A36AD960236A0BB102489847BDE8384011
:102AF00000F080BDA8230020B823002038B5124C78
:102B0000A36A1D69AA0712D05A6922F010025A61FD
:102B1000A36913B1022120469847302383F311881B
:102B200000210A4800F0D6FA002383F31188EB064F
:102B300006D51021A36A1961236A0BB10248984790
:102B4000BDE8384000F056BDA8230020B82300207F
:102B500038B50F4CA36A5D682A075D600AD5042268
:102B600022701A6822F002021A60636A13B100210F
:102B7000204698476B0706D5A36A9969236A13B163
:102B8000034809049847BDE8384000F033BD00BF52
:102B9000A823002010B50E4C204600F02FF90D4B55
:102BA0000B211320A36200F009F90B21142000F07F
:102BB00005F90B21152000F001F90B21162000F07A
:102BC000FDF8BDE8104000220E201146FFF7B0BE10
:102BD000A8230020006400400F4B10B59842044623
:102BE00005D10E4BDA6942F00072DA61DB6901222D
:102BF000A36A1A60A36A5A68D20707D56268516847
:102C00001268D9611A60064A5A6110BD0121082074
:102C100000F0B0F9EEE700BFA8230020001002404A
:102C20005B87010003291AD8DFE801F0020A0F14BC
:102C3000836A9B6813F0E05F14BF01200020704797
:102C4000836A9868C0F380607047836A9868C0F3AD
:102C5000C0607047836A9868C0F3007070470020B6
:102C60007047000010B5032927D8DFE801F00227DC
:102C70002B2F836A9968C1F30161183103EB0113AB
:102C80001078840648BF5468C0F3001158BF948878
:102C90004FEA410148BF41EAC40100F00F0058600B
:102CA00048BF41F00401906858BF41EA4451D268DE
:102CB00041F001019860DA60196010BD836A03F584
:102CC000C073DDE7836A03F5C873D9E7836A03F548
:102CD000D073D5E701290AD002290FD081B9836AC0
:102CE000DA68920701D1186903E001207047836A0E
:102CF000D86810F0030018BF01207047836AF2E71C
:102D00000020704710B539B9836AD96889071BD18B
:102D10001B699C0704D110BD012915D00229FAD1E5
:102D2000816AD1F8C031D1F8C441D1F8C80110612D
:102D3000D1F8CC015061202008610869800717D1C3
:102D4000486940F0100012E0816AD1F8B031D1F842
:102D5000B441D1F8B8011061D1F8BC015061202014
:102D6000C860C868800703D1486940F00200486124
:102D7000C3F34000C3F38001000140EA4111107920
:102D800020F030000143117189064BBF9168118911
:102D9000DB085B0D4CBF63F31C0163F30A0113797D
:102DA00048BF916064F3030313714FEA14234FEAA1
:102DB000144458BF118113705480ACE701220901FB
:102DC00000F1604303F56143C9B283F8001300F0DA
:102DD0001F039A4043099B0003F1604303F56143DD
:102DE000C3F880211A607047090100F16040C9B240
:102DF00000F56D4001767047FFF7CCBE01230370EC
:102E0000002300F10802C0E9022200F11002C0E92B
:102E10000422C0E90633C0E908334360704700006C
:102E200010B53023044683F31188022341600370F8
:102E3000FFF7D2FE04230020237080F3118810BD19
:102E40002DE9F0411F4604460D461646302383F314
:102E5000118800F108082378052B0DD0294620465B
:102E6000FFF7E0FE40B1204632462946FFF7FAFE62
:102E7000002080F3118808E03946404600F01AF936
:102E80000028E8D0002383F31188BDE8F08100001A
:102E90002DE9F0411F4604460D461646302383F3C4
:102EA000118800F110082378052B0DD02946204603
:102EB000FFF710FF40B1204632462946FFF722FFB8
:102EC000002080F3118808E03946404600F0F2F80F
:102ED0000028E8D0002383F31188BDE8F0810000CA
:102EE00000238268037503691B6899689142FBD2CD
:102EF0005A6803604260106058607047002382681F
:102F0000037503691B6899689142FBD85A6803608E
:102F1000426010605860704708B50846302383F35C
:102F200011880B7D032B05D0042B0DD02BB983F317
:102F3000118808BD00228B691A604FF0FF3383614E
:102F4000FFF7CEFF0023F2E7D1E9003213605A60A9
:102F5000F3E70000FFF7C4BF054BD9680875186890
:102F6000026853601A6001220275D860FDF74ABBFF
:102F7000D823002030B50C4B0446DD684B1C87B0CD
:102F80000FD02B466846094A00F0CAF82046FFF7E2
:102F9000E3FF009B13B1684600F0CAF8A86907B0C8
:102FA00030BDFFF7D9FFF9E7D8230020192F00081B
:102FB000044B1A68DB6890689B68984294BF0020B5
:102FC00001207047D8230020084B10B51C68D86832
:102FD000226853601A6001222275DC60FFF78EFFC1
:102FE00001462046BDE81040FDF70CBBD823002069
:102FF00038B501230025064C064907482370656053
:1030000000F03EFB0223237085F3118838BD00BF1A
:1030100030250020683B0008D823002000F09AB833
:103020008B60022308618B82084670478368A3F196
:10303000440243F8142C026943F8442C426943F8D3
:10304000402C094A43F8242CC268A3F1200043F81D
:10305000182C022203F80C2C002203F80B2C034A34
:1030600043F8102C704700BF15060008D823002035
:1030700008B5FFF7DBFFBDE80840FFF76BBF0000B6
:10308000024BDB6898610F20FFF766BFD823002052
:10309000302383F31188FFF7F3BF000008B5014622
:1030A000302383F311880820FFF764FF002383F3A4
:1030B000118808BD064BDB6839B1426818605A6058
:1030C000136043600420FFF755BF4FF0FF30704797
:1030D000D823002038B504460D462068844200D12C
:1030E00038BD036823605C608561FFF733FFF4E758
:1030F00010B50A4C23699A6891420CD85A688160CD
:103100000360426010609A685860511A99604FF0ED
:10311000FF33A36110BD1B68891AECE7D823002098
:10312000C0E90323002310B410BC4361FFF7E0BFE4
:10313000036881689A680A449A60426813605A601A
:1031400000234FF0FF320360014B9A61704700BFCC
:10315000D823002070B5124D2A46EB690133EB618C
:1031600052F8103F934206D030269A68013A9A608E
:103170002C69A36803B170BDD4E900210A605160D5
:10318000236083F311882046D4E90331984786F3FE
:10319000118861690029EBD02046FFF7A9FFE7E716
:1031A000D8230020054A30B5D369D2E908451B1B56
:1031B000181945F10001C2E9080130BDD8230020EB
:1031C00000207047FEE70000704700004FF0FF301E
:1031D00070470000BFF34F8F024AD368DB07FCD46F
:1031E000704700BF0020024008B5074B1B7853B959
:1031F000FFF7F0FF054B1A69120641BF044A5A60F7
:1032000002F188325A6008BD4825002000200240A3
:103210002301674508B5054B1B7833B9FFF7DAFF83
:10322000034A136943F08003136108BD4825002059
:10323000002002407F289ABF00F500308002002065
:10324000704700004FF48060704700008020704796
:103250007F2808B50BD8FFF7EDFF00F58063026803
:10326000013204D104308342F9D1012008BD00208D
:10327000FCE700007F2810B504461CD8FFF7AAFF22
:10328000FFF7B2FFF3220D4B4FF48061DA600222A8
:103290001A61FFF7CFFF58611A6942F040021A61C4
:1032A000FFF798FF00F02EF9FFF7B4FF2046BDE8C6
:1032B0001040FFF7CDBF002010BD00BF002002402E
:1032C0002DE9F843054612F00100144606D04FF4EC
:1032D000517200201E4B1A60BDE8F8831D4BAA18DE
:1032E0009A4204D940F24932194B1A60F4E7FFF7C9
:1032F0007BFF4FF00109FFF76DFFDFF85C806D1A6F
:10330000012C0F4605EB010603D8FFF783FF0120D0
:10331000E2E73B88C8F8109033800020FFF75AFF9F
:10332000C8F81000338831F8022B9BB29A420CD0B7
:103330004FF45872064B1A60084B1E60084B1C6015
:10334000084B1F60FFF766FFC6E7023CD8E700BFE7
:1033500044250020000002080020024038250020FB
:10336000402500203C250020084908B50B7828B1ED
:103370001BB9FFF739FF01230B7008BD002BFCD0F0
:10338000BDE808400870FFF745BF00BF4825002092
:1033900038B5EFF31185BDBBEFF30584C4F3080422
:1033A0003023C4B183F31188FFF7FCFE44014B01C5
:1033B000241A43EAD06363EB0103A2009B001218B6
:1033C00043EA947341EB0301C900D00041EA527112
:1033D00085F3118838BD83F31188FFF7E3FE4501BB
:1033E0004B012D1A43EAD06363EB0103AA009B0053
:1033F000121843EA957341EB0301C900D00041EA7A
:10340000527184F3118838BDFFF7CCFE44014B01A3
:10341000241A43EAD06363EB0103A2009B00121855
:1034200043EA947341EB0301C900D00041EA5271B1
:1034300038BD00BF38B5FFF7ABFF00230F4A104C73
:10344000C00840EA4170A0FB025EC908A0FB040C62
:10345000A1FB0440A1FB02121CEB050C5B411CEB21
:10346000040C43EB000011EB0E0142F10002411885
:1034700042F10000090941EA007038BDA59BC42053
:10348000CFF753E310B5094C013AD2B2FF2A00D16D
:1034900010BD500854F82030013054F820009BB281
:1034A00043EA004341F8043BEEE700BF046C0040F0
:1034B00010B50748013AD2B2FF2A00D110BD0C88DE
:1034C000530840F823404C88013340F82340F1E78B
:1034D000046C004007B50122002001A9FFF7D2FFCC
:1034E000019803B05DF804FB13B50446FFF7F2FF43
:1034F000A04205D00122002001A90194FFF7D8FFC6
:1035000002B010BD7047000045F25552064B1A60DC
:1035100003225A6040F2FF729A604CF6CC421A6065
:103520000122024B1A7070470030004050250020E5
:10353000034B1B781BB14AF6AA22024B1A60704754
:103540005025002000300040044B1A682AB902F1CF
:10355000804202F50432526A1A6070474C250020FE
:103560004FF08072014B5A62704700BF001002405A
:1035700008B5FFF7E9FF024B1868C0F3407008BDBB
:103580004C25002008B5FFF7DFFF024B1868C0F399
:10359000007008BD4C250020EFF30983203383F32E
:1035A0000988002383F3118870470000302080F3DE
:1035B000118862B60C4B0D4AD96821F4E061090408
:1035C000090C0A43DA60D3F8FC20094942F0807202
:1035D000C3F8FC200A6842F001020A602022DA7770
:1035E00083F82200704700BF00ED00E00003FA05F9
:1035F000001000E0302310B583F311880B4B5B689B
:1036000013F400630FD0EFF309844FF08073203C74
:10361000E36184F30988FFF7CBFC10B1044BA3618D
:1036200010BD044BFBE783F31188F9E700ED00E0E0
:10363000270600082A06000870470000FEE7000081
:103640000A4B0B480B4A90420BD30B4BC11EDA1CA2
:10365000121A22F003028B4238BF00220021FDF72C
:103660009DBE53F8041B40F8041BECE7E43B000844
:10367000D4250020D4250020D4250020FEE700001A
:1036800070B5002504461A4B86B058608562016308
:103690000E46FFF78BFF04F11003C4E904334FF02B
:1036A000FF33A361134BE561D9692B460A462046D7
:1036B000C4E9082304F134018023C4E900440E4A1C
:1036C000A560E5622565FFF7ABFC01230B4AE060CE
:1036D00003750092726868460192B268CDE90223D0
:1036E000074BCDE90435FFF7C3FC06B070BD00BF42
:1036F00030250020D8230020743B0008793B0008C7
:103700007D36000800F030B808B500F063F9FFF727
:103710006FFCBDE80840FFF717BF000070470000CE
:103720004FF0FF310E4B1A6919611A6900221A61B4
:103730001869D868D960D968DA60DA68DA6942F05D
:103740008052DA61DA69DA6942F00062DA61054AC8
:10375000DB69136843F48073136000F01BB900BF8A
:103760000010024000700040194B1A6842F001023C
:103770001A601A689007FCD51A6802F0F9021A60FC
:1037800000225A605A6812F00C0FFBD11A6842F4FA
:1037900080321A601A689103FCD55A6842F4E81224
:1037A0005A601A6842F080721A601A689201FCD559
:1037B0001221084A5A60084A11605A6842F002020F
:1037C0005A605A6802F00C02082AFAD1704700BF0A
:1037D0000010024000641D0000200240084A08B5A5
:1037E000516913680B4003F00103536123B1054A8B
:1037F00013680BB150689847BDE80840FFF7FABE60
:103800000004014054250020084A08B55169136896
:103810000B4003F00203536123B1054A93680BB1D7
:10382000D0689847BDE80840FFF7E4BE00040140B7
:1038300054250020084A08B5516913680B4003F06D
:103840000403536123B1054A13690BB150699847CA
:10385000BDE80840FFF7CEBE00040140542500201B
:10386000084A08B5516913680B4003F00803536117
:1038700023B1054A93690BB1D0699847BDE8084068
:10388000FFF7B8BE0004014054250020084A08B5DF
:10389000516913680B4003F01003536123B1054ACB
:1038A000136A0BB1506A9847BDE80840FFF7A2BE03
:1038B0000004014054250020174B10B55A691C68BC
:1038C000144004F478725A61A30604D5134A936A2B
:1038D0000BB1D06A9847600604D5104A136B0BB140
:1038E000506B9847210604D50C4A936B0BB1D06BF3
:1038F0009847E20504D5094A136C0BB1506C984700
:10390000A30504D5054A936C0BB1D06C9847BDE86C
:103910001040FFF76FBE00BF000401405425002097
:103920001A4B10B55A691C68144004F47C425A6161
:10393000620504D5164A136D0BB1506D98472305E7
:1039400004D5134A936D0BB1D06D9847E00404D5AC
:103950000F4A136E0BB1506E9847A10404D50C4A60
:10396000936E0BB1D06E9847620404D5084A136F6A
:103970000BB1506F9847230404D5054A936F0BB1E0
:10398000D06F9847BDE81040FFF734BE00040140F7
:1039900054250020062108B50846FFF70FFA062136
:1039A0000720FFF70BFA06210820FFF707FA062188
:1039B0000920FFF703FA06210A20FFF7FFF9062185
:1039C0001720FFF7FBF9BDE8084006212820FFF784
:1039D000F5B9000008B5FFF7A3FE054800F00CF8A4
:1039E000FFF70AFAFFF79AFEBDE8084000F002B8B8
:1039F000803B000800F042B8002319461C4A0133FE
:103A0000102BC2E9001102F10802F8D1194B9A6992
:103A100042F07D029A619B690268174BDA60826806
:103A20005A6042681A60C26803F58063DA604269CE
:103A30005A6002691A608269C3F80C24026AC3F8EA
:103A40000424C269C3F80024426AC3F80C28C26A7D
:103A5000C3F80428826AC3F80028026BC3F80C2C50
:103A6000826BC3F8042C426BC3F8002C704700BF74
:103A70005425002000100240000801404FF0E023D0
:103A8000044A08215A6100229A6107220B201A6118
:103A9000FFF7AAB93F19010008B5302383F3118855
:103AA000FFF7BCFA002383F3118808BD08B5FFF7C0
:103AB000F3FFBDE80840FFF79DBD000010B50139D8
:103AC0000244904201D1002005E0037811F8014F33
:103AD000A34201D0181B10BD0130F2E72DE9F041DF
:103AE0009BB10446C91A1778014403F1FF3C8C428C
:103AF000204601D9002008E005780134BD42F6D106
:103B00000CEB0405D618A54201D1BDE8F08115F8EB
:103B1000018D16F801EDF045F5D0E8E7034611F800
:103B2000012B03F8012B002AF9D170476F72672E21
:103B30006172647570696C6F742E4165726F466F47
:103B4000782D41697273706565642D444C5652003E
:103B500040A2E4F1646891060041A3E5F265699230
:103B60000700000063300000643B000830240020A0
:103B7000302500206D61696E0069646C650000008D
:103B800000180000444441444454494401000000EA
:103B900042444444444444440000000044444444F7
:103BA00044444444000000004444444444444444E5
:103BB00000000000444444444444444400000000E5
:103BC0005004000000000000009C01000000000004
:103BD000640000000000000040420F00FE2A0100C7
:103BE000D2040000FFFFFFFFFFFFFFFFFFFFFFFF0B
:103BF000FFFFFFFFFFFFFFFFFFFFFFFFFFFFFFFFD5
:103C0000FFFFFFFFFFFFFFFFFFFFFFFFFFFFFFFFC4
:103C1000FFFFFFFFFFFFFFFFFFFFFFFFFFFFFFFFB4
:103C2000FFFFFFFFFFFFFFFFFFFFFFFFFFFFFFFFA4
:10640000000300204572000865F5000899F40008B3
:1064100021F5000899F40008DDF40008477200082F
:10642000477200084772000847720008B545010826
:10643000477200084772000847720008616B010844
:106440004772000847720008477200084772000848
:106450004772000847720008F568010821690108C1
:106460004D69010879690108A569010839660108C3
:106470004D660108616601087566010889660108B4
:106480009D660108B166010847720008B5E0000882
:10649000E1E00008F1E0000847720008D169010856
:1064A00047720008477200084772000847720008E8
:1064B000477200084772000847720008E947010860
:1064C0001149010847720008477200084772000826
:1064D00047720008B94E0108477200084772000869
:1064E000396A0108477200084772000847720008BD
:1064F0004772000847720008477200084772000898
:106500004772000847720008477200084772000887
:106510004772000847720008477200084772000877
:106520004772000847720008477200084772000867
:106530004772000847720008477200084772000857
:106540004772000847720008477200084772000847
:106550004772000847720008477200084772000837
:10656000D1750008C5BD0008FDE50008BDE90008BB
:10657000FDEE0008B1F60008000000000000000079
:1065800040A2E4F164689106B0320FA22A30AE8CCA
:106590000867010003BEC59300005004FFFFFFFF22
:1065A000FFFFFFFF81F0004102E000BF83F00043E6
:1065B00030B54FEA41044FEA430594EA050F08BF9E
:1065C00090EA020F1FBF54EA000C55EA020C7FEA62
:1065D000645C7FEA655C00F0E2804FEA5454D4EBDF
:1065E0005555B8BF6D420CDD2C4480EA020281EAA9
:1065F000030382EA000083EA010180EA020281EAE1
:106600000303362D88BF30BD11F0004F4FEA013132
:106610004FF4801C4CEA113102D0404261EB410141
:1066200013F0004F4FEA03334CEA133302D05242C7
:1066300063EB430394EA050F00F0A780A4F1010483
:10664000D5F1200E0DDB02FA0EFC22FA05F28018BD
:1066500041F1000103FA0EF2801843FA05F35941A3
:106660000EE0A5F120050EF1200E012A03FA0EFC22
:1066700028BF4CF0020C43FA05F3C01851EBE3714C
:1066800001F0004507D54FF0000EDCF1000C7EEB69
:1066900000006EEB0101B1F5801F1BD3B1F5001FA7
:1066A0000CD349085FEA30004FEA3C0C04F10104C6
:1066B0004FEA445212F5800F80F09A80BCF1004FEF
:1066C00008BF5FEA500C50F1000041EB045141EA71
:1066D000050130BD5FEA4C0C404141EB0101013C3A
:1066E00028BFB1F5801FE9D291F0000F04BF014629
:1066F0000020B1FA81F308BF2033A3F10B03B3F1FB
:1067000020020CDA0C3208DD02F1140CC2F10C028A
:1067100001FA0CF021FA02F10CE002F11402D8BFE8
:10672000C2F1200C01FA02F120FA0CFCDCBF41EAB4
:106730000C019040E41AA2BF01EB0451294330BD83
:106740006FEA04041F3C1CDA0C340EDC04F1140460
:10675000C4F1200220FA04F001FA02F340EA030037
:1067600021FA04F345EA030130BDC4F10C04C4F17D
:10677000200220FA02F001FA04F340EA030029465D
:1067800030BD21FA04F0294630BD94F0000F83F4A7
:10679000801306BF81F480110134013D4EE77FEA8A
:1067A000645C18BF7FEA655C29D094EA050F08BFD6
:1067B00090EA020F05D054EA000C04BF19461046B7
:1067C00030BD91EA030F1EBF0021002030BD5FEAFB
:1067D000545C05D14000494128BF41F0004130BD23
:1067E00014F580043CBF01F5801130BD01F0004577
:1067F00045F0FE4141F470014FF0000030BD7FEAEA
:10680000645C1ABF194610467FEA655C1CBF0B46E4
:10681000024650EA013406BF52EA033591EA030FFB
:1068200041F4002130BD00BF90F0000F04BF0021F3
:10683000704730B54FF4806404F132044FF0000526
:106840004FF0000150E700BF90F0000F04BF00219F
:10685000704730B54FF4806404F1320410F0004505
:1068600048BF40424FF000013EE700BF42004FEA00
:10687000E2014FEA31014FEA02701FBF12F07F437D
:1068800093F07F4F81F06051704732F07F4208BF34
:10689000704793F07F4F04BF41F40021704730B53B
:1068A0004FF4607401F0004521F000411CE700BF87
:1068B00050EA010208BF704730B54FF000050AE00A
:1068C00050EA010208BF704730B511F0004502D50B
:1068D000404261EB41014FF4806404F132045FEA0D
:1068E000915C3FF4D8AE4FF003025FEADC0C18BFB6
:1068F00003325FEADC0C18BF033202EBDC02C2F1A8
:10690000200300FA03FC20FA02F001FA03FE40EA39
:106910000E0021FA02F11444BDE600BF80F00040F1
:1069200002E000BF81F0004142001FBF5FEA410367
:1069300092EA030F7FEA226C7FEA236C6AD04FEA67
:106940001262D2EB1363C1BFD218414048404140AC
:10695000B8BF5B42192B88BF704710F0004F40F45E
:10696000000020F07F4018BF404211F0004F41F47A
:10697000000121F07F4118BF494292EA030F3FD046
:10698000A2F1010241FA03FC10EB0C00C3F1200359
:1069900001FA03F100F0004302D5494260EB4000E8
:1069A000B0F5000F13D3B0F1807F06D340084FEA53
:1069B000310102F10102FE2A51D2B1F1004F40EB48
:1069C000C25008BF20F0010040EA030070474900B0
:1069D00040EB0000013A28BFB0F5000FEDD2B0FA4D
:1069E00080FCACF1080CB2EB0C0200FA0CF0AABF70
:1069F00000EBC25052421843BCBFD040184370470E
:106A000092F0000F81F4000106BF80F40000013213
:106A1000013BB5E74FEA41037FEA226C18BF7FEAEA
:106A2000236C21D092EA030F04D092F0000F08BF2C
:106A30000846704790EA010F1CBF0020704712F013
:106A40007F4F04D1400028BF40F00040704712F152
:106A500000723CBF00F50000704700F0004343F0B7
:106A6000FE4040F4000070477FEA226216BF0846ED
:106A70007FEA23630146420206BF5FEA412390EAB0
:106A8000010F40F4800070474FF0000304E000BFA6
:106A900010F0004348BF40425FEA000C08BF704757
:106AA00043F0964301464FF000001CE050EA01021B
:106AB00008BF70474FF000030AE000BF50EA010230
:106AC00008BF704711F0004302D5404261EB41011D
:106AD0005FEA010C02BF84460146002043F0B64342
:106AE00008BFA3F18053A3F50003BCFA8CF2083A67
:106AF000A3EBC25310DB01FA02FC634400FA02FC70
:106B0000C2F12002BCF1004F20FA02F243EB020076
:106B100008BF20F00100704702F1200201FA02FCD8
:106B2000C2F1200250EA4C0021FA02F243EB0200CB
:106B300008BF20EADC7070474FF0FF0C1CEAD0520F
:106B40001EBF1CEAD15392EA0C0F93EA0C0F6FD0D0
:106B50001A4480EA010C400218BF5FEA41211ED0AE
:106B60004FF0006343EA501043EA5111A0FB01319A
:106B70000CF00040B1F5000F3EBF490041EAD3716F
:106B80005B0040EA010062F17F02FD2A1DD8B3F1EB
:106B9000004F40EBC25008BF20F00100704790F05A
:106BA000000F0CF0004C08BF49024CEA502040EAAC
:106BB00051207F3AC2BFD2F1FF0340EAC250704772
:106BC00040F400004FF00003013A5DDC12F1190FB0
:106BD000DCBF00F000407047C2F10002410021FA22
:106BE00002F1C2F1200200FA02FC5FEA310040F13A
:106BF000000053EA4C0308BF20EADC70704792F0B3
:106C0000000F00F0004C02BF400010F4000F013AEA
:106C1000F9D040EA0C0093F0000F01F0004C02BFE5
:106C2000490011F4000F013BF9D041EA0C018FE754
:106C30000CEAD15392EA0C0F18BF93EA0C0F0AD05A
:106C400030F0004C18BF31F0004CD8D180EA010080
:106C500000F00040704790F0000F17BF90F0004F19
:106C6000084691F0000F91F0004F14D092EA0C0FFB
:106C700001D142020FD193EA0C0F03D14B0218BF8E
:106C8000084608D180EA010000F0004040F0FE40D4
:106C900040F40000704740F0FE4040F44000704770
:106CA0004FF0FF0C1CEAD0521EBF1CEAD15392EAEF
:106CB0000C0F93EA0C0F69D0A2EB030280EA010CDF
:106CC00049024FEA402037D04FF0805343EA111178
:106CD00043EA10130CF000408B4238BF5B0042F1D6
:106CE0007D024FF4000C8B4224BF5B1A40EA0C007B
:106CF000B3EB510F24BFA3EB510340EA5C00B3EBAD
:106D0000910F24BFA3EB910340EA9C00B3EBD10F9A
:106D100024BFA3EBD10340EADC001B0118BF5FEAEC
:106D20001C1CE0D1FD2A3FF650AF8B4240EBC25015
:106D300008BF20F0010070470CF0004C4CEA5020D6
:106D40007F32C2BFD2F1FF0340EAC250704740F425
:106D500000004FF00003013A37E792F0000F00F017
:106D6000004C02BF400010F4000F013AF9D040EA95
:106D70000C0093F0000F01F0004C02BF490011F429
:106D8000000F013BF9D041EA0C0195E70CEAD15321
:106D900092EA0C0F08D142027FF47DAF93EA0C0F08
:106DA0007FF470AF084676E793EA0C0F04D14B02EC
:106DB0003FF44CAF08466EE730F0004C18BF31F09E
:106DC000004CCAD130F000427FF45CAF31F0004398
:106DD0007FF43CAF5FE700BF4FF0FF3C06E000BF31
:106DE0004FF0010C02E000BF4FF0010C4DF804CD54
:106DF0004FEA40024FEA41037FEA226C18BF7FEA64
:106E0000236C11D001B052EA530C18BF90EA010F65
:106E100058BFB2EB030088BFC81738BF6FEAE170F4
:106E200018BF40F0010070477FEA226C02D15FEA90
:106E3000402C05D17FEA236CE4D15FEA412CE1D0FC
:106E40005DF8040B704700BF844608466146FFE7C3
:106E50000FB5FFF7C9FF002848BF10F1000F0FBDA5
:106E60004DF808EDFFF7F4FF0CBF012000205DF89E
:106E700008FB00BF4DF808EDFFF7EAFF34BF012023
:106E800000205DF808FB00BF4DF808EDFFF7E0FFBC
:106E900094BF012000205DF808FB00BF4DF808ED0D
:106EA000FFF7D2FF94BF012000205DF808FB00BF70
:106EB0004DF808EDFFF7C8FF34BF012000205DF852
:106EC00008FB00BF4FEA40024FEA41037FEA226C11
:106ED00002D15FEA402C08D17FEA236C02D15FEA3D
:106EE000412C02D14FF0000070474FF00100704775
:106EF0004FEA4002B2F1FE4F0FD34FF09E03B3EBC7
:106F000012620DD94FEA002343F0004310F0004F06
:106F100023FA02F018BF404270474FF0000070475C
:106F200012F1610F01D1420205D110F0004008BFFB
:106F30006FF0004070474FF00000704753B94AB9F6
:106F4000002908BF00281CBF4FF0FF314FF0FF3071
:106F500000F076B9ADF1080C6DE904CE00F006F84A
:106F6000DDF804E0DDE9022304B070472DE9F047C5
:106F7000089E0D4604468846002B4DD18A42944611
:106F800068D9B2FA82F252B101FA02F3C2F12001D9
:106F900020FA01F10CFA02FC41EA030894404FEA9E
:106FA0001C41B8FBF1F71FFA8CFE01FB178807FBA9
:106FB0000EF0230C43EA084398420AD91CEB030362
:106FC00007F1FF3580F01E81984240F21B81023F9D
:106FD00063441B1AB3FBF1F001FB103300FB0EFE00
:106FE000A4B244EA0344A6450AD91CEB040400F108
:106FF000FF3380F00981A64540F2068164440238DF
:107000000021A4EB0E0440EA07401EB10023D44047
:10701000C6E90043BDE8F0878B4208D9002E00F096
:10702000EE800021C6E900050846BDE8F087B3FA06
:1070300083F100294AD1AB4202D3824200F2FC80A4
:10704000841A65EB030301209846002EE2D0C6E9BE
:107050000048DFE702B9FFDEB2FA82F2002A40F010
:107060009180A1EB0C0001214FEA1C471FFA8CFE16
:10707000B0FBF7F307FB1300250C45EA00450EFBB8
:1070800003F0A84208D91CEB050503F1FF3802D232
:10709000A84200F2CE8043462D1AB5FBF7F007FB5D
:1070A00010550EFB00FEA4B244EA0544A64508D9DB
:1070B0001CEB040400F1FF3502D2A64500F2B680B5
:1070C0002846A4EB0E0440EA03409EE7C1F12007E6
:1070D0008B4022FA07FC4CEA030C25FA07FA4FEA28
:1070E0001C49BAFBF9F820FA07F309FB18AA8D40EE
:1070F0001FFA8CFE1D4300FA01F308FB0EF02C0C66
:1071000044EA0A44A04202FA01F20BD91CEB04043F
:1071100008F1FF3A80F08880A04240F28580A8F113
:1071200002086444241AB4FBF9F009FB104400FB84
:107130000EFEADB245EA0444A64508D91CEB040492
:1071400000F1FF356CD2A6456AD90238644440EAA2
:107150000840A0FB0295A4EB0E04AC42C846AE4624
:1071600056D353D0002E69D0B3EB080264EB0E0463
:1071700022FA01F304FA07F71F43CC40C6E9007472
:10718000002147E70CFA02FCC2F1200125FA01F3C5
:107190004FEA1C4720FA01F195400D43B3FBF7F18C
:1071A00007FB11331FFA8CFE280C40EA034001FB59
:1071B0000EF3834204FA02F408D91CEB000001F13B
:1071C000FF382FD283422DD902396044C01AB0FB58
:1071D000F7F307FB1300ADB245EA004503FB0EF0E1
:1071E000A84208D91CEB050503F1FF3816D2A842C6
:1071F00014D9023B6544281A43EA014138E7314675
:10720000304607E72F46E4E61846F9E64B45A9D293
:10721000B9EB020865EB0C0E0138A3E74346EAE739
:10722000284694E74146D1E7D0467BE764440238DC
:1072300047E7023B65442FE7084606E73146E9E6A3
:10724000704700BF02E000F000F8FEE772B6264883
:1072500080F30888254880F3098825482549086077
:10726000022080F31488BFF36F8F0FF01BF90FF02B
:10727000CDFA4FF0553020491B4A91423CBF41F8AE
:10728000040BFAE71D49194A91423CBF41F8040B2F
:10729000FAE71B491B4A1C4B9A423EBF51F8040BAC
:1072A00042F8040BF8E700201849194A91423CBF04
:1072B00041F8040BFAE70FF0F9F80FF0A9FA154CB2
:1072C000154DAC4203DA54F8041B8847F9E700F087
:1072D0006FF9124C124DAC4203DA54F8041B884784
:1072E000F9E70FF0E1B8000000030020000D0020D6
:1072F0000064000808ED00E0000100200003002009
:1073000088CA0108000D0020800D0020800D00209B
:10731000E4300020606500087865000878650008A2
:10732000786500082DE9F04FC1F80CD0C3689D4680
:10733000BDE8F08F002383F311882846A047002082
:107340000EF066FCFEE70EF02DFB00DFFEE700000E
:1073500010F8012B11F8013B012A28BF9A42F7D0FF
:10736000D01A7047034613F8012B002AFBD1181AD4
:10737000013870477047000070B50446183004F0BB
:107380006BFE04F13C0004F0F1FF04F5A27005F07F
:107390009BFE144B144914261960002304F5DA707F
:1073A0009DB206FB0512127C0133002AF8D10F4B67
:1073B0000F4A1D80136813B10E4808F0D7F810600B
:1073C0000122C4F8C43B84F8C22B04F6C83007F08D
:1073D00069F9094B1A680AB10848EEE71C602046B3
:1073E00070BD00BF041A0020FC780108001A0020BC
:1073F000C819002024780108800D00203F7801087A
:1074000038B504460FF004F80FF016F820231F4D8E
:107410001A4628684FF4E131006C02F0A1F928689F
:107420004FF4807380224FF4E131C06C02F098F980
:10743000204600F0F1F80EF0FFFF204601F03AF888
:1074400004F1180004F0C4FE0EF0F6FF06F010F888
:107450002B68D86A03685B68984710B10C4807F03E
:1074600011FB04F13C0005F06FF9012006F028FF44
:1074700030B1002006F0FCFEBDE8384008F09EB8B0
:1074800004F5A27005F050FFF6E700BF9C0D002048
:10749000607801080148FFF7B3BF00BFA00D0020CE
:1074A00010B50F4C03F08AFE23680522986A00216C
:1074B0000368DB69984723686421986A03681B693D
:1074C000984723682821986A03685B68984723686F
:1074D0000021BDE81040986A03681B69184700BF87
:1074E0009C0D002038B5054608F068F8234A04468C
:1074F0001368C31AB3F57A7F08D9214B10601B7843
:1075000023B9204AD36883F01003D36005F0D8FD77
:1075100041F288311C4A1368E31A8B4206D901688C
:1075200021B114600289194801F05AF8AB7A9B071F
:1075300009D4174A1368E31A132B1DD82846BDE84F
:10754000384001F0D1B808F039F843F69823984252
:10755000EFD91048FFF7A4FF0F480EF0B9FEBFF3B4
:107560004F8F0E490E4BCA6802F4E0621343CB60A2
:10757000BFF34F8F00BFFDE71460DFE7840D0020ED
:10758000000D002000080140880D002080780108CF
:107590008C0D0020A00D0020010007B000ED00E0E0
:1075A0000400FA050148FFF79DBF00BFA00D0020B1
:1075B00038B50546044B0A461868294603681C6816
:1075C000024BA047002038BD9C0D0020900D0020EC
:1075D00010B50A4C2046FFF7CFFE094A094920465C
:1075E0000FF0F4FA07F082FC074B084A18600849CC
:1075F0000848BDE8104001F0D1BF00BFA00D002039
:10760000C8240020757300089C0D0020A575000893
:1076100095740008900D002013B5044604F02EFA6E
:1076200003F0D0FA204604F0A7F918B1B4F90030FD
:10763000022B0BD004F0B6FC02F09AFF0223204686
:107640000DF10601ADF8063004F046FC0223204699
:107650000DF10601ADF8063004F034FC02B0BDE8CF
:10766000104003F06BBE0000F0B500F5A2750446B3
:1076700090F8A611ADB0284605F098FE002847D036
:1076800007F09CFFD4F8C031C31A312B40D9C4F89D
:10769000C001284605F0A4FE284694F8A61105F07E
:1076A0008FFE002834D094F8A611284605F0B4FEC9
:1076B00094F8A611074606AA284605F043FE184E80
:1076C00040B318490698FFF72FF9054660220021BC
:1076D00014A8069510F016F8199507AD0122294651
:1076E00014A81596179618961A96169701F038F959
:1076F00000231822049340F2034380B2CDE90250E4
:10770000CDE9003204A3D3E90023204600F046FA75
:107710002DB0F0BD3546D9E7DAF522A18BF37DC750
:107720000000C07F33938843BFF34F8F0549064B5A
:10773000CA6802F4E0621343CB60BFF34F8F00BF0F
:10774000FDE700BF00ED00E00400FA0510B50446B7
:10775000006810B103685B689847204610BD0000C0
:10776000102213B5044600218DF807200FF0CAFF40
:10777000054B21461B680DF10702D86A03681B6B95
:10778000984702B010BD00BF9C0D0020F0B58BB033
:10779000174604460E4607F011FF054602F068FB47
:1077A0004FF4C873B0FBF3F202FB130305F5167533
:1077B0009BB22B44C4F8BC3BFD7E35B91E4807F094
:1077C00061F984F8C05B0BB0F0BD384605A901F043
:1077D00015FB07460028F6D101A8FFF7C1FF9DF869
:1077E000165001A92A460DF117000FF06DFF28B1C0
:1077F000124807F047F984F8C07BE4E70F2D0CD856
:10780000D4F8BC3B2946A3F5167384F8C05BC4F8D2
:10781000BC3B0B4807F036F9D5E79DF8141000295A
:10782000D1D030460CF0DEF99DF8142094F8C21B3C
:10783000044807F027F9C6E7D8790108037A010858
:10784000247A0108467A010807B5104601A901F01B
:1078500083F958B9074B9DF804101B68A1F1FF028A
:10786000D86A5142036851411B68984703B05DF8DC
:1078700004FB00BF9C0D00202DE9F04317463D4A54
:107880001E461368884613F001033B4C85B007D1B0
:1078900023600123204613603849394A0FF096F9D6
:1078A0002568BDB90422374B29461B685868036810
:1078B000CDE900523822D3F80090334BC8472368F3
:1078C000039520601BB11A6818465268904703A8B8
:1078D000FFF73CFF2068002503684FEAD8089B6A41
:1078E000984740F23522014603A801F0B1FE206816
:1078F0000021036848F04008DB6C98473F2320686C
:107900008DF80B3003680095D3F810900DF10B0142
:107910002B460122C84720688DF80B80036800952C
:10792000D3F810800DF10B012B460122FF08C04750
:1079300047F0600720688DF80B70036800951F6999
:107940000DF10B012B460122F608B84766F07F06C1
:1079500020688DF80B600368009501221C690DF109
:107960000B012B46A04703A801F078FE05B0BDE847
:10797000F08300BF80190020A81900204D7700086F
:10798000C82400209C0D0020801A06002DE9F04735
:1079900096B0804601A9104601F08CF807460028F1
:1079A00054D1DFF8B0909DF80420FBB29A424DD933
:1079B00016AA02EB830313F8524C13F8515C13F828
:1079C000506C98F90800E400AD00F6006428E4B2B9
:1079D00005F0F805F6B231D000282FDBFFF758F894
:1079E0004946FFF7A9F882462046FFF751F851466D
:1079F000FFF7A2F8FFF77CFAFF22002100B202F0A5
:107A00002DFAC4B22846FFF743F85146FFF794F821
:107A1000FFF76EFAFF22002100B202F01FFAC5B292
:107A20003046FFF735F85146FFF786F8FFF760FA62
:107A3000FF22002100B202F011FAC6B233462A46F4
:107A400021464046FFF718FF0137ACE716B0BDE806
:107A5000F08700BF0AD7233C38B5084615461C46B8
:107A60000CF0C8F860B99DF81030022B07D1012C3A
:107A700005D11FA3D3E900230120C5E9002338BDA8
:107A80000B2C0BD8A4B1601E0A2811D8DFE800F037
:107A9000121010101A10101010221E0040F239435C
:107AA0009C421FD040F24C439C4217D0282C05D05A
:107AB0000020E4E710A3D3E90023DDE710A3D3E916
:107AC0000023D9E710A3D3E90023D5E710A3D3E916
:107AD0000023D1E710A3D3E90023CDE710A3D3E916
:107AE0000023C9E710A3D3E90023C5E7AFF3008063
:107AF000401DA12026812A0B9E6AC421818A46EE60
:107B000026417272DF25D7B7F017304A39059E56E5
:107B1000D5A4D139F922B6A7CDD269EBC51A133B4A
:107B200003806A5575F30087C41EDD8B3CD9312074
:107B300013B59DF81040CDE9003413460A460146BE
:107B4000806AFFF789FF02B010BD000070B5D0F861
:107B5000B84B06460D467CB90C2101200EF0B6FA52
:107B6000C6F8B80B08B9002070BD05608460043009
:107B7000FAE72646A46824B12368AB42F9D1201D58
:107B8000F2E70C2101200EF0A1FAB0600028EAD043
:107B90000560B3689C60B068E9E700002DE9F0413A
:107BA00090B0BDF8587000F6C8310446164601A8DA
:107BB00040F24342984601F02FFD012F0ED120469E
:107BC00046EA0741FFF7C2FF054670B9002401A845
:107BD00001F044FD204610B0BDE8F08104F5E270EC
:107BE0000CF008F80028EAD1F0E73822002102A8BA
:107BF0000FF088FD02238DF808309DF85C30CDE948
:107C000004688DF82030189BADF818700993BDF802
:107C100064300795ADF8283007F0D2FC074BC01848
:107C200041F10001CDE90C0104F5E27002A90BF06D
:107C3000E3FF0028D4BF00240124C8E740420F001E
:107C400030B514468FB00D463822002168460FF03B
:107C500059FDDDE91223CDE90223BDF85030ADF81E
:107C6000103004F119030593A37E8DF81830159B8D
:107C70000793BDF85830ADF8203007F0A1FC084B51
:107C80006A46C01841F10001CDE90A012846E17EAB
:107C90000BF0F6FF0028D4BF002001200FB030BD4C
:107CA00040420F00F0B591B004460E46104608A9B8
:107CB000154601F06BF988BB9DF82030012B11D1DE
:107CC00004F070F902F054FC03F038FB03F0D6FE28
:107CD000164904F13C0003F009FE154904F5A270B1
:107CE00003F004FE102200210CA80FF00BFD01226E
:107CF00006AF39460CA88DF8382001F06BF90A233D
:107D000080B2CDE903700293314606A3D3E9002384
:107D10002046CDE900232A46FFF792FF11B0F0BDBF
:107D2000AFF30080CDD269EBC51A133B207E01086A
:107D30004C7F01082DE9F041ADF5487D66AC054664
:107D40000E46174600214FF4C47220460FF0DAFCAD
:107D500007F034FC4FF47A72B0FBF2F02D4B186050
:107D600093E8070084E8070001F0C6FA037C237457
:107D700001F0C2FA437C0DF5DD7063740323A37434
:107D8000254B5A6962619A68DB68A261E361FFF77B
:107D9000E7FC45F20403EA682384204B002A1868B4
:107DA0001F4B29DDCDE900320DF2CB2150221D4BB6
:107DB000C06A01F071FD50210DF2CB200FF00EFDD5
:107DC0000DF11C08414684F832010122204600F0E2
:107DD000DDFE012380B2CDE90380029331460BA37F
:107DE000D3E900232846CDE900233A46FFF728FFD0
:107DF0000DF5487DBDE8F081009350220A4B0DF24D
:107E0000CB21C06A01F048FDD5E700BF9E6AC421BE
:107E1000818A46EE84190020806500089C0D0020B0
:107E20006B7A0108647A010840C301082DE9F0412A
:107E30001546ADF5866D06460F460EF0FDFA28464E
:107E400008A901F0DDF80446002840F09F800146B3
:107E50004FF4D072A4A80FF055FC9DF8B880B8F18B
:107E6000100F7ED808F1FF330F2B2BD842460DF1AF
:107E7000B9010DF2D1300FF037FC424651490DF1F6
:107E8000B9000FF083FC0246B0B94F480DF11F0155
:107E900003F084F80446002C63D09DF8B83073B327
:107EA0009DF828305BB39DF81F20013A032A6DD856
:107EB000DFE802F01C2E384122460DF11F010DF2C1
:107EC000D130E5E7BDF8200047AA0DF11F01479426
:107ED00003F010FC0446002843D001230DF2D132F8
:107EE000009347A9112302F095FFD4E7012B4DD150
:107EF0000C9B204647A98DF81C3103F0D1FF9DF85B
:107F00001F30013B032B41D8DFE803F01C444A4FEC
:107F1000012B3BD10C9B204647A9ADF81C3103F047
:107F2000F3FFECE7012B31D10C9B204647A9479387
:107F300004F028F8E3E7022B28D120460CA903F02F
:107F400071FFDCE701238DF8903294F90030DA17E5
:107F5000CDE9A6325C210DF2D1300FF03FFC8DF857
:107F6000D00347AC01222146A4A801F071F90B23EC
:107F700080B2CDE903400293394610A3D3E9002330
:107F80003046CDE900232A46FFF75AFE0DF5866DEF
:107F9000BDE8F08101238DF89032B4F90030D6E7C6
:107FA00001238DF890322368D1E702238DF89032B7
:107FB0002368A693CEE700BFAFF30080D5A4D139E4
:107FC000F922B6A7907A0108997A01082DE9F04FB5
:107FD0000446DFF8C490DFF8C4A089B004F5E27865
:107FE00040460BF089FE0646002851D00025007E51
:107FF000CDE905550495ADF81C5001F093FA327E99
:1080000006F110018DF81C0005A80FF06DFB336818
:1080100043F00043049307F0D3FA214B0646C218FD
:10802000D9F804000F4641F1000338B30168009508
:1080300009698C4604A9E047A8421FDCD9F804006E
:1080400003689B6A9847D0E90A23CDE9022307F029
:10805000B7FADDE90223801A61EB0301824575EB73
:1080600001030BD394F8C13B072B0ED932463B4694
:10807000404684F8C15B0BF04DFE09E040460BF032
:108080003FFE002384F8C13BA8E7013384F8C13BDD
:1080900009B0BDE8F08F00BF901900207F841E005A
:1080A00040420F004FF000532DE9F041DFF8D4803B
:1080B0001B68054643450C461646FCB004D0DC223E
:1080C000002131480FF01EFB4FF000573046C7F833
:1080D000008049A900F0DEFE002849D19DF8243136
:1080E0003B750BB9F37E3B759DF825210DF593711A
:1080F00026480FF0F9FA20460BF07CFD4FF00053B4
:1081000007AF58758122002128A80FF0FBFA3946E5
:10811000012228A800F004FF282380B2CDE90370D3
:108120000293214615A3D3E900232846CDE9002375
:108130003246FFF785FD3326154F013E16F0FF0648
:10814000284608D0FFF742FF3B680121986A036880
:108150005B689847F1E7FFF7A3F920460BF04AFD6B
:1081600040F0304040F400200EF0B2F8FFF7DCFAA7
:108170007CB0BDE8F08100BFAFF300802641727291
:10818000DF25D7B79AAD44C50400002016000020B3
:108190009C0D0020F0B5054689B008460E461446F1
:1081A0000BF028FD68B9237E022B23D1E38A012B33
:1081B00020D122463146284609B0BDE8F040FFF7FD
:1081C000E5BAE38A0B2B0BD8A3B1013B0A2B11D8DC
:1081D000DFE803F0121010102210101010494100B7
:1081E00040F2394293424ED040F24C42934242D048
:1081F000282B09D009B0F0BD22463146284609B0E7
:10820000BDE8F040FFF796BD22463146284609B04A
:10821000BDE8F040FFF746BF224806F033FC0122DC
:1082200007AF394606A88DF8182000F089FD052310
:1082300080B23146CDE903700293284617A3D3E9F3
:108240000023CDE900232246FFF7FAFC07F0B6F938
:10825000C5F8C40BCEE722463146284609B0BDE832
:10826000F040FFF7E3BD22463146284609B0BDE89D
:10827000F040FFF717BD22463146284609B0BDE859
:10828000F040FFF7E1BA22463146284609B0BDE882
:10829000F040FFF77BBB00BFAFF30080F017304A20
:1082A00039059E56A47A01080A460146806AFFF7FE
:1082B00071BF00002DE9F0470024DFF8988092B0EC
:1082C000D8F804300546CDE907440694ADF82440BB
:1082D000002B3CD04FF0010900260027D8F80400FD
:1082E0008DF80C908DF80D400368CDE900670DF115
:1082F0000D02D3F808A003A90023D0479DF80C3045
:108300002BB3202200210AA80FF0FCF9D8F80400B2
:1083100004AA036806A9D3F814A00DF10E03D047F0
:10832000002814DD9DF8240001F018F907A9024681
:108330008DF840000EA80FF0D7F9069B0AA90A9302
:1083400005F5E270DDE904230BF00AFFC6E712B081
:10835000BDE8F0879019002007B500F5E271684686
:108360000BF0BCFE6423BDF804005843BDF8003098
:10837000B0FBF3F080B203B05DF804FB70B588B0D9
:10838000044607F01BF94FF47A73B0FBF3F0154B7A
:10839000154D1B682860D86A06AE03685B6D984768
:1083A0004FF6FF73984228BF1846314628810122B4
:1083B000284600F09DFC00231822049340F2551338
:1083C00080B2CDE90260CDE9003204A3D3E90023F5
:1083D0002046FFF7E3FB08B070BD00BFF1C6A7C1A0
:1083E000D068080F9C0D00208419002070B5044649
:1083F0008CB000F5E2700BF0FDFB2C4E20B1002399
:10840000012033700CB070BD07F0D8F83378054602
:108410003BB12046FFF7A0FF01210246244806F0A9
:1084200031FB01F025FD4FF4C873B0FBF3F202FB02
:10843000130305F516709BB2184400238DF818300D
:1084400094F8C03BC4F8BC0B23B9012284F8C23BAA
:108450008DF8182008A8FFF783F994F8C01B08AB23
:10846000C1F11005EDB2062D28BF062519442A4694
:108470000DF119000FF038F906AB0026182202930F
:1084800001230135EDB2CDE9003206A3D3E9002383
:10849000204604960395FFF781FB304684F8C06BB5
:1084A000B0E700BF401DA12026812A0B000D00204F
:1084B000B47A01087FB54FF48073234D0446AB8036
:1084C00007F07CF84FF47A73B0FBF3F02860628811
:1084D000B4F902301D4E7F2A98BF337000230DF18E
:1084E0000F0104F109008DF80F3003F0D9FC4FF4AF
:1084F000A76000F005FF054608B105F057FA002215
:10850000134B1D60134B5D601A702DB12B68012257
:1085100028465B68616898470F4B04F5E275009345
:1085200004F5FA7140F6C41228460C4B01940BF086
:108530002DFB317829B1284604B0BDE870400BF01E
:1085400051BB04B070BD00BF84190020AC190020DD
:108550009819002090190020317B0008A98200089A
:1085600070B50C461546062898BF1B4BC4B098BF83
:108570001E5C4FF07C024FF0000125A888BF00264A
:108580000FF0C0F82B4622465A210DF1B60006F036
:1085900037FA5A2828BF5A2006AC21468DF8B50074
:1085A000012225A88DF8946000F0D4FB0023182246
:1085B000049343F6FF7380B2CDE90240CDE9003267
:1085C00003A3D3E900230548FFF7E8FA44B070BDE0
:1085D000759D040C8EA454D6707B0108A00D00205C
:1085E0000FB407B504AA52F8041B07200192FFF745
:1085F000B7FF03B05DF804EB04B0704737B504462D
:1086000000F5E2700BF086FB2046FFF7A5FE46283A
:1086100002D92B4806F036FA2046FFF7AFFE94F950
:108620000950002D38D0002304F10900EDB201A952
:108630008DF8043003F034FC2A2D224C0AD1224D4F
:108640002846FFF7CDFF23686421986A03685B68BA
:108650009847F5E72B2D04D11C48FFF7C1FF1C4BB1
:1086600098474FF4FA6101A800F0BCFF24684FF46A
:108670007A71A06A03685B689847E06A03689B6A3E
:10868000984718B1012816D0124800E01248FFF7A9
:10869000A7FF01A800F0B2FF0022104B5A7106F0AC
:1086A0008DFF47F23053984207D90D4803B0BDE81B
:1086B00030400DF00DBE0B48E9E703B030BD00BF00
:1086C000EC7A01089C0D00200A7B01081B7B010845
:1086D00038ED00E0567B01082B7B0108841900204F
:1086E000263A09B0407B0108F7B5044606F066FF5C
:1086F000394905460B68C31A322B1AD9374B1B78F8
:10870000BBB1012336480278934023F4AA4323F0F7
:1087100055031B041B0C002B0EBF01260026102343
:10872000013243EA06532F4E02F01F0233610270FA
:108730000D6006F043FFD4F8BC3B984202D92046B6
:10874000FFF754FE284A1368EB1AB3F57A7F07D374
:10875000156006F035FF02460B462046FFF74EFF38
:10876000204600F051F82046FEF77EFF06F024FF79
:1087700005461E4F04F6C83606F01EFF401BB0F536
:108780007A7F16D23B684FF48061986A03689B68D1
:10879000984740F2D772314601A800F03DFF2046CD
:1087A000FFF714FC2046FFF785FD01A800F056FFF7
:1087B000E2E7D4F8C43B63B106F000FFD4F8C43B51
:1087C000C01AB0F57A7F04D92046FEF769FEFEF79D
:1087D000ABFF03B0F0BD00BFA0190020000D0020CA
:1087E000A4190020000801409C1900209C0D0020C5
:1087F00010B590F80511044603F0F0FD6423C0B2F3
:1088000003FB0044A06E10BD70B590F941300446E2
:108810009EB0002B51D090F83F31002B4DD006F088
:10882000CDFED4F8B831C01A272846D904F13C054A
:10883000284603F0FDFD2846D4F8B861FFF7D8FFBD
:1088400086423AD0284694F8411103F0EBFD002807
:1088500033D02846FFF7CCFF94F84111C4F8B80193
:10886000284603F0BBFDC1B2642000FB0141164A5B
:10887000983107A801F014FB2822002114A80EF05B
:1088800041FF079B0AAD1193089B01221293099B9C
:10889000294611A8139300F019F800231822049315
:1088A00040F2E93380B2CDE90250CDE9003204A3B1
:1088B000D3E900232046FFF771F91EB070BD00BF59
:1088C000F2C20B46A9D4A7E26F12833A2DE9F34115
:1088D0000E46044617460021192230460EF012FFBC
:1088E0000025A4F1040858F8040F0BF0FFFB2946FB
:1088F000ADF80600102230460DF1060310350BF0DE
:10890000A5FB302DEFD1237B092B28BF09238DF840
:1089100005303FB92946042230460DF105030BF01E
:1089200095FB34254FF0000810349DF8053005EB19
:108930000817984504D3F81DC00802B0BDE8F081BF
:1089400054F8040B0BF0D2FB1022ADF806003946A8
:1089500030460DF106030BF079FB08F10108E4E75E
:108960002DE9F3410D4604460021164628463222E1
:108970000EF0C8FE23460822002128460BF066FBB5
:10898000202208212846231D0BF060FB20222821ED
:1089900004F1080328460BF059FBE0680BF0A6FB36
:1089A000102248210DF10603ADF8060028460BF011
:1089B0004DFB20690BF09AFB102258210DF10603A4
:1089C000ADF8060028460BF041FB60690BF08EFB0A
:1089D000102268210DF10603ADF8060028460BF0C1
:1089E00035FBA0690BF082FB0DF10603ADF8060024
:1089F0001022782128460BF029FB237F102B28BF5B
:108A000010238DF80530AEB90522882128460DF1D6
:108A100005030BF01BFB4FF08D08002720349DF859
:108A2000053008EB07169F4207D3F01DC00802B0BF
:108A3000BDE8F0814FF08808EFE754F8040B0BF025
:108A400055FB1022ADF80600314628460DF106030D
:108A50000BF0FCFA0137E2E7F7B50C46154606467F
:108A600000920023082209680BF0B0F921686F1CFE
:108A70000831216000970023052230460BF0A6F94B
:108A80002168AF1C05312160002306223046009783
:108A90000BF09CF92168033506310023052230468E
:108AA000216000950BF092F90020236805332360C4
:108AB00003B0F0BDF0B5067F05460C4685B02EB17B
:108AC000838A3D2B02D9012005B0F0BD002303931A
:108AD000002E3BD1334605223146284600940BF048
:108AE00075F9039B053303932378142BEBD8671C8C
:108AF00023789E421BD23A46284603A9FFF7ACFFD3
:108B000004370028DFD10136F2E7013FDBD02278BD
:108B1000284604EB8202013203A9FFF79DFF0028DB
:108B2000D1D1237801332370039B9E42EDD8039B60
:108B30002A7F0733A88ADB0822B9834294BF00202A
:108B40000120C1E7181A18BF0120BDE72370AE8AC3
:108B50001527F600073EE7E713B50446007F10B17E
:108B6000A38A012B0CD80023009108221946204625
:108B70000BF02CF9237FA08A23B9B0FA80F04009CA
:108B800002B010BD013818BF0120F9E72DE9F34705
:108B90000D46044600219046284640F279120EF018
:108BA000B1FD23462022002128460BF04FFA022275
:108BB00020212846231D0BF049FA032222212846B2
:108BC000631D0BF043FA032225212846A31D0BF059
:108BD0003DFA10222821284604F108030BF036FA4A
:108BE00008223821284604F110030BF02FFA08223E
:108BF0004021284604F111030BF028FA08224821ED
:108C0000284604F112030BF021FA202250212846B5
:108C100004F114030BF01AFA40227021284604F1E3
:108C200018030BF013FA0822B021284604F12003A0
:108C30000BF00CFA0822B821284604F121030BF0AE
:108C400005FAC02604F122073B4631460822284691
:108C500008360BF0FBF9B6F5A07F07F10107F3D159
:108C600094F8323031468DF80730082228460DF14D
:108C700007030BF0EBF9002604F1330A9DF80730E7
:108C80004FEAC6099E4209F5A47720D394F8323101
:108C9000502B28BF50238DF80730B8F1000F08D1B2
:108CA0003946072228460DF107030BF0CFF909F2E8
:108CB0004F17002604F233149DF8073007EBC60166
:108CC0009E420DD30731C80802B0BDE8F0870AEB19
:108CD00006030822394628460BF0B8F90136CDE7DD
:108CE000A319082228460BF0B1F90136E4E7000089
:108CF00038B50C460021054621600346C4F8031030
:108D0000204620220BF0A2F920462B1D0222202112
:108D10000BF09CF920466B1D032222210BF096F9E3
:108D20002046AB1D032225210BF090F9204610228E
:108D3000282105F108030BF089F9072038BD000050
:108D400008B5034608460021012201700BF07EF9A8
:108D5000012008BD2DE9F3410D46044600211646C9
:108D600028467B220EF0CEFC234603220021284613
:108D70000BF06CF9637805221F2B28BF1F230321FA
:108D80008DF8063028460DF106030BF05FF901233C
:108D90009DF80620DF0003F10108013B9A421CD830
:108DA00094F821305A2B28BF5A238DF807303EB94A
:108DB0003946072228460DF107030BF047F907371C
:108DC000002622349DF8073007EBC6019E420DD3E2
:108DD0000731C80802B0BDE8F08104EB080308229F
:108DE000394628460BF032F94346D1E7A319082249
:108DF00028460BF02BF90136E4E70000F7B5047FB5
:108E000005460E462CB1838A122B02D9012003B0ED
:108E1000F0BD002307221946284600960AF0D6FF27
:108E2000731C009301220023072128460AF0CEFF7D
:108E3000D4B9B31C009305222346082128460AF022
:108E4000C5FF0D24B378102BE0D83746B278BB1B92
:108E5000934210D32B7F0734A88AE408B3B9844225
:108E600094BF00200120D2E7AB8A0824DB00083B36
:108E7000DB08B370E6E7FB1C2146009308220023C1
:108E800028460AF0A3FF08340137DFE7201A18BF8D
:108E90000120BCE7F7B5047F05460E462CB1838A56
:108EA000CA2B02D9012003B0F0BD002308221946C5
:108EB000284600960AF08AFF731CD4B90822009352
:108EC0001146234628460AF081FF10247378C82BE8
:108ED000E8D8012372785F1C013B934210D32B7FAB
:108EE0000734A88AE408B3B9844294BF0020012063
:108EF000D9E7AB8A0824DB00083BDB087370E5E7A1
:108F0000F319214600930822002328460AF05EFF49
:108F100008343B46DEE7201A18BF0120C3E70000F3
:108F2000F7B50D46044600211646284681220EF06C
:108F3000E9FB23460822002128460BF087F894F924
:108F400001206378002AB8BF7F238DF807309EB9CF
:108F50000722082128460DF107030BF077F80F27A9
:108F6000002602349DF8073007EBC6019E4205D368
:108F70000731C80803B0F0BD0827F1E7A31908229C
:108F800028460BF063F80136ECE7000037B50446DD
:108F9000007F0D4610B1A38A072B15D800230822A5
:108FA00019460095204608350AF010FF01233022AB
:108FB0000821204600950AF009FF237FA08A2BB9DB
:108FC00006288CBF0020012003B030BD073818BF31
:108FD0000120F9E738B50C4600210546216003461B
:108FE000C4F80310204630220BF030F8204601224E
:108FF000302105F108030BF029F8072038BD0000E7
:109000002DE9F04390F81C8006460D4685B0B8F176
:10901000000F06D0838AE02B03D9012005B0BDE8FC
:10902000F08300230D221946304600950AF0CEFE4B
:109030000DF10F030093032200230D2130460AF0A7
:10904000C5FE9DF80F30042BE7D82B72013B032B94
:1090500003D8DFE803F025303B461024B8F1000FB9
:109060005FD105F19803214600930722434630461D
:109070000AF0ACFE073495F898305C2BCDD82F461B
:1090800095F898207B1B934252D3337F0734B08AE4
:10909000E408002B58D1844294BF00200120BDE792
:1090A00005F11003009340220123102130460AF0FD
:1090B0008DFE5024D2E705F11003009320220123F6
:1090C000102130460AF082FE3024C7E705F1100374
:1090D000009308220023102130460AF077FE18245E
:1090E000BCE705F11003009308220023102130464D
:1090F0000AF06CFE2B7C802B8FD8002705F111091C
:109100002B7CFC009F4204F11804A7D209EB070353
:10911000009308220023214630460AF057FE01370B
:10912000EEE7B38AC4EBC303DB0885F89830A2E707
:1091300007F19903214600930822002330460AF0E4
:1091400045FE083401379BE7201A18BF012065E768
:10915000F7B50C461546137809688DF806300322DA
:109160000DF1060306460AF071FF21680331216004
:109170002B78013B032B0CD8DFE803F0020D161F00
:1091800005F10803402230460AF060FF23684033AF
:10919000236003B0F0BD05F10803202230460AF039
:1091A00055FF23682033F3E705F108030822304612
:1091B0000AF04CFF23680833EAE72B7A0027802B5C
:1091C00028BF802308228DF8073030460DF10703B1
:1091D0000AF03CFF23680935083323609DF8073007
:1091E0009F42D6D2EB190822304621680AF02EFFA2
:1091F0002368013708332360F0E7000073B50C469D
:109200001546137809688DF8073002220DF107031F
:1092100006460AF01BFF2168023121602B78012BE2
:1092200003D0022B0BD002B070BD05F10803402221
:1092300030460AF00BFF236840332360F3E705F163
:109240000803202230460AF001FF23682033F4E7A8
:1092500073B50D46044600211646284640F27312A7
:109260000EF050FA05232246284601A90193FFF784
:109270006FFF019B2846053304F1900201A9019379
:10928000FFF766FF019B2846063304F5907201A99B
:109290000193FFF7B3FF019B2846063304F598724C
:1092A00001A90193FFF7AAFF94F840315C2B28BF76
:1092B0005C238DF803304EB90DF1030307222846D5
:1092C00001990AF0C3FE019B07330193002604F2C3
:1092D00041149DF8033001999E4203D30731C80819
:1092E00002B070BDA319082228460AF0AFFE019B08
:1092F000013608330193ECE700487047C07B010852
:109300000121884238BF08460CF0E0BEFFF7F8BFE5
:1093100008B10CF0DFBE7047FFF7FABF10B4026867
:1093200054681A46234610BC1847000000207047B6
:1093300001207047002070470020704700207047D0
:109340007047000000207047002070477047000001
:109350007047000037B50C4605468322011D01A861
:1093600000F05AF9611EC9B202299EBF002305EB25
:10937000C101C1E9073301A800F070F903B030BDA5
:109380002DE9F7431E461B8805465B07884620D417
:10939000011D422201A800F03FF92C4605F11809F1
:1093A0004C4513D0E3696BB12B6828465B6C98473A
:1093B0003388C1B24246276AE06943F00403B847E4
:1093C0000834EDE7236A002BEED1F9E701A800F09D
:1093D00045F9012003B0BDE8F08300007FB56D467C
:1093E000044685E80600011D712203A81E4600F010
:1093F00013F921460022C869D3B288B9086A78B93E
:1094000095E8030004EBC20201241C32013382E818
:109410000300337003A800F021F9204604B070BDAA
:109420000132032A01F10801E5D10024F2E700002E
:109430002DE9F04E04468AB00E465322011D01A8C4
:10944000BDF84890254600F0E7F8002704F1180A17
:1094500009F0040BAA4538D0EB690BB92B6A63B14C
:10946000BBF1000F0BD1236820465B6C98474B463D
:10947000C1B23246D5E9070CE0470835EAE7002FCC
:10948000FBD100220023CDE902233346ADF8107052
:1094900005AA06F1080C174618685968083303C76F
:1094A00063453A46F7D1186838609B88BB8006F060
:1094B00087F80423ADF810302368CDE902019B6CD6
:1094C000204602A998470127D7E701A800F0C6F86F
:1094D00001200AB0BDE8F08E30B503680968DD0FE1
:1094E000B5EBD17F23F0604421F060424FEAD170A8
:1094F0000BD0002BB8BFA40C0029B8BF920C94422B
:1095000002D034BF0120002030BD944205D1C1F308
:109510008070C3F380738342F6D194422CBF002045
:109520000120F1E7082817D90C280CD910280CD9EC
:1095300014280CD918280CD920280CD930288CBF15
:109540000F200E207047092070470A2070470B201B
:1095500070470C2070470D2070470000082817D96D
:1095600009280CD00A280CD00B280CD00C280CD0C1
:109570000D280CD00E2814BF4020302070470C203E
:109580007047102070471420704718207047202023
:1095900070470000436818478368184710B5024CAD
:1095A0008260C0E9004110BD587C0108007B00F0DA
:1095B00001007047704700008160828070470000A2
:1095C000826838B504465AB1037B13F0010507D110
:1095D00043F0010303739047237B65F30003237378
:1095E00038BD000010B50446034B1B68986A036839
:1095F0001B699847204610BD9C0D002010B50446FD
:10960000044B00211B68986A03681B699847204631
:1096100010BD00BF9C0D0020F8B50C4B01601E680A
:109620000446B06A174603681B6C9847054610B19C
:10963000F36AA3F84270206803689B6898471DB1DD
:109640000022F36AA3F842202046F8BD9C0D0020BA
:1096500010B50446FFF7E0FF204610BD10B50446E4
:1096600000680368DB689847204610BDC181B1FAE5
:1096700081F0400970470000C089704770470000C2
:1096800000207047704700007047000000207047BE
:1096900000207047704700004FF4B450704700003E
:1096A000002070470020704700207047002070475E
:1096B00000207047007B70477047000007B50368C3
:1096C0008DF807100122DB680DF10701984703B000
:1096D0005DF804FB08B5036801225B6A984700281F
:1096E000D4BF0020012008BD07B503680DF10701B4
:1096F000DB69984720B19DF8070003B05DF804FBD3
:109700004FF0FF30F9E7000070B5044608460D46FB
:10971000FDF728FE2368024629462046BDE8704032
:10972000DB68184705F04CBF10B4446824B90368DF
:1097300010BCD3F880301847002010BC70470000E0
:1097400082681AB90368D3F8903018470020704730
:1097500082681AB90368D3F894301847002070471C
:1097600030B4456825B90468E46FA44630BC60474E
:1097700030BC704700231A46FFF7F2BF10B484686C
:109780000CB19C4205D1036810BCD3F8843092B26E
:109790001847002010BC70470023FFF7EFBF000000
:1097A000481E01288CBF0020012070470020704710
:1097B00000207047002070477047000000230B70A6
:1097C000704700007047000070470000002070479D
:1097D000704700000020704700207047704700006D
:1097E0004368C26893423CBF8268D15443680133E6
:1097F0004360012070470000F8B505460C4600267E
:109800008F18BC4207D02B6828469B6814F8011BB0
:1098100098470644F5E73046F8BD00000020704741
:1098200000207047002070470020704738B590F83E
:109830009C3004468B420D460CD080F89C1005F0FD
:10984000BDFE2368C4F8A0005B682046984708B9AD
:1098500084F84D5038BD00007FB50D4614461946BA
:1098600000267AB1531E0B4A6846CDE90026089AB5
:10987000CDE9025300F062F80198844204D92E54D5
:1098800004B070BD1346EEE7002CF9D02C4404F868
:10989000016CF5E7687C010808B410B585B007AC29
:1098A00054F8043B00940394FFF7D6FF05B0BDE8DD
:1098B000104001B07047000007B503680DF10701C3
:1098C000DB69984720B19DF8070003B05DF804FB01
:1098D0004FF0FF30F9E70000F8B506460F46144692
:1098E0000025AC420AD0336830469B699847431C38
:1098F00001D12846F8BD78550135F2E72046F9E751
:109900000EB403B503AA52F8041B036801925B6806
:10991000984702B05DF804EB03B0704700F00EB852
:1099200070B5044608460D46FDF71CFD2368024647
:1099300029462046BDE87040DB6818472DE9F04F06
:109940000B468046144689B0197800294BD025294A
:1099500008D003F1010AD8F8003040469B689847C8
:109960005346F1E7597803F1020A2529F3D04FF065
:1099700000094D464E461F2E43D82B2936D01AD803
:10998000202935D0232939D0A1F13003DBB2092BAE
:1099900040D872064BBF09EB890905EB850503EB3F
:1099A000490903EB45054EBF09F0FF0905F0FF0526
:1099B00046F0200605E02D291DD03029E4D146F0DF
:1099C00001061AF8011B0029D5D126F006077029D7
:1099D000BFB200F0C28000F2B780582900F0C0800A
:1099E0006F2900F0C48009B0BDE8F08F46F0020690
:1099F00046F00406E5E746F00806E2E746F0100602
:109A0000DFE77F2EC0D9370612D56C2910D146F476
:109A10008076D6E72E2904D17306E4D446F04006BA
:109A2000CFE76C2902D146F08006CAE76829C8D082
:109A3000632930D0732949D064295DD126F090077D
:109A400016F4807FBFB202AE72D0E21D22F0070290
:109A50001446516854F8080B002904DA404261EBBF
:109A6000410147F080070A23324600F067F9861B60
:109A7000F6B27B0640F1848027F001034E459BB28D
:109A800080F09A8007F01402102A02D127F0110307
:109A90009BB2CB4676E0012754F8043B0DF1080B4E
:109AA0008DF80830300701D4BD421CD85F44BB4557
:109AB00000F0E780D8F8003040469B681BF8011B97
:109AC0009847002DF3D0013DEDB2F0E754F804BB08
:109AD00016F0400F14BF49464FF0FF3158460DF0C5
:109AE0007DFE0746DEE7D8F80030202140469B681F
:109AF000013D9847EDB2D7E769299FD075297FF4DA
:109B000064AF0A2326F01007BFB217F4807FDBB2E0
:109B100002AE2ED0073424F007043246F4E80201E6
:109B200000F00CF9861B27F08007F6B2BFB2A0E761
:109B300054F8040B0A2200283146BCBF404247F0CB
:109B4000800700F0ABF892E778297FF44CAFF90674
:109B500001D547F004071023D7E747F01007F6E7D1
:109B6000F20601D547F006074FF40473CDE708234A
:109B7000CBE71A46314654F8040B00F08FF8D1E7D2
:109B8000B3463B46D80623D508AA324412F8192C0E
:109B9000302A13D123F016039BB213F008022AD106
:109BA000DF0719D5AB454ED206EB0509A9EB0B092A
:109BB0005FFA89F9002523E0B346E3E75A0702D4A8
:109BC0000BF1010B01E00BF1020B5FFA8BFBE4E7F9
:109BD00013F0860FE1D0F3E7D8F80020AB45926888
:109BE000E8D20193202140460BF1010B90475FFA28
:109BF0008BFB019BF0E7AB45DCD2A5EB0B05EDB28F
:109C0000D8F80020D80692681FD50193302140462D
:109C10009047019B5A0709D513F0020F14BF582132
:109C20007821D8F80020926840469047D8F8003054
:109C30004E459B6816D23021404609F1FF399847BE
:109C40005FFA89F9F2E7B146B4E713F0860FEDD079
:109C500013F0020F14BF2B21202113F0800F18BF27
:109C60002D21E1E7771EFFB202AB1F44D8F8003088
:109C7000013EF6B240469B6817F801199847002E3E
:109C8000F4D1002D3FF46CAED8F8003020214046CE
:109C90009B68013D9847EDB2F3E70000082A0346B0
:109CA00030B5084606D11A46DB08FCD102F1300374
:109CB00003700DE0102A0CD103F00F0101F1300206
:109CC000392A88BF01F137021B0900F8012BF3D1B3
:109CD00030BD0022D9B223F00103023342F1000269
:109CE0005C0844EAC274E31842EB52021C0944EADD
:109CF0000274E41842EB1212230A43EA02631C19AD
:109D000042EB1222230C43EA02431B1942EB12429C
:109D1000D31842F100041B0943EA0473C3EB431553
:109D2000C3EB8505303101EB450100F8011B53EA17
:109D300014114FEA1412CDD1CAE70000082B30B538
:109D4000044610460AD12346E40844EA4174C9088F
:109D500054EA0102F7D13033037013E0102B12D113
:109D600004F00F0202F13003392B4FEA141488BFBC
:109D700002F1370344EA0174090900F8013B54EA8F
:109D80000103EDD130BDE2B224F00104023441F10F
:109D90000003610841EAC371091943EB53030C093D
:109DA00044EA0374611843EB13130C0A44EA036496
:109DB000611843EB13230C0C44EA0344641843EB8F
:109DC00013431C1943F10003240944EA0374C4EB50
:109DD0004415C4EB85053032190902EB450254EAFB
:109DE000131300F8012BCED1CCE7000008B5FCF727
:109DF00099FD4FF0505120F00040FDF73BF800383E
:109E000018BF012008BD0000F8B50D460146044604
:109E100016461F46FDF756F888B103F051F9BAB25D
:109E20004FF4806103F038F931462846FCF77CFD99
:109E30004FF07C51FCF780FE04462046F8BD2946D1
:109E40002046FDF717F838B931462046FDF730F8BF
:109E50000028F2D03446F0E72C46EEE703468B426A
:109E6000084603DB9342A8BF13461846704700001C
:109E700049F26900084A136899B21B0C00FB0133D0
:109E800044F250611360054B186882B2000C01FB6C
:109E90000200186080B27047080D0020040D0020F9
:109EA000F8B504460E46104609681546FCF744FE10
:109EB000716807462846FCF73FFE0346B16828460E
:109EC0001D46FCF739FE0346276020466560A36007
:109ED000F8BD00BF38B504460D4600680968FCF7B8
:109EE00023FD0346696860682360FCF71DFD034697
:109EF000A968A0686360FCF717FD03462046A360CD
:109F000038BD00BF38B5044600680D46FCF714FEA6
:109F10000346294660682360FCF70EFE0346294687
:109F2000A0686360FCF708FE03462046A36038BDC6
:109F300038B5044600680D46FCF7B2FE03462946D4
:109F400060682360FCF7ACFE03462946A0686360A6
:109F5000FCF7A6FE03462046A36038BD016810B595
:109F600004460846FCF7AEFF60B961680846FCF796
:109F7000A9FF38B9A1680846FCF7A4FF003818BF4C
:109F8000012010BD012010BD38B50468054624F03D
:109F9000004420461649FCF795FF30B92046144985
:109FA000FCF772FF08B9012038BD6C68104924F035
:109FB00000442046FCF786FF28B920460C49FCF7F0
:109FC00063FF0028EFD0AD68094925F00045284619
:109FD000FCF778FF4FF0010428B928460449FCF744
:109FE00053FF00B9044684F00100C0B238BD00BF81
:109FF000FFFF7F7F2DE9F04104462B2900F25E82AE
:10A00000DFE811F04300180212020102FC01EE0128
:10A010005701470140015C015300380182018A0168
:10A020004500D8000401EF00340121011A010A01A2
:10A030009B01DE01D801D30145005300C801C201D4
:10A04000BA01AF01A601CE00C500BD00B300A70054
:10A050005C0057002C0044023402200283684668EA
:10A06000056803F10043436029463046FCF75CFC79
:10A070009A49FCF761FD034631462846A360FCF788
:10A0800051FC9649FCF758FD2060BDE8F08102685C
:10A09000D0E9011302F1004201F1004103F1004354
:10A0A00021606260A360BDE8F08183680268416856
:10A0B000F4E78668056831462846D7E70568884989
:10A0C0002846FCF739FD6768804686493846FCF724
:10A0D00033FD01464046FCF727FCA66880468249CE
:10A0E0003046FCF729FD01464046FCF71DFC0346BF
:10A0F0007E4923602846FCF71FFD7D49804638468F
:10A10000FCF71AFD01464046FCF70EFC79498046F3
:10A110003046FCF711FD01464046FCF705FC0346BE
:10A12000754963602846FCF707FD744905463846C3
:10A13000FCF702FD01462846FCF7F6FB0546704990
:10A140003046FCF7F9FC01462846FCF7EDFBA06021
:10A150009BE782680368416802F1004203F1004313
:10A16000A16022606360BDE8F0818168D0E90032BF
:10A1700002F1004203F1004382600160F2E74368AC
:10A18000816802686160A2602360BDE8F081436875
:10A19000016803F10043826843608160226074E7D4
:10A1A00082684368016802F1004203F100434260A3
:10A1B0008160E9E74668056831462846FCF7B4FB4C
:10A1C0005049FCF7B9FC0346314628466360FCF76A
:10A1D000A9FB4249FCF7B0FCA36803F10043A3606C
:10A1E00052E7876843680668394683603046FCF763
:10A1F0009BFB394605463046FCF794FB3749FCF794
:10A200009BFC03463549284663603BE78368426808
:10A2100003F100438260A5E743688768066803F19D
:10A220000043394683603046FCF77CFB39460546DF
:10A230003046FCF779FBE1E74368826803F10043AD
:10A240008360626021E787684368066839468360F7
:10A250003046FCF767FB394605463046FCF764FBA1
:10A260001E49FCF769FC27490346CCE78268416830
:10A27000036875E70668456831462846FCF754FBD5
:10A2800016499EE7D0E9012302F1004203F10043A1
:10A2900007E70568466829463046FCF743FB0F4947
:10A2A000FCF74AFC0346314628466360FCF73CFB5A
:10A2B000E7E60368426803F1004352E74668056831
:10A2C00031462846FCF72EFB0449FCF735FC0346D3
:10A2D000314628466360FCF727FB7AE7F304353FF5
:10A2E000CF78123E46D0BC3E4D1F6BBF4F0DAABE6D
:10A2F000C9355BBFF184CABEC6AC6EBFDB26B93EB2
:10A30000F63BCC23F30435BF0268836802F10042B8
:10A3100003F100432260C5E60568466829463046D9
:10A32000FCF700FB6A49FCF707FC03463146284668
:10A330006360FCF7F9FA67494CE783684268016893
:10A3400002F1004203F100438260036041609CE639
:10A3500003684268816803F10043416003608260E2
:10A3600093E681684368026801F1004102F100420E
:10A3700003F100434160CDE78168D0E9002303F198
:10A38000004302F10042FDE6D0E90113026801F149
:10A390000041F4E782680368416802F1004203F17A
:10A3A00000434260836001606FE68368026803F1E6
:10A3B0000043E8E60368826803F100438360EDE64A
:10A3C00043688768066803F1004339468360304676
:10A3D000FCF7AAFA394605463046FCF7A3FA3FE7F0
:10A3E0000668456831462846FCF79EFA3949FCF76D
:10A3F000A3FB034631462846636040E6D0E90023CC
:10A4000002F1004257E74668056831462846FCF7E6
:10A4100089FA2F49FCF790FB0346314628466360D2
:10A42000FCF782FA2B492DE64368026803F10043EA
:10A43000036006E74668056831462846FCF774FA6B
:10A440002349D4E74568866829463046FCF76AFA0E
:10A450001F49FCF771FB034631462846A360FCF711
:10A4600063FA1B49FCF768FB60600EE68668456886
:10A4700031462846FCF758FA1549FCF75DFB0346C0
:10A4800031462846A360FCF74DFAEAE7076812490F
:10A490003846FCF751FBA668054610493046FCF7E4
:10A4A0004BFB01462846FCF73FFA03460C49384669
:10A4B0002360FCF741FB0849054641E602F000FE37
:10A4C000BDE8F04140F211124FF4800102F0E4BD0A
:10A4D000F304353FF30435BF81177E3FA296F93D63
:10A4E000A296F9BD0346416870B5056808469E68A6
:10A4F000FCF722FB314604463046FCF71DFB0146C3
:10A500002046FCF711FA294604462846FCF714FBBE
:10A5100001462046FCF708FABDE870400CF0E8BBA5
:10A520007047000038B5056804462DB1284605F08F
:10A53000E5F92846FEF7ECFE204638BD13460246F4
:10A54000014801F069BD00BFFC190020042213B5C9
:10A55000054B044601460DEB02000193FFF7EEFFA9
:10A56000024B1C8002B010BDFFFF3F00F01900201D
:10A57000502307B58DF804304123042200218DF8C3
:10A58000053006230DEB02008DF806308DF807101C
:10A59000FFF7D4FF0420FFF7D9FF03B05DF804FBF9
:10A5A00000EB0212907B20B91BB19289120758BFB1
:10A5B0003F20984008447047430608D4000A08D05A
:10A5C000054B1B88184214BF012000207047002053
:10A5D00070470120704700BFF419002010B5142403
:10A5E0000A4B01301A880A4B80B21B6804FB003307
:10A5F000824206D9DC8914338C4204D0013080B207
:10A60000F6E7002010BD0120FCE700BF001A002083
:10A61000041A002003469B898068DB0648BF006857
:10A620007047000003469B898068DB0648BF0068CE
:10A6300070470000042307B500220DEB03010B480F
:10A64000019201F0C9FC9DF80430502B07D19DF810
:10A650000530412B03D19DF80630062B01D0FFF7C2
:10A6600087FF012003B05DF804FB00BFFC19002048
:10A6700082894368920705D51B68181E18BF012000
:10A680000B6070470120FBE737B58B891446DA076A
:10A690000D4605D523684A6813442360012012E063
:10A6A0009B07FBD514220A4B01A91B6802FB003053
:10A6B000FFF7DEFF48B1019922686B680A44D3585E
:10A6C0001BB15B1A236003B030BD0020FBE700BF65
:10A6D000041A00202DE9F04F1F46142305461646A4
:10A6E0004FF0000B53438BB09DF85480059308F155
:10A6F0000603DBB2069107935FFA8BFA07EB0A19A0
:10A7000099F80F40002C4CD0062C28D1B8F10B0F33
:10A7100021D84846FFF77EFF0446C8B1169B49463C
:10A72000304609AA0993FFF7AFFF88B14346524666
:10A7300014993846FFF734FF099B32460293079B72
:10A740000699CDE9000323462846FFF7C3FF18B951
:10A750000BF1010BD0E700200BB0BDE8F08F4346B2
:10A76000524638461499FFF71BFFB0EB953FEFD1E7
:10A77000C5F30423A342EBD10B4C059B206809A928
:10A780001844FFF775FF0028E2D0D9F80430099A81
:10A790001344169A1344069A13602068059B1844C4
:10A7A000DAE72046D8E700BF041A00202DE9F04779
:10A7B0000F46054600211D4B5FFA80F8B3F8009064
:10A7C000C0F3403348EA0328194B86B01E68C0F333
:10A7D000042A8AB2914526D9F389344643451FD1CC
:10A7E000337C062B0ED13046FFF71CFF0346B8B171
:10A7F00000212846CDE9011100913946FFF76AFF93
:10A80000044609E09A450BD1304605A9FFF730FF11
:10A810000028F5D0059B3B60204606B0BDE8F087D8
:10A8200001311436D5E70024F6E700BF001A0020F6
:10A83000041A00202DE9F04F9846142353438DB09D
:10A840000693484B04461868069B0E4618440AA90E
:10A8500017469DF85890DDF868B0FFF709FF00280B
:10A860007DD00023079309F10603DBB209939DF81D
:10A870001CA006EB0A15EB7B002B70D0062B3BD1FE
:10A880002846FFF7C7FE0890002831D0B9F10B0F1A
:10A8900065D8179B294638460BAA0B93FFF7F4FEA1
:10A8A00030B39BF80030012B59D85A1C0BEB8303B3
:10A8B0008BF80020414652465D6030464B46FFF71C
:10A8C0006FFE1B9A0346CDE904B2199A2046039203
:10A8D000189A089902920B9A0192099A00923A46A4
:10A8E000FFF7A8FF00BB9BF80030013B8BF800305E
:10A8F000079B01330793BAE7179A686810440A9ACE
:10A900001044A04213D14B46524641463046FFF711
:10A9100047FE189B1B9A1860199B1D60002313703B
:10A92000104B1868069B18440DB0BDE8F08F052B3E
:10A93000DED1031D9C4203D000F108039C42D7D115
:10A940001B9B201A8008187052464B4641463046E1
:10A95000FFF726FE189B1860199B1D60E0E700209A
:10A96000E2E700BF041A00202DE9F04F002506465B
:10A970000F4690468BB0DFF89CA007931560264BDE
:10A980001FFA85FB1B885B4541D91423DAF80000C8
:10A9900009A903FB0B04204694F81090FFF768FE0A
:10A9A00098B3B9F1060F17D12046FFF73BFE0146D9
:10A9B00058B3149B5A460593079B3046CDE9038351
:10A9C00000230297CDE90033FFF734FF0446E0B1DE
:10A9D00020460BB0BDE8F08F0998B04204D10023A7
:10A9E000149A3B601370F3E7B9F1050F0DD1031D05
:10A9F0009E4203D000F108039E4206D1149B301AF8
:10AA00008008187000233B60E2E70135B7E70024B7
:10AA1000DEE700BF041A0020001A00202DE9F04FE5
:10AA2000044614209946254BB1F800A01D68CAF3CE
:10AA3000080A00FB0A5589B0284607A91746DDF821
:10AA40004C8095F810B0FFF713FE20B9002528467A
:10AA500009B0BDE8F08F0026BBF1060FC9F8006011
:10AA600014D12846FFF7DEFD01460028EED0129BE8
:10AA70005246CDE9039320463346CDE90167CDF830
:10AA800014800096FFF7D6FE0546E0E70798A0423F
:10AA900003D13E6088F80060D9E7BBF1050FD5D13E
:10AAA000031D9C4203D000F108039C42CED1002339
:10AAB000241AA40888F800403B60C8E7041A002064
:10AAC0000138C0B204289ABF014B185C00207047BF
:10AAD000EC7C01082DE9F04F002405460E46174690
:10AAE000A146A0464FF0010A85B00193931DDBB249
:10AAF0000293E0B2020105EB001090F80FB0BBF139
:10AB0000000F59D0837B3F2B02D92D4804F02EFD36
:10AB100017B1002B08BF3F23C3F1200EA3F1200C77
:10AB200029FA03F108FA0EFE28FA0CFC41EA0E019C
:10AB300041EA0C0111F0010FC3F1200CA3F1200137
:10AB4000E3D10AFA01F12AFA0CFC41EA0C010AFAF3
:10AB500003F3BBF1060F43EA090941EA080812D1E1
:10AB60000B2FD2D8FFF756FD834650B1A858FCF7FB
:10AB7000F9FB019B31460344029A5846DBB2FFF7CA
:10AB8000A9FF0134B5E75846FFF79AFF0390002864
:10AB9000BBD0A858FCF7E6FB019BBBF1050F18449E
:10ABA000C0B204BF0230C0B21028039BADD83088B9
:10ABB000043003443380E4E705B0BDE8F08F00BF04
:10ABC000947C010804232DE9F74F00244FF0140A68
:10ABD000DFF88890ADF80630214B1FFA84F81B8807
:10ABE000434537D90AFB08F2D9F800108D182F7C9D
:10ABF000B5F80EB0062F21D1B8F1000F02D11948D7
:10AC000004F0B4FC2846FFF70DFD0646A0B18858B5
:10AC1000FCF7A8FB0022C3B20DF106013046FFF796
:10AC200059FF59464046FFF7D9FC0028E7D1062FC7
:10AC300002D0AB899B07E2D40134CDE73846FFF759
:10AC40003FFF0028DBD0BDF8063004331844ADF8D0
:10AC50000600E6E703B0BDE8F08F00BF041A00204D
:10AC6000001A0020947C0108437803F01F021F2A79
:10AC70000FD00278C3F3401342EA032340F2FF12DD
:10AC8000934206D000680138C31C94BF0020012005
:10AC900070470120704700002DE9F34106460D463C
:10ACA0000424214FDFF884807B88A34237D9042312
:10ACB00022460DEB0301384601F08EF99DF8051090
:10ACC000737881EA0302D20618D196F800C09DF885
:10ACD0000400C3F34013C1F340124CEA032340EADB
:10ACE000022293420AD13268019B534013EA080FB3
:10ACF00004D101202C8002B0BDE8F08101A8FFF74B
:10AD0000B3FF20B10A4B2C801C800020F3E701F038
:10AD10001F00FFF7D5FE031D1C44A4B2C4E74FF685
:10AD2000FF732B80F1E700BFFC19002000C0FFFF7C
:10AD3000F019002070B50C461146204615461E46F7
:10AD40000CF04CFD831CAB420AD85F22225422181F
:10AD50000330A84206F1580656709CBF0022E25408
:10AD600070BD00002DE9F74F9B46DDE90D549DF8BD
:10AD70003C3007468A4616462846224609689DF812
:10AD8000308000934FF000090CF014FD9BF8001088
:10AD90005FFA89F29142019212D9214628460CF0BD
:10ADA0001DFDC0B28442019A07D90BEB82025168A3
:10ADB000221A096828440CF0FDFC09F10109E5E7B5
:10ADC000E6B1214628460CF009FDC0B2844204D900
:10ADD000221A316828440CF0EDFC009B13B9B8F13D
:10ADE000000F13D0F37B052B10D143462246294692
:10ADF000384603B0BDE8F04FFFF79CBF009B13B986
:10AE0000B8F1000F02D09AF81030ECE703B0BDE8BB
:10AE1000F08F0000F0B51F4600238BB007ACC4E9EB
:10AE2000013307930DF11303CDE90043154606AB3B
:10AE300005AA0646FFF7F2FD014610B928700BB0CF
:10AE4000F0BD9DF840303046CDE902739DF81330D7
:10AE5000069A009301952346FFF784FFEFE7000071
:10AE60002DE9F04F9846142304460E464FF0000992
:10AE70004B4389B0DFF820A1039204935FFA89F570
:10AE80002B0108EB051595F80FB00593BBF1000FEA
:10AE90007FD0BBF1060F58F803702AD13846FCF773
:10AEA00061FA3946024620460CF04EFC002869D172
:10AEB0002846FFF7AFFB0746002863D0039B2946CF
:10AEC000304607AA0793FFF7DFFB00285AD0059BFF
:10AED00058F80300FCF746FA129B31460093079A94
:10AEE0003B462044FFF7BCFF00284BD009B0BDE82B
:10AEF000F08F394620460CF00DFC88B9DAF80000D6
:10AF0000049B07A91844FFF7B3FB00283AD0129B13
:10AF100083F800B06868079B1844039B1844E5E772
:10AF2000BBF1050F2ED1102138460CF057FC5FFA0B
:10AF300080FB5A46394620460CF028FC10BB14F919
:10AF40000B305F2B1ED10BF1010B14F80B30583B6B
:10AF5000022B17D8DAF80000049B07A91844FFF762
:10AF600087FB78B16868079B129A1844039B1844C2
:10AF70000423137014F90B30592B06D05A2B06D02A
:10AF8000582BB3D009F1010978E70430AEE7083057
:10AF9000ACE75846AAE700BF041A00202DE9F04F9D
:10AFA0000446174600258BB0DFF8BCB002912F4B4A
:10AFB0001FFA85FA1B88534552D91422534653432E
:10AFC000DBF8002002EB030999F81080D358B8F1A0
:10AFD000060F33D11021184603930CF0FFFB039B9F
:10AFE0005FFA80F84246194620460CF0CFFB064631
:10AFF000002833D14846FFF715FB034670B3029A89
:10B0000004EB0800009251463246FFF729FF8046C4
:10B0100020B37FB10DF11303009306AA07AB05A976
:10B02000CDE9076605960996FFF79EFC069B0BB1D6
:10B030009B893B8040460BB0BDE8F08F1946204607
:10B040000CF068FB50B9029B484683F8008007A9C2
:10B05000FFF70EFB20B1DDF81C80EBE70135A6E71A
:10B060004FF00008E6E700BF041A0020001A002095
:10B07000002230B50A4B1C880A4B1B6895B2AC42C3
:10B080000CD91D7C062D06D15D68854203D10120B7
:10B09000DB890B8030BD01321433EFE70020F9E784
:10B0A000001A0020041A0020002310B590B0CDE94A
:10B0B000083306930A930DF11703009306A908AB12
:10B0C00007AA0446FFF750FC014668B1112301228C
:10B0D000CDE902320BAB01939DF817302046009367
:10B0E000079A08ABFFF73EFE10B010BDF0B5304D2B
:10B0F00087B040F2A51202908DF80C1006460C465F
:10B1000001A8291DFEF788FA052204A9286804F081
:10B1100037FD074601A8FEF7A1FA052F06D1049BCB
:10B12000B34203D19DF81430A3423ED0214E224FAA
:10B130004FF4B072314601A8FEF76EFA286804F0A9
:10B1400045FC042821D90522286802A904F0B4FC92
:10B15000431F5C425C4101A8FEF780FA2CBB3C68AF
:10B16000E36A93F89C3093B9A06A012103681B69D4
:10B170009847A06A4FF4FA7103689B689847A06AE1
:10B18000002103681B699847D2E70024E3E7A06A1F
:10B1900003681B6C98470028E6D001F091FF40F24D
:10B1A000FA424FF4801101F077FF07B0F0BD00BF05
:10B1B000CC190020D01900209C0D00202DE9F3416E
:10B1C000C924154E154F06F10408013CA4B2FCB188
:10B1D00040F24B12414601A8FEF71EFA306804F017
:10B1E000DDFB054601A8FEF739FA042D10D93D68AC
:10B1F0000A21A86A03681B699847A86A0A2103689C
:10B200005B689847A86A002103681B699847DCE7D8
:10B2100002B0BDE8F08100BFCC1900209C0D0020D9
:10B22000002300B58BB0CDE90733049309930DF1EA
:10B230000D03009305AA07AB04A9FFF795FB10B314
:10B24000059B23B3DB7BC28903F01F038DF8182015
:10B250001B02C2F3002243EA4233049A0DF10E01AD
:10B2600043EA82339DF8182006A813430693FFF79C
:10B2700013FD40B19DF8193003F01F03052B03D0D7
:10B280009DF80D3003B100200BB05DF804FB037C8A
:10B29000D9E70000F0B5144F06463B880D4689B04B
:10B2A000FBB100240DF10B03009304AA05AB03A925
:10B2B000CDE9054403940794FFF756FB88B10B4B87
:10B2C00038881B68A2B290420BD91A461168013423
:10B2D0008E4203F10C03F5D10120137A2B7009B0D3
:10B2E000F0BD0020FBE700BFF8190020EC1900209A
:10B2F00013B50DF107010446FFF7CCFF10B9204646
:10B30000FFF78EFF02B010BD0346013B10B510469B
:10B310000C46032B06D8DFE803F002060A0EFBF703
:10B32000E7FD207010BDFBF7E3FD2080FAE7FBF797
:10B33000DFFD2060F6E70860F4E7000030B5224B3F
:10B3400085B01A7872B901221A70204B204A1B6806
:10B350000292986A1F4A0368039204AA9B6A12E940
:10B360000600984704241C4D6B88A34229D9042366
:10B3700022466946284600F02FFE6846FFF774FC17
:10B3800018B1164B1C8005B030BD009801A9FFF71D
:10B390000DFA60B19DF80100221D00F01F00FFF7BB
:10B3A0008FFB92B203460199284600F015FE9DF8E6
:10B3B000010000F01F00FFF783FB04300444A4B237
:10B3C000D2E70020DFE700BFFA1900209C0D002023
:10B3D000AD190020B5BD0008FC190020F0190020AF
:10B3E00037B503680C4603F000430360094B1B8824
:10B3F00013B9002003B030BD074D01A92868FFF73D
:10B4000037F90028F5D014B12B681B7C2370019804
:10B41000F0E700BF001A0020041A00202DE9F04FC9
:10B420008FB09B469DF8703007460B93142343431F
:10B4300088460A9300239DF860901A9D089207930E
:10B440009DF81CA008EB0A16F47B002C00F0BC80D1
:10B45000B089FFF7B1F8002800F0B380062C2FD197
:10B460003046FFF7D7F80446002800F0AA80199B61
:10B47000314638460DAA0D93FFF706F9002800F073
:10B48000A0804B46524659464046FFF789F81D9A20
:10B49000034605920B9A214604921B9A3846CDE941
:10B4A00002520D9A019209F10602D2B20092089A54
:10B4B000FFF7B4FF002800F084800FB0BDE8F08FE4
:10B4C000089B1B780993002B3CD02B88524667F3CE
:10B4D00008032B8059464B464046FFF761F83B4B2B
:10B4E00003EA40302B6823F0FF4323F4FF0323F4E7
:10B4F000FC4318431B9B286003B11C70344B0DA9FF
:10B5000018680A9B1844FFF7B3F8002859D00D9A21
:10B5100073681344199A98180B9A002ACDD02D4AB3
:10B520001278002AC9D0F27B012AC6D1B28952070B
:10B53000C3D5199A9B56002BBFD1EB7843F08003FB
:10B54000EB70BAE74B46524659464046FFF728F89B
:10B550002B68C3F35133984233D10123089A1370F7
:10B5600095F90330002B06DAEB78099A62F3C713DA
:10B570001046EB70A1E7052C23D16B78C3F343028F
:10B58000022A1ED8013262F344036B701B9B13B175
:10B5900004231B9A13700E4B0DA918680A9B1844BC
:10B5A000FFF766F868B170680D9C95F801B0199BBB
:10B5B0002044CBF3430B18440BF1FF3B00EB8B0013
:10B5C0007BE7079B01333AE7204676E700E0FF7F01
:10B5D000041A00200C0D00202DE9F04F1F46002317
:10B5E000DFF8E0908BB004888DF82730B9F8003090
:10B5F000C4F30804A34205460E4607925FD91422FD
:10B60000DFF8C4806243D8F8003013441B7C052B5C
:10B6100018D14378C3F34301022915D8013161F3EE
:10B62000440343700EB1042333706878D8F80010D7
:10B63000C0F343000A44431E506800EB83000BB084
:10B64000BDE8F08F062B04D001230134A4B28DF89D
:10B6500027304FF0140B4FF0000AB9F80030A34226
:10B660002DD9D8F800200BFB04229089FEF7A4FF07
:10B67000B8B1117C062917D11046FEF7D3FF014659
:10B6800078B1079B2046CDE90363CDE901A50023EE
:10B690000597CDF800A00DF12702FFF7BFFE0028A7
:10B6A000CDD10134A4B2D8E72B68C4F3080403F069
:10B6B000004323432B6006B131705068BFE7002080
:10B6C000BDE700BF001A0020041A002073B505462C
:10B6D0000C4616463346012228460DF10701FFF7B6
:10B6E0007BFF28B19DF80730042BF3D804B12370F9
:10B6F00002B070BDF8B514460746002220460E463B
:10B700000025FFF76DFE40B1BD4206D00022314654
:10B710002046FFF7DBFF0135F5E7F8BD01390329C6
:10B720000BD8DFE801F00204060800F0C5BB00F00A
:10B73000F7BB00F031BC00F085BB0148704700BF8B
:10B740000000C07F37B5037A028803F01F038DF82D
:10B7500004201B02C2F3002243EA423342680C4633
:10B7600043EA82339DF804200DF10201134301A83E
:10B770000193FFF791FA054670B19DF80500214647
:10B7800000F01F00FFF79CF9BDF8022003460432C9
:10B79000034892B200F020FC284603B030BD00BF41
:10B7A000FC1900202DE9F04F83B0044600AF007A69
:10B7B000FFF786F9C31D23F00703E946ADEB030D40
:10B7C00088468246694620461646EB46FFF7BAFF92
:10B7D00080B30022E068F91DFFF7E0FB054640B9A1
:10B7E0002F4BE2681B682F49986903681B689847CC
:10B7F00020E0B2071AD5227AFB799A421FD14FF086
:10B800007E514046FEF7F2FAC8B1C6B952465946D3
:10B8100028460BF059FF68B15246594628460BF0AE
:10B8200063FF31462846FFF761FC03E0FFF7F8FCB1
:10B830000028E0D0CD460C37BD46BDE8F08FFB793F
:10B84000042B07D9164BE2681B68174998690368EF
:10B850001B68CCE7217A0429F4D85846FFF75EFF2D
:10B86000F307044604D51149FEF7C0FAA8B900242D
:10B87000F9792846FFF752FF01462046FEF7B6FA4F
:10B8800006460028D6D141462046FBF755F9294601
:10B890000246F879FFF738FDC3E74FF07E54E7E73B
:10B8A0009C0D0020A87C0108C17C0108000080BF1D
:10B8B000002270B50B4B1E880B4B1B6894B2A6423E
:10B8C00008D91C4625680132854203F10C03F5D1E5
:10B8D000606870BD8B891B0649BF8B688868C01A79
:10B8E0000068F6E7F8190020EC1900202DE9F04176
:10B8F00004460F464FF000085FFA88F307EB031188
:10B90000CD7BCDB1042D0CD84E6826443046FFF7D0
:10B91000CFFF314602462846FFF7F6FC08F1010842
:10B92000EAE7052DFAD14E68A5192846FFF7C0FFB2
:10B93000A0516860A860F1E7BDE8F081002270B511
:10B940000B4B1E880B4B1B6894B2A64208D91C46B1
:10B9500025680132854203F10C03F5D1606870BDA2
:10B960008B891B0649BF8B688868C01A0068F6E798
:10B97000F8190020EC19002000232DE9F0418AB0CD
:10B98000CDE90733039309930DF10903009304AA4A
:10B9900007AB03A90446FEF7E7FF054620B90026DA
:10B9A00030460AB0BDE8F081049B002B3BD0DB7B26
:10B9B000EA8903F01F038DF814201B02C2F3002252
:10B9C00043EA4233039A0DF10A0143EA82339DF8B8
:10B9D000142005A813430593FFF75EF9064668BBDC
:10B9E000284606A9FEF744FE0028D9D09DF8157018
:10B9F0000499DDF8188007F01F07C1B19DF81C30CD
:10BA00009BB1089A012B556802D0099B5B681D44C5
:10BA10002046FFF74DFF0246496841442944384615
:10BA2000FFF772FCBCE7037CC2E73546F0E7294626
:10BA30002046FFF783FF41460246F0E79DF81500D8
:10BA40009DF8093000F01F02052A0FD0002BA6D167
:10BA500000F01F00FFF734F8BDF80A200346043257
:10BA6000214692B2044800F0B7FA99E7002BEFD0D4
:10BA7000A4EB8304ECE700BFFC1900202DE9F34799
:10BA8000FEF7D8FD00254FF01408124E124F3288F1
:10BA9000ABB29A421AD91C463B6808FB043494F8AE
:10BAA0001090B9F1040F0FD8204601A9FEF7E0FD70
:10BAB00050B1DDF804A021465046FFF73FFF514644
:10BAC00002464846FFF720FC0135E0E702B0BDE83A
:10BAD000F08700BF001A0020041A00202DE9F34768
:10BAE000DFF8809040F6782268461F49FDF794FD04
:10BAF000B9F800702FB11D4B1A881D4B1B889A4254
:10BB000028D005244FF00008184E194DB9F80070E0
:10BB10001FB132882B889A421CD0013C14F0FF04DC
:10BB200018D0002201A811463788CDF804804FF0C4
:10BB3000000AFFF755FC1FFA8AF30AF1010A28B13F
:10BB4000002201A81146FFF7C1FDF4E7A9F8003073
:10BB50002F80DBE76846FDF781FD384602B0BDE87F
:10BB6000F08700BFF2190020B0190020EA19002068
:10BB7000F6190020024A138801331380704700BF72
:10BB8000EA19002000232DE9F04190B0CDE90833F7
:10BB900005930A930DF1110300930E4608AB06AA14
:10BBA00005A90446FEF7E0FE0546D8B10699E1B1C5
:10BBB000CA7BEB8902F01F028DF81C30C3F3002012
:10BBC0001302059A43EA403343EA82339DF81C206E
:10BBD0009DF811701A43C3F30423052B079200F05C
:10BBE000828027B110B0BDE8F081027CE1E7012B33
:10BBF00005D121B18B895B0701D5FFF7BBFF274634
:10BC000075E04FF6FF73BDF812209A420AD14B4BF4
:10BC100083F800804A4B4B491B68986903681B688E
:10BC20009847DFE79DF81D1001F01F01042925D971
:10BC30009DF81D00BDF8122000F01F00FEF740FF28
:10BC400041491318498808338B4248D204321044C2
:10BC500080B2FEF77BFC9DF81D0000F01F00FEF790
:10BC60002FFFBDF8121002460431384689B2FEF7A4
:10BC700065FC0422BDF8121007A85CE02046FFF71F
:10BC80004DFD0699804659B12046FFF711FE044646
:10BC900001464046FEF7AAF838B1002EC8D1A1E708
:10BCA00029462046FFF74AFEF1E7002EC0D19DF855
:10BCB0001D3003F01F03032BBAD021464046FAF78C
:10BCC00031FE224920F0004428F00040FAF734FF0A
:10BCD00001462046FBF7CEF80028A9D082E70122D2
:10BCE000164B1A7096E7002F89D0A4EB8707112313
:10BCF0004FF00108CDE902380BAB01939DF81130EC
:10BD0000294620460093069A08ABFFF72BF80DF161
:10BD1000120107A8FEF7C0FF00283FF472AF9DF89C
:10BD20001D0000F01F00FEF7CBFE02463846BDF8AE
:10BD30001210043189B2FEF701FC53E7E819002024
:10BD40009C0D0020DC7C0108FC19002017B7D138BD
:10BD50007FB5164D2E1D40F27F12314601A8FDF72A
:10BD60005BFC286803F01AFE042812D90522286813
:10BD700002A903F01FFF431F5C425C4101A8FDF7CD
:10BD80006DFC44B101229DF80C100298FFF7FAFEF9
:10BD9000E1E70024F2E7064B1B68986A03685B6BD7
:10BDA000984708B1FFF79AFE04B070BDCC19002087
:10BDB0009C0D0020FFF7CCBF10B50446FDF7A8FA94
:10BDC000204610BD38B51148114D02F06BFC114AE8
:10BDD00011490E480AF0FAFE0023284640F8043BB9
:10BDE00002F060FC1420FDF78BFA044610B19B2191
:10BDF00003F072FD0949074A05482C600AF0E6FE87
:10BE0000BDE838400021064800F0DEB8B019002037
:10BE1000CC190020C824002021A5000825A5000871
:10BE2000FC19002038B50D68044601682846FBF768
:10BE300017F830B9204625600121BDE83840FFF7EA
:10BE400055B938BD0068704738B504460D46FFF750
:10BE50004FFA10B995F90030237038BD91F90020E0
:10BE600090F90010914202D00270FFF71DB970479F
:10BE700038B5044691F9005090F90000401BFAF7DC
:10BE800007FE4FF0505120F00040FAF7F3FF011E7B
:10BE900025702046BDE8384018BF0121FFF726B9BC
:10BEA00091F9002090F90010914203D00121027015
:10BEB000FFF71CB97047000008B590F90000FAF7C9
:10BEC000E7FD08BD38B504460D46FFF711FA10B975
:10BED000B5F90030238038BD38B50446B1F90050BB
:10BEE000B0F90000401BFAF7D3FD4FF0505120F09D
:10BEF0000040FAF7BFFF011E25802046BDE838400C
:10BF000018BF0121FFF7F2B8B1F90020B0F9001015
:10BF1000914203D001210280FFF7E8B8704700008A
:10BF200008B5B0F90000FAF7B3FD08BD38B504460E
:10BF30000D46FFF7DDF908B92B68236038BD000016
:10BF40000B680360704700000A6801688A4202D0EB
:10BF50000260FFF7A9B8704738B504460D6800685D
:10BF6000401BFAF795FD4FF0505120F00040FAF7D2
:10BF700081FF011E25602046BDE8384018BF012121
:10BF8000FFF7B4B80A6801688A4203D00121026051
:10BF9000FFF7ACB87047000008B50068FAF778FD05
:10BFA00008BD000008B5064B1B68586903685B684C
:10BFB000984720B9BDE80840024802F063BD08BDBB
:10BFC0009C0D0020F47C0108017011B10023438016
:10BFD00070474FF44873FAE770B51C460378ABB965
:10BFE000B2F5487F12D2A3B21344B3F5487F094B90
:10BFF000C8BFC2F548751B68D8BFA5B25869C8BF8D
:10C00000ADB20368641B9E682B46B047B4FA84F057
:10C01000400970BD9C0D002070B51C460378ABB97B
:10C02000B1F5487F12D2A3B20B44B3F5487F094B58
:10C03000C8BFC1F548751B68D8BFA5B25869C8BF4D
:10C04000ADB20368641BDE682B46B047B4FA84F0D7
:10C05000400970BD9C0D002010B50446034B0449F7
:10C060001860FFF743FC204610BD00BF081A0020EF
:10C07000707D010890F8233063B9012380F82330E4
:10C0800005484FF40073006880224FF4E131006CE2
:10C09000FDF766BB704700BF9C0D0020002850DDF7
:10C0A0006F2846D01BDC132845D00EDC431E082B1E
:10C0B00011D8082B33D8DFE803F04105323632328D
:10C0C000323239004FF416607047392839D064286D
:10C0D0003AD026283AD04FF47A7358437047B0F5D7
:10C0E000FA7F36D010DCB0F5807F34D006DC7328C0
:10C0F00034D0E628EFD14FF461307047B0F5E67FD9
:10C10000E9D14FF4E120704740F2DC53984228D047
:10C11000B0F5FA6F27D040F29933984225D0B0F5A8
:10C12000FA6FD8DD70474FF4965070474FF41650B1
:10C1300070470F4870474FF4964070474FF4966031
:10C1400070474FF4614070470A4870474FF41640FB
:10C150007047094870474FF47A3070474FF4E13028
:10C16000704706487047064870474FF46120D9E78A
:10C17000FCB10100A086010020A1070060E31600C9
:10C1800080841E000068FFF789BF00000E4A70B56A
:10C190001568CAB2092A03460C4611D8103255F860
:10C1A000220003EBC10302689988526B904750B993
:10C1B000A8692246BDE87040036804491B68184717
:10C1C00000231B68FFDE70BD9C0D0020147D01085C
:10C1D0002DE9FF41FF2380460126732703A9213063
:10C1E0008DF80C30FFF75CFE4046FFF743FF554BE0
:10C1F00008F108041B680193019A06F1100352F834
:10C200002350E6717DB34046B1B2FFF7BFFF94F90A
:10C2100006300133332B00F28C80DFE803F0241A60
:10C220001A1A2C3335353D478A338A528A8A245A62
:10C230008A8A698A8A4C8A7D8A8A8A8A8A248A8A30
:10C240008A8A8A8A8A8A8A8A8A8A1A8A8A8A8A8ABE
:10C250008A242046FFF796FF4FF480730146802220
:10C260002846FDF77DFA0136042E04F10804C3D1F7
:10C2700004B0BDE8F0810923204603A90393FFF72A
:10C280005FFEF0E73923F7E72046FFF77BFF102337
:10C2900001464FF48072E3E703A920460397FFF7B6
:10C2A0004FFE80234FF4E1311A46D9E7204603A917
:10C2B0000397FFF745FE2046FFF764FF8023014602
:10C2C000CDE7092303A9A01D8DF80C30FFF7D0FDA1
:10C2D000C9E703A920460397FFF732FE2046FFF780
:10C2E00051FF1E2301461A462846FDF739FA0DE094
:10C2F0002046FFF747FF802301461A462846FDF7F0
:10C300002FFA2B6801212846DB6C98472B68002107
:10C310002846DB6B9847A6E703A920460397FFF75B
:10C3200005FE2046FFF72EFF102301464FF4007252
:10C33000DAE72046FFF726FF01462846FDF71AFAFE
:10C3400091E700BF9C0D002037B504460846089DC4
:10C3500011461A46036801959DF81C5000951D680A
:10C36000069BA8472060204603B030BD4FF0FF3346
:10C370000021002210B543610446417200F1200300
:10C38000E830D9709A60DA601A615A629A62DA62A9
:10C390001A635A639A63DA631A645A645A659A652F
:10C3A000DA6564338342ECD1044B1A6822B9204623
:10C3B00003491C60FFF79AFA204610BD0C1A0020B2
:10C3C000207E010890F82210034621B901205884EC
:10C3D0001170987170470020704700004FF0000006
:10C3E000704700000346084649B11A79012A05D072
:10C3F000511C197143F8220001207047002070473A
:10C4000038B5054690F8220058B10023012003F00A
:10C410004BFA00210446A86B03F056FA231A58423F
:10C42000584138BD11B990F821007047002070477D
:10C4300038B590F90530044633B390F803311BB397
:10C4400000252279EBB29A4206D954F8230001352F
:10C4500003689B689847F4E703F0B0F8A36EC01A2E
:10C46000B0F5FA7F2CBF0020012094F9E83084F861
:10C47000210013B1002384F80531204694F80511FA
:10C48000BDE83840FFF7CEBF002038BD10B50346E9
:10C4900090F9050080B193F8030168B15C6B08491D
:10C4A0002046FAF7E7FC40B94FF07F512046FAF7F3
:10C4B000FFFCB0FA80F0400910BD0020FCE700BF8F
:10C4C000ABAA2A3F014B1868704700BF0C1A002026
:10C4D00010B50446006810B103685B6898472046B1
:10C4E00010BD000070B5D0F8F460044616F4805614
:10C4F00088B01FD10D223146FFF782FF0546002884
:10C5000000F0C180CDE905660021069B0A2207A83C
:10C51000CDE9061300F0C4FB01462046FFF762FF99
:10C5200007A8FBF713F906A8FBF710F915B105A842
:10C53000FBF70CF9D4F8F46016F4803640F0A180D3
:10C54000202231462046FFF75BFF0546002800F019
:10C55000A880CDE904660022059B114607A8CDE915
:10C560000522079300F05AFD01462046FFF73AFFE7
:10C5700007A8FFF7ADFF06A8FFF7AAFF05A8FBF77E
:10C58000E5F815B104A8FBF7E1F8D4F8F46016F467
:10C59000803676D1212231462046FFF731FF05460D
:10C5A000002800F08C80CDE904660022059B11462E
:10C5B00007A8CDE90522079300F030FD014620468B
:10C5C000FFF710FF07A8FFF783FF06A8FFF780FF1C
:10C5D00005A8FBF7BBF815B104A8FBF7B7F8D4F82A
:10C5E000F46016F480364CD1222231462046FFF703
:10C5F00007FF0546002870D0CDE904660022059BA0
:10C60000114607A8CDE90522079300F007FD014672
:10C610002046FFF7E7FE07A8FFF75AFF06A8FFF737
:10C6200057FF05A8FBF792F815B104A8FBF78EF8A1
:10C63000D4F8F46016F4803623D123223146204604
:10C64000FFF7DEFE0546002855D0CDE9046600223E
:10C65000059B114607A8CDE90522079300F0DEFCF3
:10C6600001462046FFF7BEFE07A8FFF731FF06A8E8
:10C67000FFF72EFF05A8FBF769F815B104A8FBF733
:10C6800065F808B070BD04232249CDE90103224BAF
:10C690000968009302460D23496806A8FFF754FE77
:10C6A00032E704231B49CDE901031B4B09680093C2
:10C6B00002462023496805A8FFF746FE4BE70423FE
:10C6C0001449CDE90103144B096800930246212364
:10C6D000496805A8FFF738FE67E704230D49CDE94F
:10C6E00001030D4B0968009302462223496805A8FF
:10C6F000FFF72AFE82E704230649CDE90103064B32
:10C700000968009302462323496805A8FFF71CFE29
:10C710009DE700BF9C0D0020801A060010B504465E
:10C72000FFF7E0FE23790BB1A37943B9BDE81040D0
:10C73000034B04491B68986903681B68184710BDC0
:10C740009C0D0020E07D010810B590F905300446ED
:10C750001BB3012380F80431836B13B1002280F8EE
:10C7600004212364A37923B92046FFF7D7FFA379D7
:10C770004BB10A4B64211B68986A03685B68984751
:10C780002046FFF755FE94F8223003B9A363012336
:10C7900084F80331002384F8043110BD9C0D00207F
:10C7A000064B10B503600446FFF78CFE606004F191
:10C7B000080001F077FF204610BD00BF787E010819
:10C7C000642370B50C464568064603FB02552046B7
:10C7D00095F87010FDF70EFC95F9203033B97368A9
:10C7E000597A2046BDE87040FDF704BC95F8241046
:10C7F000F7E700002DE9F04164260C460746904615
:10C80000564345682046A9192831FDF763FB414688
:10C810007868FFF73BFE30B135442046696BBDE8D0
:10C82000F041FDF76FBBBDE8F0810000642310B557
:10C83000446803FB024407C904F15C0383E8070072
:10C8400002F0BCFEA06602F0B7FEE06610BD00007C
:10C850002DE9F74307468846642400F1080116468F
:10C8600001A8A722FCF7D8FE7D6804FB0854D4F881
:10C870008090B9F1000F05D101A8FCF7EFFE03B0DD
:10C88000BDE8F08376B13168606FFAF755F96067FB
:10C890007168A06FFAF750F9A067B168E06FFAF716
:10C8A0004BF9E0676423484603FB08F4FAF7ECF819
:10C8B0002E19743601463046FDF73AFB42463146A2
:10C8C0003846FFF7B3FF00222B19DA679A675A67D9
:10C8D0000022C3F88020CFE74068FFF773BD000057
:10C8E00073B564254D430646406801A92844383095
:10C8F00014460192FFF728FB71680D44EC6302B007
:10C9000070BD0000642307B54B434068C11891F91E
:10C910002010022907D020300DF1070118448DF8AE
:10C920000720FFF79BFA03B05DF804FB642243681D
:10C9300002FB013393F92000003818BF0120704733
:10C940004368642000FB013383F8702070470000C7
:10C950002DE9F843054608460E46FDF715FB18B1CC
:10C9600000242046BDE8F8833046FDF7F7FA044678
:10C970000028F5D16B6893F9F890B9F1000F0DD04C
:10C980003046FDF7AFFDD5F8208006464FF05051F8
:10C9900028F00040FAF76EFA10B12E620124E0E7A9
:10C9A00031464046F9F7BEFF414620F00047304689
:10C9B000F9F7BAFF01463846FAF772F907465FFA07
:10C9C00089F0FAF761F8164981463846FAF7B4F863
:10C9D00001464846FAF74EFAF0B138461149FAF7DF
:10C9E000ABF801461048FAF75BF907466B6A01336A
:10C9F0006B6239464FF07E50F9F794FF4146FAF7E3
:10CA00009BF8394680463046FAF796F8014640468C
:10CA1000F9F78AFF2862A4E70124034FE9E700BF82
:10CA20000000484300002041CDCCCC3D2DE9F3412E
:10CA300005460F4614461E46FFF7C2FE39462846F5
:10CA40002246FFF7D7FE39462846FFF781FF20B37D
:10CA500005F10801992201A8FCF7DEFD6422544388
:10CA60006D68394605EB040808F174082C4440460B
:10CA7000FDF730FAD4F880200132C4F880204EB19E
:10CA8000B24207D352084FF080414046C4F880209C
:10CA9000FDF74EFA01A8FCF7E1FD02B0BDE8F08118
:10CAA000002290F82D10FFF7D3BE000013B5044606
:10CAB000012300210DF10702806A02F079FE0123B3
:10CAC0000C21A06A0DF1070202F072FE70B19DF810
:10CAD0000730012B0AD10D21A06A0DF1070202F0E7
:10CAE00067FE18B19DF80730FF2B00D0002002B080
:10CAF00010BD00007FB50446806A03689B6A9847B2
:10CB000003689B689847A06A0A210368DB6C984712
:10CB10002046FFF7CBFF002869D0002301220B211C
:10CB2000A06A02F021FE002861D0002340222021CB
:10CB3000A06A02F019FE002859D000230122212109
:10CB4000A06A02F011FE002851D000231922092109
:10CB5000A06A02F009FE002849D0A06A03210368F8
:10CB6000DB6C9847A06A03689B6A98470368DB6898
:10CB700098470D21A06A02F0B9FDA36A2046996882
:10CB800004F12D02FFF7A8FE054668B3A36A20460C
:10CB90009A6894F82D10FFF7A3FEA36A1848597AF3
:10CBA0001A7A00919B681749D20801F06BFF204662
:10CBB00094F82C2094F82D10FFF7C2FE94F82E3034
:10CBC000DB0705D50122204694F82D10FFF79AFEC9
:10CBD000A06A0294036842F21071DE6A0A4B039362
:10CBE00004AB13E90C00B047284604B070BDA06A3E
:10CBF000002503689B6A98470368DB689847F3E75A
:10CC00008D7E0108847E01089DCC000870B586B039
:10CC1000044601230621806A0DF1030202F0C8FDDB
:10CC2000002837D09DF803305B0733D50623002159
:10CC3000A06A01AA02F0BCFD60B3BDF90400404245
:10CC4000F9F726FF1449F9F777FF0646BDF9060004
:10CC5000F9F71EFF1049F9F76FFF0546BDF9080007
:10CC60004042F9F715FF0C49F9F766FF94F82D10CB
:10CC70000590204603960495FFF758FE18B102214F
:10CC800003A8FDF7B7F91423204694F82D2003A933
:10CC9000FFF7CCFE06B070BDABAAAA3EFFF7B6BF49
:10CCA000F7B503680D4616461BB90024204603B0AD
:10CCB000F0BD002707603020CDE90073FCF720FBB2
:10CCC000044670B1FFF76CFD104B84F82C602360B4
:10CCD000019B0197A36294F82E3065F3000384F85A
:10CCE0002E3001A8FFF7F4FB6846FFF7F1FB002C9C
:10CCF000DBD02046FFF7FEFE05460028D6D123688C
:10CD000020465B6898472C46D0E700BFC07E0108EC
:10CD100010B50446034B40F8283BFFF7D9FB2046EB
:10CD200010BD00BFC07E010810B50446FFF7F0FF3C
:10CD30002046FCF7EDFA204610BD0000002290F8D6
:10CD40002C10FFF785BD0000F8B504460D461746C8
:10CD50001E46FFF725FD074B002223602B68204667
:10CD6000A3624FF07E532A6084F82D7084F82E6001
:10CD70002363F8BD047F01087FB50446806A036819
:10CD80009B6A984703689B689847A06A037A03F0F8
:10CD90000703022B02D1802102F084FDA06A0A2140
:10CDA0000368DB6C984701230421A06A0DF103029C
:10CDB00002F0FEFC50B9A06A002503689B6A984700
:10CDC0000368DB689847284604B070BD012305213D
:10CDD000A06A0DF1020202F0EBFC0028EBD0012367
:10CDE0000621A06A0DF1050202F0E2FC0028E2D063
:10CDF00001230721A06A01AA02F0DAFC0028DAD098
:10CE000001230821A06A0DF1070202F0D1FC0028DD
:10CE1000D1D001230921A06A0DF1060202F0C8FC5D
:10CE20000028C8D09DF80230C82BC4D19DF804302A
:10CE3000C82BC0D19DF805209DF8033013439DF801
:10CE400007201343B7D19DF80630C82BB3D10A226F
:10CE50000821A06A02F032FC012394220B21A06A6F
:10CE600002F082FC012371221946A06A02F07CFCC8
:10CE7000012300220421A06A02F076FC0123C822CB
:10CE80000521A06A02F070FC012300220621A06A9D
:10CE900002F06AFC0123C8220721A06A02F064FCA8
:10CEA000012300220821A06A02F05EFCC8220123AF
:10CEB0000921A06A02F058FC254BA06A236303688D
:10CEC0000321DB6C9847A06A03689B6A9847036854
:10CED000DB6898471121A06A02F008FCA36A20468B
:10CEE000996804F12C02FFF7F7FC054600283FF48F
:10CEF0006AAFA36A20469A6894F82C10FFF7F0FCFA
:10CF0000144BA26A1B68527A9869134903681E6819
:10CF100094F82C30B047204694F82E2094F82C102A
:10CF2000FFF70EFD94F82D302BB10122204694F826
:10CF30002C10FFF7E7FCA06A0294036843F2D401C7
:10CF4000DE6A064B039304AB13E90C00B0473AE7E3
:10CF50008988083E9C0D0020CC7E010819D000086D
:10CF6000F0B589B0044601233421806A0DF107022F
:10CF700002F01EFC002849D09DF90730002B45DA4D
:10CF800009232421A06A02AA02F012FC00283DD045
:10CF90009DF809009DF80830000440EA03609DF800
:10CFA0000A309DF80C6040EA03209DF80B303604EF
:10CFB00046EA03669DF80D309DF80F5046EA0326B9
:10CFC0009DF80E302D04276B45EA03659DF810305F
:10CFD000001245EA0325F9F75BFD3946F9F7ACFD88
:10CFE00005903012F9F754FD3946F9F7A5FD069082
:10CFF0002812F9F74DFD3946F9F79EFD0A230790EF
:10D0000094F82C20204605A9FFF710FDA06A02F035
:10D01000F3FB09B0F0BD0000FFF7A2BF73B50368D2
:10D020000D4616461BB90024204602B070BD0022F2
:10D03000026034200193FCF763F9044620B13346C3
:10D040002A4601A9FFF780FE01A8FFF741FA002C4C
:10D05000E9D02046FFF790FE05460028E4D123687A
:10D0600020465B6898472C46DEE7000010B5044672
:10D07000034B40F8283BFFF72BFA204610BD00BFBA
:10D08000047F010810B50446FFF7F0FF2046FCF7C7
:10D090003FF9204610BD000010B503680281194316
:10D0A0004368016001334360044B1B68DC6AA16282
:10D0B000D96A40688885DB6ADA8510BD9C0D00203E
:10D0C00000487047101A002013B50446143000F0D1
:10D0D000ABF94FF0FF3320460B496366FEF706FCC1
:10D0E00009230DF1070104F11C008DF80730FEF74C
:10D0F000ABFE064B1A6812B1054802F037FA20461B
:10D100001C6002B010BD00BF4C7F01081C1A00203B
:10D11000207F01082DE9F0419AB005A9FDF7A8FF8D
:10D12000002830D0194D0EAC0FCD0FC40FCD0FC459
:10D1300095E80F0084E80F00002103254FF07E588A
:10D140000D220AA809910AF0DDFA114B09AE1B68FD
:10D15000104F08960EAC0393237A03988DF81C3079
:10D16000236811220693E36831460093C06A3B4668
:10D17000FCF792FB0022414605A8FEF713FB013D98
:10D1800004F11004E8D11AB0BDE8F081F477010889
:10D190009C0D0020407F010838B5836E0446002BAB
:10D1A0003DD14FF07E53036590F91C30013B122BAB
:10D1B00022D8DFE803F00A2116353D4551215D658F
:10D1C0006D7521217D2195899D004820FCF798F8F7
:10D1D000054680B10022214603F0D0FC4A4B2B606B
:10D1E00009E06820FCF78CF8054620B1FF230022F7
:10D1F000214604F007F9A566A06E50B103689B684C
:10D20000984730B9A06E10B103685B689847002357
:10D21000A366A36E002B74D0012384F8633038BD5D
:10D220006820FCF76DF805460028E4D00023DEE70F
:10D230006820FCF765F805460028DCD00123D6E716
:10D240004420FCF75DF805460028D4D00022214692
:10D2500003F094FC2D4BC2E74820FCF751F805463B
:10D260000028C8D02A4B0022214603F025FDC2E742
:10D270004820FCF745F805460028BCD0254BF2E7CE
:10D280004820FCF73DF805460028B4D0224BEAE7D9
:10D290004820FCF735F805460028ACD01F4BE2E7E4
:10D2A0004820FCF72DF805460028A4D01C4BDAE7EF
:10D2B0004420FCF725F8054600289CD00022214692
:10D2C00003F05CFC174B8AE76820FCF719F8054669
:10D2D000002890D00E4B0022214603F0A9F98AE7DE
:10D2E0006820FCF70DF80546002884D0094BF2E7CA
:10D2F0006820FCF705F8054600283FF47CAF074B93
:10D30000E9E763618BE700BF7CC20108F8C201084E
:10D310000000A040000020410000A0410000F041BA
:10D3200000007042DCC1010810B50446FFF7F2FEB0
:10D3300094F91C3023B12046BDE81040FFF72CBF04
:10D3400010BD000041B990F91C302BB1806E18B1AE
:10D35000036811461B6918470020704713B504463F
:10D36000B9B990F91C30A3B1836E93B102F026F9DC
:10D370006063A06E03685B6998470346A06E53B173
:10D38000036804F124019B699847636A84F83800B4
:10D39000236202B010BD00230193036801A9DB687A
:10D3A0009847019B84F838002363F2E729B990F984
:10D3B0001C00003818BF0120704700207047000093
:10D3C000034651B990F91C0040B193F8380028B1D8
:10D3D000986E003818BF0120704700207047000089
:10D3E00010B504460021FFF7B9FF627820461146C8
:10D3F000FFF7E6FF014630B184F862202046BDE821
:10D40000104003F039BD2046FFF7DAFF0028F5D0C1
:10D4100084F86210F2E7000021B990F91C300BB1DA
:10D42000006B70470020704710B504460249FEF7B4
:10D430005DFA204610BD00BF6C7F010808B50449A5
:10D44000F9F786FF0028034818BF002008BD00BF79
:10D45000AC7F0108BCBB010810B50C46FFF7EEFF1E
:10D4600010B183682360006910BD000070470000A0
:10D4700010B4064B064A1B680649986903681C6885
:10D48000537EA446127E10BC604700BF9C0D002056
:10D4900080650008D0BB0108002070470E2070474F
:10D4A00090F8F004C0F340007047000000F5A06061
:10D4B0007047000090F9F80470470000C0F8F414B9
:10D4C000012070472DE9F7430C68064614F000541C
:10D4D0000D4694461F46BDF828E040F0918091F833
:10D4E0000C80B8F1080F00F28B80D0F8008508F1AD
:10D4F0000108C0F800854FF0300888F31188D0F893
:10D500003C80D8F8089019F0806F19D1D8F80840FD
:10D51000240114D4D8F8084014F080546CD1D0F809
:10D5200008550135C0F80855D0F80C55002D65D1C7
:10D53000CDF800E0FBF77CFF84F3118859E001246B
:10D540002B6804F11802002BB8BFDB004FEA02126F
:10D55000B4BF43F004035B0548F802302B6813F0B6
:10D56000804F4FEA04131CBF08EB0301D1F8802160
:10D5700043441CBF42F00202C1F880212A7B08EB21
:10D580000418C3F88421AA6805F10C01C8F88C219D
:10D590006A68C8F88821D3F8802142F00102C3F8F4
:10D5A00080212A46630106EB4414C4F890C4C4F8F1
:10D5B000947404F5936452F8040B8A4244F8040B03
:10D5C000F9D112883344228093F8AC140EF0030290
:10D5D00021F00B010A4383F8AC24002383F3118864
:10D5E00062463B4629463046CDF800E0FBF720FF77
:10D5F000012003B0BDE8F0830224A1E720469BE7A9
:10D600004FF0FF30F5E700002DE9F04F90F838308B
:10D61000032B40F095800E2A00F29280002900F042
:10D620009180302383F31188C46B6FF07845D4F870
:10D63000003243F00103C4F80032C46BD4F8003266
:10D6400023F47C53C4F80032C46BD4F8003243F4A2
:10D650006063C4F80032C36B3B4CC3F81442002330
:10D66000C46BC4F80432C46BC4F80C5290F8F8547C
:10D670009D4218BF0E25DAB9C36B05F1480143F886
:10D680003120C36B03EBC1035A600123C26B03FA61
:10D6900005F5C2F81C52C26BD2F8003223F0010328
:10D6A000C2F80032002383F311880120BDE8F08F17
:10D6B0004FF0010801F10409EF189A42D0F83CA09C
:10D6C00008FA07FE35DD51F833B059F833C0BBF125
:10D6D000000F02DBBCF1000F26DB4FEACB044FEA60
:10D6E000CC0644F004041BF0804F18BF44F0020441
:10D6F00048374AF83740C46BBCF1000FB8BF46F05A
:10D7000004061CF0804F18BF46F0020604EBC70465
:10D710006660C66BD6F81C424EEA0404C6F81C428A
:10D7200001330E2BC8D1B6E74FEA4B544FEA4C56A3
:10D73000D9E7DAF81C4224EA0E04CAF81C42EFE7E3
:10D740000020B3E70846B1E7AAAAAA0A38B50446FA
:10D75000D0F884040D4602F039F91F280AD9202296
:10D760002946D4F8840402F0A7F9A0F12003584216
:10D77000584138BD0020FCE708B5302383F31188F9
:10D78000D0F8840402F0F8F8002383F3118808BD70
:10D790000022026082814260826070470022002382
:10D7A00010B5C0E900230023044603810C30FFF7C5
:10D7B000EFFF204610BD00002DE9F04190F8F03455
:10D7C000044613F0040FC3F3800008BF104660F353
:10D7D000820384F8F03404EB411595F8AC3488B03A
:10D7E000D8074FEA4118DDE90E6737D5002A37D050
:10D7F000190735D46846FFF7D1FF05F5936303AAEF
:10D8000005F594659446186859680833ACE8030038
:10D81000AB426246F6D118686946CCF800009B8896
:10D820002046ACF804300123ADF808302368CDE978
:10D8300000679B6C9847A04498F8AC341A070FD443
:10D8400043F0080388F8AC34D4F80C3504F5A6642A
:10D85000013344F8243C44E9026701E0002AEAD19C
:10D8600008B0BDE8F08100002DE9F0479A46054672
:10D8700088469146302388B083F311886846FFF7C5
:10D880008DFFD5F8840402F089F81F282BD92022B7
:10D890006946D5F8840402F08DF9202823D1444646
:10D8A00003AE05AB374603CF9F42206061603E4622
:10D8B00004F10804F6D138682060BB88A380DDE954
:10D8C0000023C9E90023BDF80830AAF8003000237E
:10D8D00083F3118853464A464146284608B0BDE8BE
:10D8E000F047FBF74DBD002080F3118808B0BDE87C
:10D8F000F08700002DE9F0470446284B0E4640F81B
:10D90000043B00F0CFFE1822002104F11C0009F0B6
:10D91000F9FE2046224B04F1700740F8403BFFF728
:10D9200037FF04F15000FFF739FF3D4604F58E68DC
:10D9300028462035FFF732FF4545F9D14FF4806383
:10D94000C4F87074C4F87434002701234FF0000841
:10D950004FF00009C4F88454C4F87874C4F87C7497
:10D9600084F8803484F8883404F5966504F5A26A56
:10D9700045E90889A5F11800FFF70AFF203545F8A9
:10D98000287C5545F4D184F8F86416B1054801F0B7
:10D99000EDFD054B2046E363BDE8F087047C0108FC
:10D9A00008BC0108E0BB01080064004010B5044653
:10D9B000034B19784A1C1A70FFF79CFF204610BDD4
:10D9C000241A00202DE9F04300294FD0284F294B7D
:10D9D000B7FBF1F499428CBF0A231123B4FBF3FC8B
:10D9E000581E03FB1C43C5B22BB102280346F5D8D1
:10D9F0000020BDE8F0830CF1FF36B6F5806FF7D25A
:10DA00004FF47A74C5EBC50E0EF103034FEAE30938
:10DA100009FB0444C3F3C703E81AC0B209F10108C3
:10DA20008044B4FBF8F4B4F5617FC2BF0EF1FF335C
:10DA3000C3F3C703E81A03F10104C8BFC0B2E4B2DC
:10DA400004440CFB04F4B7FBF4F4A142D0D1013B35
:10DA5000DBB20F2BCCD80138C0B20728C8D80021C0
:10DA60001071168001209170D370C2E70846C0E79C
:10DA7000005125023F420F0070B505460E464FF497
:10DA80007A74EB6B01205B6803F00103B34204D0AE
:10DA900008F0DCF8013CF4D1204670BD30B5C26B13
:10DAA000936913F0700F1CD000230E4C936100EBB0
:10DAB000431202F5956192F8AC2455070ED59207F2
:10DAC0000CD5C26B54F8235095600A7942F00402D9
:10DAD0000A71D0F814250132C0F814250133032B44
:10DAE000E5D130BDF4BB010873B51D46C36B1646C6
:10DAF0009A680446D20709D501219A689960C2F351
:10DB000040020021CDE90065FFF756FEE36B9A68FD
:10DB1000D1050BD54FF480719A6820469960C2F305
:10DB200040220121CDE90065FFF746FEE36B9A68CC
:10DB3000D2030BD54FF480319A6820469960C2F326
:10DB400040420221CDE90065FFF736FED4F8F40427
:10DB500038B1D4F830350133C4F8303503681B6967
:10DB60009847204602B0BDE87040FFF797BF00001D
:10DB7000F8B50446C66B002940F0898006F10C0711
:10DB80003868850700F08C8038684FEA011CC006B1
:10DB900042BFD4F820050130C4F8200506EB01107F
:10DBA000D0F8B011D0F8B051490746BFED0845F0A4
:10DBB00000456D0D2564D0F8B011890744BF45F0CC
:10DBC00080452564D0F8B40106EB0C0100F00F008D
:10DBD00084F84C00D1F8B80104F14C0584F84400F5
:10DBE000D1F8B801000A84F84500D1F8B801000C5A
:10DBF00084F84600D1F8B801000E84F84700D1F847
:10DC0000BC0184F84800D1F8BC01000A84F849003E
:10DC1000D1F8BC01000C84F84A00D1F8BC1104F121
:10DC20005C00090E84F84B103821396004F1400182
:10DC300051F8046BA94240F8046BF9D109880180BE
:10DC4000C4E9142300232146A4F8583051F8503B6E
:10DC500020469B6C9847E8B1D4F818350133C4F8D6
:10DC6000183594F8F034D4F8F40443F0040384F83D
:10DC7000F03438B1D4F830350133C4F830350368A6
:10DC80001B6998472046BDE8F840FFF707BF06F13B
:10DC9000100775E7D4F81C350133C4F81C35E0E7EC
:10DCA000F8BD000010B5044601F08AFC02460B46A0
:10DCB00052EA030102D0013A63F100030449086803
:10DCC00020B12146BDE81040FFF752BF10BD00BF94
:10DCD000201A0020F0B5302181F311880021154E63
:10DCE00000F5926400EB411505F5956C95F8AC5480
:10DCF0006F0715D4ED0613D5D4E9007597429D4101
:10DD00000ED2C56B56F82170AF609CF8045045F0F8
:10DD100004058CF80450D0F810550135C0F81055A2
:10DD20000131032904F12004DCD1002383F311889D
:10DD3000F0BD00BFF4BB010808B5302383F31188A0
:10DD4000FFF7ACFE002383F3118808BDF8B5C36B61
:10DD5000044698680E4600F0E050B0F1E05F1FD036
:10DD6000E8B1302383F31188002504F5936704EBB1
:10DD7000451393F8AC341A0706D50135032D07F186
:10DD80002007F4D1012007E05B07F6D4394630467E
:10DD9000FBF7A2FB0028F0D1002383F31188F8BD24
:10DDA0000120FCE708B5302383F31188D0F8840400
:10DDB00001F0F4FD002383F3118843090CBF012017
:10DDC000002008BDF8B51D46002313700F46064617
:10DDD0001446FFF7E7FF80F00100387025B12946AF
:10DDE0003046FFF7B3FF2070F8BD0000F8B50C46D1
:10DDF00015461E46074601F0E3FB0B462178024616
:10DE000009B9287850B13846FFF764FFFFF794FF4F
:10DE100033462A462146FFF7D5FF0120F8BD000012
:10DE200038B50446302080F31188164BDA6942F089
:10DE30000072DA611A6942F000721A611A6922F0FE
:10DE400000721A61002383F3118894F8F03413F000
:10DE5000010516D1A9B180F311880321132007F021
:10DE600035F80321142007F031F80321152007F0BD
:10DE70002DF894F8F03443F0010384F8F03485F37E
:10DE8000118838BD001002402DE9F04790F8F834B1
:10DE90000446012B0F46154688B000F28780844E59
:10DEA00056F8232042B946F8230001F023F894F8ED
:10DEB000F83400EB8300C463D6F80090676384F8FD
:10DEC0003850B9F1000F63D094F8F834012B6FD0BB
:10DED00001212046FFF7A4FF302383F311884FF080
:10DEE0000008E26B136823F002031360E26B13680F
:10DEF00043F001031360E36BC3F8148088F31188C7
:10DF000001212046FFF7B8FD002800F09280D4F8E8
:10DF1000840401F031FDA14604F1600A20220021B1
:10DF2000684609F0EFFB02A8FFF732FC6A46CDF81D
:10DF3000188009F592630DF1180C164603CE66455C
:10DF400018605960324603F10803F6D1306809F1D0
:10DF5000200918603279CA451A71DFD1002694F879
:10DF6000F0346A466FF3820384F8F0343946204671
:10DF7000ADF80060ADF802608DF80460FFF722FD97
:10DF8000E36B48BB4FF400421A6008B0BDE8F0876D
:10DF90004FF4A760FBF7B4F9804610B14946FFF78C
:10DFA000A9FCC6F80080B8F1000F8DD10020ECE785
:10DFB000306803689B6B98470146002888D1306819
:10DFC000FFF72EFF30682A46036839465B6898479A
:10DFD00000287FF47DAFE9E76122022D0CBF4FF0EE
:10DFE000004100211A609DF802309DF803201B06B5
:10DFF000120402F4702203F040731343BDF80020B2
:10E000002046C2F3090213439DF80420120502F4CE
:10E01000E0021343E26B0B43D3611322E36B3146FF
:10E020005A61E26B136823F001031360FFF724FDCC
:10E0300008B9E36BA6E794F8F83493BBE16BD1F829
:10E04000002242F00102C1F80022E16BD1F8002267
:10E0500022F47C5222F00E02C1F80022E16BD1F8CA
:10E06000002242F46062C1F8002241F6FF71E26BC7
:10E07000C2F81432E26BC2F80432E26BC2F80C123E
:10E08000E26BC2F84032E26BC2F844320122E36B29
:10E09000C3F81C22E26BD2F8003223F00103C2F86D
:10E0A000003294F8F03443F0020384F8F0346CE763
:10E0B000201A002008B501F083FA02460B4652EA06
:10E0C000030102D0013A63F100030449086808B172
:10E0D000FFF70AFDBDE8084006F09ABA201A0020B2
:10E0E00008B50020FFF7DEFDBDE8084006F090BA55
:10E0F00008B50120FFF7D6FDBDE8084006F088BA54
:10E100007047000013B5046800920B462469A047CD
:10E1100002B010BD7047000000207047002070471B
:10E1200013B56C4684E8060000F1140394E803007C
:10E1300083E8050002B010BD0020704713B56C469F
:10E1400084E8060000F10C0394E8030083E805006E
:10E1500002B010BD0023C0E90333704782B002ABA8
:10E1600003E9060002B070477047000000207047C6
:10E170007047000080F82D107047000080F82C10C8
:10E180007047000001207047806A0430704700002B
:10E1900080F834107047000000207047012070475D
:10E1A00008B503685B689847002008BD03685B6892
:10E1B00018470000704700007047000070470000DB
:10E1C0001FB502AC84E80C00009094E80C00806A53
:10E1D00003F01EFE04B010BD806A03F071BE0000A3
:10E1E00010B50446006B07F075FF044B606A2360AE
:10E1F00008B1FBF791F8204610BD00BFA4BC010890
:10E2000010B50446FFF7ECFF2046FBF781F82046E7
:10E2100010BD000070B5044688B0503007F082FA97
:10E22000104B1420CDE905340F4B04940793FBF7F2
:10E2300067F8054690B194F848300C4E08AA06EBF2
:10E24000031601AB12E9030083E80300059B28468F
:10E2500000937279049BB17900F048FAE56108B047
:10E2600070BD00BFB5E10008B9E10008F4BC0108C9
:10E2700070B500BB012202210F4800F03DFC0122D5
:10E28000054603210D4800F037FC0126044605F041
:10E290000F0106FA01F125F00F00022206F01CFA28
:10E2A00004F00F0106FA01F124F00F000222BDE88C
:10E2B000704006F011BA70BD070C0140060C014019
:10E2C000B0FA80F04009704738B50A4B0A4C036039
:10E2D00000230546204684F84830FFF79BFF0123C2
:10E2E000064A2846E26484F83C30226484F84430CC
:10E2F00038BD00BF0CBD0108281A0020A08601000F
:10E3000070B51E4600230D466421C0E90333C0E901
:10E31000053303711D4B044603601D4B80F82D200F
:10E3200001FB05338362022380F82C309DF8103006
:10E33000427280F83530059B16498363EB0043F049
:10E3400001030372134630302A4600F08BFBA36AA8
:10E35000DA6CB24217D91E64A36A0F49DE640F4B10
:10E360009E429EBF0122A36A83F844200C4B1B6887
:10E370009869A36ADA6C03681E684FF47A73B2FB7B
:10E38000F3F32A46B047204670BD00BF24BD010804
:10E39000281A002054BC010860BC0108A0860100B6
:10E3A0009C0D0020F7B516461F460D4689B93C2046
:10E3B000FAF7A6FF044648B1099B324601939DF83F
:10E3C0002030294600933B46FFF79AFF204603B0D2
:10E3D000F0BD0024FAE700002DE9F04F0446164690
:10E3E00089B00693836ADDF8488093F84830574D2A
:10E3F0001B01E8581FFA88F9079106F0F1FDA06AA1
:10E40000CDF8009006ABB2B207A903F071FD074644
:10E4100050B9A36A93F848301B01E85806F0E4FDB0
:10E42000384609B0BDE8F08F4FF0000A06EB08034C
:10E430000593A26A4649D36C4FF47A7BB1FBF3F3A0
:10E440000599D0694B43B3FBFBF3A16B5B00013330
:10E450008B4238BF0B46049300F09EFAA16A91F8F4
:10E4600048303C311B01E85806F06EFD302383F341
:10E470001188384B00211B68DA6A536B01335363F0
:10E4800081F3118840F2E730DDF810C00023ECFB87
:10E490000B014FF47A72F8F751FDA36A94F82D102E
:10E4A00093F848C04FEA0C1C96BB00904346069A6E
:10E4B00055F80C0006F07EFDA36A834693F84830B9
:10E4C0001B01E85806F04EFDA36A0121D86900F04F
:10E4D00059F9A06A90F848301B01EB589B681B065D
:10E4E00021D5FEF7EDFD40F293124FF40021FEF727
:10E4F000D3FDDDE906214B46A06A03F01FFDA36AA8
:10E50000002793F848301B01E85806F06DFD87E7B7
:10E51000069BCDE901800093079A334655F80C001D
:10E5200006F02EFDC8E7BBF1000F05D14B46DDE933
:10E53000062103F003FD6CE794F82C200AF1010A90
:10E540005FFA8AF39A42BFF474AFD2E7F4BC0108D1
:10E5500000127A009C0D00202DE9F7430446806AE2
:10E560000E46043017469846DDF8289000F0A6F8CD
:10E57000054668B91F4BA2681B681F499869036864
:10E580001E6894F82D30B047284603B0BDE8F083EC
:10E5900094F83520A36ABAB1032283F83C2094F89A
:10E5A000345005B396B9B8F1000FEDD0B9F1000FB2
:10E5B000EAD0002243461146CDF82890204603B009
:10E5C000BDE8F043FFF708BF0122E6E7002FEAD0DD
:10E5D00000233A46314620460093FFF7FDFE00280F
:10E5E000E1D10546D0E743463A463146CDF828907A
:10E5F000E4E700BF9C0D002074BC010808B5B02101
:10E60000044803F0EFFBBDE808400020024A03493C
:10E6100008F0DCBA281A0020C8240020BDE1000858
:10E62000036800211B68184708B5043007F0E8F8B4
:10E63000012008BD043007F0D9B800002DE9F843E7
:10E6400006460D4621B9043007F0AEF8012424E057
:10E6500003685B6898470028F8D100F0B1FF88464E
:10E660004FF47A7107460E4B4D43D3F80090D9F81A
:10E670002800C82103689B689847336830465B6868
:10E68000984704460028E1D100F09AFFC01B61EBD7
:10E690000801A84271F10003E9D32046BDE8F883E0
:10E6A0009C0D002010B50446034B40F8043B07F0D6
:10E6B00039F8204610BD00BF84BD0108034BC06877
:10E6C000DB68C31A58425841704700BF802E0020B3
:10E6D00038B50024044D2846013407F023F8102CE7
:10E6E00005F12005F7D138BD901A002082B010B591
:10E6F0000446039300239142C0E90033C0E902338A
:10E7000004F108030174427484BF02744174DDE9AA
:10E71000030184E80300DDE9050183E803002046E6
:10E72000BDE8104002B070470F2838B50AD8074C32
:10E7300004EB4014A568204607F036F815B1A3682D
:10E740009D4201D1002038BD0120FCE7901A002035
:10E750000F2938B5044615460FD8084800EB41107C
:10E7600007F04EF84DB1064B1B6833B10C21227CEB
:10E7700001FB02339A6801329A6038BD901A00207A
:10E780008C1A002038B5002304460D460A468374CF
:10E79000417CFFF7DDFF2A462046217CBDE838405A
:10E7A000FFF7D6BF2DE9F04FDFF8CC808146D8F8CF
:10E7B00000308DB023B9CC20FAF7A8FDC8F80000CE
:10E7C00048462E4900F03CFF0027DFF8B4A0DFF8F0
:10E7D000B4B00C2303FB07F6D8F80030FDB29A5909
:10E7E000991922B94A6812B98A68002A3DD00724CB
:10E7F000B5FBF4F498599A590B924A6806928A68C4
:10E8000007924A689B5908920993C4EBC403ED1A16
:10E81000F8F73AF95146F8F78FF90B9A069B0A90E8
:10E82000D0180130F8F730F90A9B01461846F8F77E
:10E8300037FAF8F71BF8099B01350293089B01345E
:10E840000193079BEDB2E4B2CDE9040122460093A7
:10E8500059462B46484600F0F3FE0022D8F8003017
:10E860009A51D8F8003033445A600137102FB0D194
:10E870000DB0BDE8F08F00BF8C1A00209CBD0108D0
:10E880000000C842A3BD010809C8184738B5037C79
:10E8900004460F2B10D83E4D580105EB4313D969A0
:10E8A00051B1A14208D014302844FFF7EDFF237C7A
:10E8B00005EB43150023EB61637C0F2B10D8344D1F
:10E8C000580105EB4313D96951B1A14208D0143066
:10E8D0002844FFF7D9FF637C05EB43150023EB6168
:10E8E000227C0F2A04D82A4B03EB4213DB693BB18D
:10E8F000627C0F2A26D8264B03EB4213DB690BBB45
:10E9000021462046FFF7C0FF237C0F2B0BD8D4E90C
:10E9100002011F4A02EB4313143383E80300237CF4
:10E9200002EB4312D461637C0F2B0BD8D4E90201B4
:10E93000174A02EB4313143383E80300637C02EBB2
:10E940004312D46113480268B2B1237C0F2B07D85D
:10E950000C214B43E57CD1188DB1D1580131D150F8
:10E96000637C0F2B08D80C2253430268E07CD1183B
:10E9700048B1D1580131D1500123A37438BD4B683F
:10E9800001334B60ECE74B6801334B60F4E700BFA9
:10E99000901A00208C1A002038B50446007CFFF73E
:10E9A000C3FE0546607CFFF7BFFE002D08BF05468D
:10E9B0002046E574BDE83840FFF768BF112200210A
:10E9C000034B013AC3E9051103F12003F9D1704764
:10E9D000901A00200CB430B585B008AC0A4607493F
:10E9E00054F8043B0D6800940146E86A0394FAF772
:10E9F00033FF05B0BDE8304002B070479C0D0020E9
:10EA000013B5054C0093246813460A460146E06A94
:10EA1000FAF722FF02B010BD9C0D00202DE9F8434B
:10EA200013460E4617460A46002180460846FFF761
:10EA3000E7FF041E04DC4FF0FF342046BDE8F883F6
:10EA400004F101090121484607F040FB0546002872
:10EA5000F1D03B4632464946FFF7D2FFC8F8005096
:10EA6000EBE700000EB403B503AA52F8041B0192B1
:10EA7000FFF7D4FF02B05DF804EB03B0704700006D
:10EA8000F8F770BC0FB407B5054B04A951F8040B97
:10EA90001B680191984703B05DF804EB04B0704720
:10EAA000100D0020704700000020704770470000E4
:10EAB000704700007047000000207047704700005A
:10EAC00000207047002082B002A901E90C0002B0CA
:10EAD00070470000002070470079704700207047A1
:10EAE000002070470020704701207047014B0360F1
:10EAF000704700BFE0BD01087047000013B504680F
:10EB000000920B462469A04702B010BD0020704758
:10EB100000207047704700000020704700207047B9
:10EB200082B002A901E90C0002B0704770470000F2
:10EB300000207047704700007047000001207047B8
:10EB4000012070470120704728307047002082B0B4
:10EB500002A901E90C0002B07047000070470000F4
:10EB60007047000070470000084607F09FB900009A
:10EB7000084607F041BA000073B51E460C4615461C
:10EB8000011D102201A8FAF747FD3246294620460A
:10EB900007F0D4F9044601A8FAF760FD204602B058
:10EBA00070BD000013B50C460D22011D01A8FAF737
:10EBB00033FD204607F08CF9044601A8FAF74EFD14
:10EBC000204602B010BD000007F06EB9084607F0FD
:10EBD00067B90000084607F05BB9000010B50446AD
:10EBE000054B40F86C3B00F089FE04F1580000F042
:10EBF00085FE204610BD00BF68C5010808B530205D
:10EC0000FAF77EFB70B100230222C0E90333C0E9AA
:10EC100005330371037A62F302030372024B03604C
:10EC2000024B836208BD00BF5CBE01081CC1010825
:10EC300010B4BDF80440019410BC00F09BBB000070
:10EC400010B4BDF80440019410BC00F041BB0000BA
:10EC500000F056BB00F084BB10B5044B04460360C3
:10EC6000406A08B1FAF758FB204610BDA4BC010861
:10EC700010B50446FFF7F0FF2046FAF749FB20469F
:10EC800010BD0000002110B504461B4B90B003607E
:10EC90000171102200F54A7008F034FD04F54E7041
:10ECA000FFF700FD172007F0FBF8144B10A9CDE982
:10ECB0000B34134B0A94CDE90D34124B02460F93DB
:10ECC00005AB11E9030083E8030003ABDDE90C01A8
:10ECD00083E8030001ABDDE90A0183E803000A4B86
:10ECE00004F10801009304F55970234601F054F82B
:10ECF000204610B010BD00BF9CBF010841EC0008C9
:10ED000051EC000855EC000831EC00081B4B10B525
:10ED100003601B4B044643601A4B1B4A836000236D
:10ED200002611A4A1A4942611A4AC1618261026447
:10ED3000194A1A4942641A4A01628264194A1A49F4
:10ED4000C2641A4A41620265194A1A4942651A4A5E
:10ED50008162826519491A4AC162C26519491A4A13
:10ED60000163026619491A4AC36041634266C3637C
:10ED700000F0FAFB174B2046236010BD38BE010897
:10ED8000DC230020E0230020C424002040200020B9
:10ED9000B01C00206C1E00207C1E0020B81C00202F
:10EDA0008C1E0020A01E00209C1D0020E01F0020C3
:10EDB000F01F0020E423002000200020C81D0020B8
:10EDC00010200020140D002020200020141D002001
:10EDD00030200020FCBE010808B5302383F31188E1
:10EDE000074B1B689A68996B8A4201D0824200D215
:10EDF0009860986306F0ECFD002383F3118808BD4A
:10EE0000101D00202E4D2F4E08B5F2682B602E4BA2
:10EE1000B4201A6006F002FFFFF75AFC07F066FA0A
:10EE20002A4B4FF4E1311C68206CFAF7A3FC2069EF
:10EE300003681B689847A06A03681B6898470A2004
:10EE4000FFF7CAFF07F018FB40B11321204807F075
:10EE500023FB4C221E49881808F046FC01221D4B5A
:10EE600028689A7303681B6898471B4B1B6813B18B
:10EE70001B6ADB0701D507F0CBFAE06A03685B6821
:10EE8000984738B1FEF71CF94FF497724FF40061C0
:10EE9000FEF702F90F4803F0DFFAA06A0D4C036891
:10EEA0001B6B9847F3680D4AB420DA6106F0B6FE92
:10EEB000286803685B689847204603F0CDFAF7E7B7
:10EEC000301D0020802E0020101D00209C0D0020F1
:10EED000CC1D0020E4230020DC24002024BE0108F7
:10EEE000014B1868704700BF101D00200048704794
:10EEF000341D002000487047341D002038B53A48C2
:10EF000000F044FF394D3A4800F040FF394C3A4890
:10EF100000F03CFF0321284603F00EFE374922464D
:10EF2000284607F053FE364800F030FF354800F021
:10EF30002DFF354800F02AFF344800F027FF344801
:10EF400000F024FF334800F021FF3348FFF7BCF9FD
:10EF5000324B334A334D1A60334800F065FE284681
:10EF6000FFF790FE224631492846314D07F02EFE2C
:10EF70003048FFF7BBFD28462F4B2422002140F8E4
:10EF8000043B08F0BFFB05F13400FFF78BFB4FF0AB
:10EF9000FF332A492246EB64284607F017FE302249
:10EFA000274B28481A714FF47A72DA804FF4FA62CC
:10EFB0001A81254A254D1A6003F0F2F900222846ED
:10EFC000234B83F89C20234A1A60234B40F8043BD0
:10EFD000FFF768FB22462846204907F0F7FDBDE809
:10EFE00038401F48FFF792BE6C1E0020A01E002074
:10EFF0007C1E0020C82400208C1E0020DDEB0008B1
:10F00000E01F0020F01F0020002000201020002022
:10F010002020002030200020DC230020E0230020DE
:10F02000C0BE010840200020C42400205DEB000881
:10F03000B81C0020B01C00204CC3010861EB000884
:10F040009C1D0020E42300203CC00108141D00206A
:10F05000C81D002034C70108D8BE010865EB0008B0
:10F06000341D002070470000037933B14FF448731A
:10F070000830086001201360704718467047000090
:10F0800000F5597001F052B810B50446007948B146
:10F0900000F094FAD4F86033C01AB0F5FA6F2CBFC0
:10F0A0000020012010BD000008B5FEF709F8A222DB
:10F0B0004FF40031FDF7F0FF002008BDF8B506461B
:10F0C000EAB10127CC0801390A44C2F3CC05A542B4
:10F0D00015D3632C0ED8630906EB830304F01F02DB
:10F0E00007FA02F1D3F828230A43C3F8282301348E
:10F0F000A4B2ECE7FFF7D8FF0028ECD1F7E7F8BDA2
:10F10000172110B50446A0F8581318220548FFF738
:10F11000B9FC04F5597001F047F810B9024800F045
:10F1200025FA10BD00BF010826BF010810B50179FE
:10F13000044671B9102200F54A7008F0E3FA20463F
:10F14000FFF7DEFF022103482171BDE81040FFF701
:10F1500099BC10BD44BF0108B3F5487FF8B5074618
:10F160000E4614461D460DD8C3F548739A4209D879
:10F170000834FFF7DBFF2A4630463919BDE8F8406E
:10F1800008F0B2BAF8BD0000B3F5487F2DE9F341AD
:10F1900005460E4690461C4622D8C3F54873994250
:10F1A0001ED801F10807074422463946404608F0B8
:10F1B0008BFAA8B12846FFF7B9FFF12205F54E7189
:10F1C00001A8FAF729FA22464146384608F08CFA97
:10F1D00028463146A2B2FFF771FF01A8FAF73EFABE
:10F1E00002B0BDE8F081000037B50C4605460121AC
:10F1F00001A8FAF7F7F9E100082289B205F559707C
:10F2000000F0D4FE044601A8FAF7F8F9204603B04E
:10F2100030BD00002DE9F74F0379044603B300F534
:10F220004A7300F54E7853F8042B32B94345FAD1AE
:10F2300000F0C4F9C4F8600312E000250123C5F30F
:10F240004A1604EB8606D6F8282305F01F0703FAB2
:10F2500007F717421FFA85FA05D10135642DEED163
:10F2600003B0BDE8F08FED004FF4887241460835D9
:10F2700001A8FAF7D1F9635904EB050BC4F8503330
:10F28000DBF8043001A8C4F85433FAF7E7F923791E
:10F2900004F55479022BE3D151462046FFF7A4FF31
:10F2A0000028DDD04FF49C72414601A8FAF7B4F96A
:10F2B00008225946484608F007FA28B9D6F82833F4
:10F2C00023EA0703C6F8283301A8FAF7C7F9C7E706
:10F2D00038B51C46094B15461B68B0F858035B6BE4
:10F2E00001441A68184612689047BDF81020411969
:10F2F000204608F0F9F9012038BD00BF9C0D002020
:10F300002DE9F74306460F460524DFF850904FF4E9
:10F310007A7101A8FAF766F9D9F80080B6F858139F
:10F32000D8F8340039440368DB689847054630B1A3
:10F3300001A8FAF763F9284603B0BDE8F083D8F8CE
:10F34000280001210368013C5B68984701A8FAF78F
:10F3500055F914F0FF04DAD1EDE700BF9C0D002051
:10F36000034B1B68DB6A93F89C0080F00100704738
:10F370009C0D00202DE9F04F04460F4687B0039303
:10F38000274BB4F85813D3F800903944D9F8340017
:10F3900090460368BDF840B01B689847052500EB10
:10F3A000080A012105A8FAF71DF9D9F834005146D9
:10F3B0000368039A1E695B46B047064630B105A84C
:10F3C000FAF71CF9304607B0BDE8F08FD9F82800ED
:10F3D00001210368013D5B68984705A8FAF70EF91B
:10F3E00015F0FF05DDD12046FFF7BAFF0028E9D070
:10F3F00000F0E4F841F28832D4F85C33C31A934247
:10F40000E0D9C4F85C0304F5597000F0BBFE5B461C
:10F410000090424639460348FFF734FBD2E700BF6D
:10F420009C0D002064BF010870B51D46164B1B687B
:10F4300013B11B6ADB0725D5144B1E68F46A94F8D8
:10F440004630C3B9124BA4F84400DB6884F8461078
:10F45000E26163B19A6884F84720D96939B194F9B7
:10F46000483023B9042204F1480000F0ABF8094BFE
:10F470005B68C4E90835F06A1321BDE870400430C8
:10F4800007F004B870BD00BFDC2400209C0D0020F4
:10F49000802E002000ED00E030B589B0EFF3098345
:10F4A0006C4603F12005224618685968083303C2E8
:10F4B000AB421446F7D1EFF30581074BC9B29A6B03
:10F4C000D86A986A986A986A986A986A9B6A7B2050
:10F4D000059BFFF7A9FFFEE700ED00E030B589B01E
:10F4E000EFF309836C4603F120052246186859683A
:10F4F000083303C2AB421446F7D1EFF30581074B43
:10F50000C9B29A6B986A986A986A986A986A9B6A6C
:10F51000BF20059BFFF788FFFEE700BF00ED00E07E
:10F5200030B589B0EFF309836C4603F1200522461C
:10F5300018685968083303C2AB421446F7D1EFF399
:10F540000581064BC9B25A6B986A986A986A986A9C
:10F550009B6AE320059BFFF767FFFEE700ED00E0F5
:10F56000FEE70000FEE70000704700000FB483B51F
:10F5700004AC54F8048BFDF7A3FD4FF4A5722021D1
:10F58000FDF78AFD42F21075094F0A4E21464046AA
:10F590000194FFF775FA3846FFF774FA3368294685
:10F5A000986A4FF4FA7503685B689847EEE700BF06
:10F5B000D4BD01089C0D002006F008BE06F010BE68
:10F5C00006F0B2BDF8B50D46074611462846164668
:10F5D00008F004F90446864294BF0246421C2946BC
:10F5E000384608F081F82046F8BD000070B5467B2B
:10F5F00005460EBB4468836804EB8404A40804F544
:10F600000074E21A914288BFCC180C4B29681B6821
:10F61000621CD86A03681B6D984718B901232B73C5
:10F62000304670BDAB68C5E900040021E21A1844F9
:10F6300008F068F80126F3E70026F1E79C0D0020AA
:10F640000EB470B5017B044685B019BBD0E9012327
:10F650009A421BD0134B0AAD1E6820680095D4E96E
:10F660000121099B521A0144F06A0395FAF7F4F854
:10F67000011E0FDBD4E901301B1A8B420FD8204644
:10F680000131FFF7B3FF0028E7D103E0FFF7AEFF3A
:10F690000028DFD105B0BDE8704003B070470844D2
:10F6A000A060F7E79C0D00201022002108F02AB886
:10F6B0000148FFF7F9BF00BFCC24002070B5044615
:10F6C000406A0D46164620B1F9F726FE0023A383B3
:10F6D000A37705EB4500F9F719FE606228B1002316
:10F6E00001202577E67784F8203070BD817270475D
:10F6F000F0B4446A0E4611467CB122460027457F8D
:10F700005FFA87FC65450DD992F801C08C4506D19A
:10F7100092F800C0B44502D19370F0BC7047013735
:10F720000332EDE7027FAA4204D1F0BC82680A48A6
:10F73000FFF7A8B905EB45056655457F05EB45057F
:10F7400025446970427F02EB42021444A370437F58
:10F7500001334377E1E700BFB8BF010813460A460B
:10F760000021FFF7C5BF0000F0B587B004460E4684
:10F770008DF80F208DF814108DF815200BB1FFF7C0
:10F78000EDFF00232268009315692046022205A997
:10F79000A847A76905463FB130B1012331466069EA
:10F7A00000930DF10F02B847284607B0F0BD0000E6
:10F7B0002DE9FF419846037917460B438DF80F302A
:10F7C0000368CDF800801D690E4613460DF10F0148
:10F7D00001220446A8470546606908B9A3693BB100
:10F7E00035B1002300933A4643463146A469A04709
:10F7F000284604B0BDE8F081F7B5437F04460BB955
:10F8000001201CE090F82030C27F0133DBB29A4225
:10F8100080F82030F4D80023857F476A80F82030B4
:10F82000036905EB45057E195BB1795DC0689847B2
:10F8300038B97B5BA4F82130B37884F8233003B067
:10F84000F0BD0123204671780DF10602FFF7B0FFED
:10F8500068B1B2789DF806309A4208D1A37F627FE2
:10F860000133B3FBF2F102FB1133A377C8E70DF1CB
:10F870000702012320467178FFF79AFFB27818B18A
:10F880009DF807309A42E9D0002320467178FFF7AF
:10F890006BFF7B5B0020A4F821309DF8063084F8D4
:10F8A0002330CCE70171704713B5002400F0070046
:10F8B00040EAC10001948DF804008DF805208DF810
:10F8C0000630019802B010BD82B001908DF806108C
:10F8D000019802B07047000070B500260446C0E9E8
:10F8E000026601200D4606F0F1FBB04208BF354626
:10F8F000206065602046267470BD000010B5037C52
:10F90000044613B9006806F0E5FB204610BD000070
:10F9100070B5057C04460E46DDB9BFF35B8FC5604C
:10F92000BFF35B8FBFF35B8F8560BFF35B8F436873
:10F930008B420CD0006806F0CDFB3146012006F06A
:10F94000C5FB206010B96560284670BD6660012562
:10F95000FAE70025F8E7000038B505460C4644B143
:10F9600021462846FFF7D4FF20B904EB4404A4083D
:10F97000F5E7204638BD00000023BFF35B8FC3606E
:10F98000BFF35B8FBFF35B8F8360BFF35B8F704709
:10F99000BFF35B8F0068BFF35B8F704770B50546A0
:10F9A0000C30FFF7F5FF05F1080604463046FFF777
:10F9B000EFFFA04206D930466D68FFF7E9FF2C44FF
:10F9C000201A70BD3046FFF7E3FFF9E770B5054632
:10F9D0004068A0B105F10800FFF7DAFF05F10C0659
:10F9E00004463046FFF7D4FF844288BF00253046E6
:10F9F00098BF6D68FFF7CCFF013C2C44201A70BD06
:10FA000038B50C460546FFF7C9FFA04210D305F1F3
:10FA10000800FFF7BDFF04446868BFF35B8FB4FBC9
:10FA2000F0F100FB1144AC60BFF35B8F012038BDE7
:10FA30000020FCE72DE9F041144607460D46FFF78C
:10FA4000C5FF844228BF0446D4B1B84658F80C6BB1
:10FA50004046FFF79DFF06442E6040467E68FFF754
:10FA600097FF331A9C4203D801206C60BDE8F081F7
:10FA70006B603B68A61B0644AB600220EE60F5E7B6
:10FA80002046F3E738B50C460546FFF79FFFA04236
:10FA900010D305F10C00FFF77BFF04446868BFF347
:10FAA0005B8FB4FBF0F100FB1144EC60BFF35B8FA4
:10FAB000012038BD0020FCE72DE9FF410F466946D3
:10FAC00006466C46FFF7B6FF002504EBC008444528
:10FAD00008D062682068791907F006FE6368083468
:10FAE0001D44F4E729463046FFF7CCFF284604B012
:10FAF000BDE8F081F8B505460C300F46FFF748FF2A
:10FB000005F1080604463046FFF742FFA0423046A2
:10FB100088BF6C68FFF73CFF201A386020B1304680
:10FB20002C68FFF735FF2044F8BD0000F7B51746F5
:10FB300006460D46FFF732FFB842044628BF3C4652
:10FB40000190DCB1304601A9FFF7D4FF019B33B926
:10FB50003268C5E90233C5E9002401200CE09C426B
:10FB600038BF01942860019884426860F5D9241A4E
:10FB700002203368EC60AB6003B0F0BD2046FBE7C9
:10FB80002DE9FF410E466946FFF7D0FF6C46002580
:10FB900004EBC007BC4209D0D4F804807019424677
:10FBA00054F8081B07F0A0FD4544F3E7284604B0CD
:10FBB000BDE8F08138B50546FFF7E2FF044601468F
:10FBC0002846FFF71DFF204638BD00000020704783
:10FBD00000207047002070470368DB68184700006A
:10FBE0004068704708B504494068F6F7A5FF4FF034
:10FBF0006A51F6F7A1FF08BD0000A0400120704740
:10FC000070470000004870470000A04008B5082079
:10FC1000F9F776FB18B1024B0360024B436008BD55
:10FC2000FCBF01087B148E3F014B0360704700BF8F
:10FC30001CC001087047000070470000002070479A
:10FC400070470000704700007047000003689B6B1E
:10FC5000184700000368DB6B18470000704700007E
:10FC60000020704770470000002070470048704730
:10FC70000000C842002070470020704700207047F5
:10FC80007047000000207047002070470020704738
:10FC900070470000704700007047000000230120FB
:10FCA0000B607047002070470020704770470000CD
:10FCB0007047000070470000704700007047000068
:10FCC0007047000000207047704700000020704718
:10FCD0007047000070470000002070470020704708
:10FCE00000207047704700000020704770470000F8
:10FCF0007047000070470000704700007047000028
:10FD00007047000032207047704700000F299CBFE9
:10FD100000EB4100428170470F299ABF00EB410080
:10FD200040894FF461707047102A0B4628BF10229B
:10FD300000F10A015200184607F0D6BC03460079CC
:10FD400008B100221A71704703685B681847000009
:10FD50000279034612B901201871704700207047DC
:10FD60007047000010B50446F9F7D2FA204610BDDE
:10FD70007047000070470000002070470020704767
:10FD8000012070471046704700207047014B036008
:10FD9000704700BF3CC1010882B010B5044602A8FC
:10FDA00040F8043F04F10803C4E9001203C883E8E3
:10FDB0000300DDE9050104F1100383E80300DDE938
:10FDC000070104F1180383E80300DDE9090104F1E8
:10FDD000200383E803002046BDE8104002B07047CE
:10FDE00010B50A4492B2914208D004684B1C615C81
:10FDF0009BB209B1002010BD1946F4E70120FAE7D3
:10FE00000068431C08D010F10F0F07D0044B984234
:10FE100014BF042003207047012070470220704760
:10FE2000F1FFF2FF10B4BDF80440019411C8A446DC
:10FE300010BC60472DE9F0430546894608244FF081
:10FE4000020885B000F110076B68023BA3423BD962
:10FE5000224649463846CDF8008003ABFFF7E2FF63
:10FE600040B19DF80C3003F00303012B08D0032BA5
:10FE700002D063B1002000E0EC6205B0BDE8F08381
:10FE80009DF80D305B0904EBC3040A34DCE7BDF8D0
:10FE90000C309DF80D20C3F38A035209DB000132B8
:10FEA0009BB2D60003EBC202B2F5487FE2DC2A68BF
:10FEB0004946134438460096A21CFFF7B3FF0028BA
:10FEC000D8D002363444BFE70120EC62D5E7000009
:10FED00010B4BDF80440019411C8A44610BC60479A
:10FEE0002DE9F043076B044685B06FB9082690F8FA
:10FEF00028503A4685F00105294600960DEB060389
:10FF00001030FFF78FFF08B900202FE0BDF80C90EC
:10FF1000B9F1510F03D0012384F83430F4E702A87B
:10FF2000FFF76EFF0128F6D1124B04F10808029387
:10FF30003A46404694F82810009602ABFFF7C8FFF7
:10FF40000028E1D06FF00E033A460293294640465E
:10FF5000009602ABADF80C90FFF7BAFF0028D3D0A3
:10FF60004FF45673C4E90B6384F8285005B0BDE81C
:10FF7000F08300BFF1FFF2FF7FB50446D4E906032A
:10FF80000D461646984778B176B15123ADF80C303E
:10FF90004FF0FF33029308230022009329466B445D
:10FFA00004F10800FFF794FF04B070BD2DE9F041A3
:10FFB00090F8343005460F46164694B0002B42D1D7
:10FFC0004FF00108002E61D03F2E94BF34464024EC
:10FFD0006B68EA6AE4B29A1A2B6B42339A4236D3C0
:10FFE0009DF80C30C7F3CA0168F301038DF80C309B
:10FFF000BDF80C30073461F38C03C4F3C404ADF8CE
:020000040801F1
:100000000C30621EC3F3072362F347138DF80D30E3
:100010002B68E40003EBC10122460DF10E0007F04E
:1000200063FB9DF80C30EA6A6FF301038DF80C3026
:10003000A31C9BB2009395F8281003AB05F10800B0
:10004000FFF746FF98B9002014B0BDE8F0812846BC
:10005000FFF746FF0028C3D1D5E9080398470028D9
:10006000F1D0284600F04CF80028B9D1EBE7EB6A54
:1000700002332344EB6207F00703E41AE4B2B4420C
:10008000E2DC2744341BBFB2A6B29BE70120DBE7CA
:10009000F8B505464FF44874402C2746A8BF4027C2
:1000A000C4F54876B6B2BFB23A4631462846FFF7A5
:1000B00097FE28B1403C14F1200FEDD1012006E05D
:1000C0003A4631462846FFF771FF0028F2D1F8BDC5
:1000D000002310B580F8343003630446FFF7D8FFDF
:1000E00060B1012294F8281020465140FFF744FFE8
:1000F00020B12046BDE81040FFF7F2BE002010BD41
:1001000038B590F83550044645B1FCF7D9FF912237
:100110004FF40011FCF7C0FF002038BD012380F828
:100120003530FFF7D5FF84F83550F6E77FB5002569
:1001300008262A46294680F8345080F82850C6629E
:100140000446FFF719FF10B9002004B070BD94F801
:1001500028200121013A18BF01222046FFF70CFF99
:100160000028F1D05123ADF80C306FF00E032A4671
:10017000029394F82810009602AB04F10800FFF7F0
:10018000A7FEE2E710B50446D4E90803984740B15A
:100190002046FFF7CBFF20B12046BDE81040FFF717
:1001A00077BF002010BD00002DE9F047804688B0E1
:1001B00005464FF44872002158F8100B04AF07F0C1
:1001C000A1FA0026B9464FF0080A3B460022314604
:1001D0004046CDF800A0FFF725FE044630B90024C4
:1001E000204608B0BDE8F0870126EEE708AB03EB38
:1001F000C603384633F80C2CFFF702FE0138C0B2B4
:10020000022801D8512A04D02846FFF78FFF044660
:10021000E6E70837002EE7D04846FFF7F1FD07462E
:100220008DF80C0006A8FFF7EBFD874280468DF89D
:100230000D0003D1012FE7D1002608E0032FFBD0EA
:10024000032804D0022FF7D0831E5E425E4108AB24
:10025000334413F8149CA9F10203012B05D831464D
:100260002846FFF7E7FD0028CED086F0010108AB55
:100270000B4413F8143C023B012B04D82846FFF72B
:10028000D9FD0028C0D00023B9F1030F85F8343020
:100290002B6315D0032F06D1012200212846FFF73A
:1002A0006BFE00289BD0B8F1030F06D1012228462F
:1002B0001146FFF761FE002891D000232B638FE7E2
:1002C00086F00106284685F82860FFF7E1FE002841
:1002D000E0D199E700207047002070477047000088
:1002E00010B5054B04460360006C10B103685B68F1
:1002F0009847204610BD00BFDCC1010837B5044651
:100300008E220D46011D01A8F9F786F9FFF756F96F
:10031000E36BC01A642817D8606B40B9E36A2B609E
:10032000012401A8F9F79AF9204603B030BDF6F789
:10033000ABFB0146A06AF6F7B3FC002328606363B9
:100340000023E062A362EBE70024EAE737B5044646
:10035000A4220D46011D01A8F9F75EF9FFF72EF959
:10036000E36BC01A642817D8A06B40B9236B2B60CD
:10037000012401A8F9F772F9204603B030BDF6F761
:1003800083FB0146606AF6F78BFC00232860A363B9
:10039000002320636362EBE70024EAE710B504461C
:1003A000FFF79EFF2046F8F7B3FF204610BD000080
:1003B00013B501230446A421006C0DF10702FFF7D9
:1003C000F7F9B8B19DF807300BB1662B12D10023B5
:1003D0006622A421206CFFF7C7F958B10123206CD5
:1003E00019460DF10702FFF7E3F918B19DF8073040
:1003F000662B00D0002002B010BD000046F66C5302
:100400002DE9F04F044602254FF0040989B0ADF8FC
:1004100010302D4BDFF8B4A01B6804AE0293029B92
:1004200016F8012BD3F804802046D8F80030039248
:10043000D3F800B0002700F0B9FB53460146039AF9
:100440004046CDF804900097D8472064C8B10368AF
:100450009B6A98473422014605A8F9F7F9F8206C01
:1004600039460368DB689847206C02210368DB6C1F
:1004700098472046FFF79CFF074640B905A8F9F7C3
:10048000EDF8012D01D1002719E00125C7E70A2168
:10049000206CFFF72BF9236C2046996800F098FB3D
:1004A000206C0694036843F2D401DD6A084B07937D
:1004B00008AB13E90C00A84705A8F9F7CFF83846B0
:1004C00009B0BDE8F08F00BF9C0D0020801A060027
:1004D000810501087FB5044600230A223021006C03
:1004E000FFF742F901233021206C0DF10302FFF7E1
:1004F0005FF9002842D09DF803301B073ED5052345
:100500000621206C02AAFFF753F9002836D09DF887
:1005100009509DF808302D0445EA03659DF80A301E
:10052000812245EA0325211D01A8BDF80B60F9F7DA
:1005300073F82812F6F7ACFA4FF07051F6F7FCFAA0
:100540000146A06AF6F7F0F9F6BAA0623046F6F76F
:100550009FFA4FF06E51F6F7EFFA0146606AF6F730
:10056000E3F9636B606201336363A36B0133A363DD
:10057000FFF724F8E06301A8F9F770F804B070BD44
:10058000FFF7A8BF10B5054B04460360C06A10B161
:1005900003685B689847204610BD00BF04C201088D
:1005A00037B504460D4640F25D12011D01A8F9F76A
:1005B00033F8E36D2B60FFF701F8646A041BC72C66
:1005C0008CBF0024012401A8F9F748F8204603B0A5
:1005D00030BD000037B504460D4640F26512011DDE
:1005E00001A8F9F719F8236E2B60FEF7E7FF646A9C
:1005F000041BC72C8CBF0024012401A8F9F72EF896
:10060000204603B030BD000010B50446FFF7BAFF26
:100610002046F8F77DFE204610BD000013B50B46BE
:100620000168009200220C691146A04702B010BD7B
:1006300038B504461D4600F0A1FA2346044A204678
:1006400043F82C2B636300236566A36338BD00BFAA
:1006500004C201081FB5AE238DF80F3043680DF1B9
:100660000F01186800230268009314690122A04753
:1006700004B010BD2DE9F743436804460E46174603
:10068000694607221868FFF7C9FF002800F0A58017
:10069000A2689DF80030002A0CBF502240229A42E6
:1006A00007D013F0200F0CBF0220012003B0BDE8DB
:1006B000F0839DF802009DF80130000200EB03403A
:1006C0009DF803301844A0F50000F6F7E1F944491D
:1006D000F6F7E6FA0546E168F6F72EFA2946F6F748
:1006E0002BFA2946F6F728FA216980462846F6F7BC
:1006F00023FA2946F6F720FA01464046F6F714F9A0
:10070000616980462846F6F717FA01464046F6F733
:100710000BF9A169F6F708F92946F6F705F98146BC
:100720009B209DF805509DF804302D0205EB0345F4
:100730009DF80630DFF8AC801D446843F6F7A8F951
:100740004FF04E51F6F7F8F92749F6F7EBF84FF06E
:100750007E5138604846F6F7E7F84FF07C51F6F7DF
:10076000EBF9A844B8F1000F4FF07C51CCBFD4F89E
:100770002090D4F824900546F6F79AFB48B34FF042
:100780007C512846F6F7CEF807461849E069F6F797
:10079000D3F93946F6F7D0F901464FF07E50F6F717
:1007A000C1F804464046F6F773F901462046F6F7CD
:1007B000C3F94946F6F7C0F90D49F6F771FA014653
:1007C0002846F6F7AFF80B49F6F7B6F93060002087
:1007D0006CE729464FF07C50D4E7022066E700BF63
:1007E000FEFFFF4A19638CFF0000344200002040E6
:1007F0000300C84EFFFF7F4B70B54FF0040C002480
:100800001A4B05461E6886B070680368CDE9004C37
:100810001C68174BA0470446E86218B303683035DC
:100820009B6A98473622014603A8F8F711FF55F84E
:10083000040C0A210368DB6C98472846FFF70AFF7F
:10084000044660B1B06A142103685B689847284683
:1008500005AA04A9FFF70EFFB0FA80F4640903A803
:10086000F8F7FCFE204606B070BD00BF9C0D0020CE
:10087000801A060073B5044600F098F92622014656
:100880002046FFF7B9FF0546A0B10B21E06AFEF74D
:100890002DFFE36A2046996800F09AF9E06A009417
:1008A000036844F62061DE6A044B019302AB13E94E
:1008B0000C00B047284602B070BD00BF750B0108A0
:1008C000F0B5856A87B0044616468DF80F102DB135
:1008D000012D4FF000050FD0284623E04368012288
:1008E00018680DF10F01036800951E692B46B0478B
:1008F000C0B10123A362EFE783688562002B4368E0
:100900004FF00302186805A90CBF50274027FFF7D6
:1009100085FE38B19DF81430BB42DDD1BDF81530ED
:100920005BBA338007B0F0BD37B583680446002B4F
:1009300003680CBF2B212F21092B17D8DFE803F008
:1009400005182E41576A8093AAC50DF10602FFF7DC
:10095000B7FF58B1BDF806000004F6F799F84FF05C
:100960004051F6F7E9F80123E060236003B030BDA1
:100970000DF106020131FFF7A3FF0028F6D0BDF804
:100980000600F6F781F84FF04051F6F7D5F801462A
:10099000E068F5F7C9FF0223E060E6E70DF1060223
:1009A0000231FFF78DFF0028E0D0BDF806000004FB
:1009B000F6F76EF84FF04051F6F7BEF803232061CA
:1009C000D3E70DF106020331FFF77AFF0028CDD0FF
:1009D000BDF80600F6F758F84FF04051F6F7ACF8BE
:1009E00001462069F5F7A0FF04232061BDE70DF162
:1009F00006020431FFF764FF0028B7D0BDF80600F7
:100A00000004F6F745F84FF04051F6F795F8052346
:100A10006061AAE70DF106020531FFF751FF0028DA
:100A2000A4D0BDF80600F6F72FF84FF04051F6F7C6
:100A300083F801466069F5F777FF0623606194E764
:100A40000DF106020631FFF73BFF00288ED0BDF8FE
:100A500006000004F6F71CF84FF04051F6F76CF86A
:100A60000723A06181E70DF106020731FFF728FF98
:100A700000283FF47BAFBDF80600F6F705F84FF00D
:100A80004051F6F759F80146A069F5F74DFF0823E4
:100A9000A0616AE70DF106020831FFF711FF002897
:100AA0003FF464AF9DF90700F5F7F2FF1349F6F73D
:100AB000F7F8BDF80650206268B2F5F7E9FF0F4974
:100AC000F6F7EEF8092360624FE70DF106020931EF
:100AD000FFF7F6FE00283FF449AF9DF80600F5F752
:100AE000D7FF0649F6F7DCF80A2323606368E06164
:100AF000186802210368DB6C984737E70000FE4264
:100B000037B5036B04460A2B00F1300505D02846A3
:100B100003B0BDE83040FFF707BF90F8283043B17D
:100B200000F1600201A92846FFF7A4FD40B10128A9
:100B300004D02846FFF78EFD84F8280003B030BDAE
:100B4000FEF73CFD4FF0964160620198F5F7EAFE32
:100B50004FF04E51F5F7F0FF0549F5F7EDFF01466F
:100B6000F5F7E2FE616EF5F7E7FFE065E1E700BF4C
:100B700000809B43FFF7C4BF0020704770B5044658
:100B80000E461546044B40F8043BFDF78BFD20460E
:100B9000E66184F8205070BD2CC201080C21C369A5
:100BA00090F8202001FB0233986970470C21C3693B
:100BB00090F8202001FB0233587F70470C2290F8F8
:100BC0002030C06953431D331844FAF791BB00002D
:100BD00007B50C2290F82030C069534314330191BB
:100BE000184401A9FBF7B8F903B05DF804FB000055
:100BF00010B5054B04460360406C10B103685B6898
:100C00009847204610BD00BF54C2010837B50446BE
:100C100094220D46011D01A8F8F7FEFCFEF7CEFC5C
:100C2000E36BC01A642815D8A06B50B1F5F72CFF00
:100C30000146206BF6F734F80023A36300236062BB
:100C40002363636A01242B6001A8F8F707FD20469F
:100C500003B030BD0024F7E737B50446A7220D46A0
:100C6000011D01A8F8F7D8FCFEF7A8FCE36BC01A39
:100C7000642815D8606B50B1F5F706FF0146E06AAD
:100C8000F6F70EF8002363630023A062E362A36A11
:100C900001242B6001A8F8F7E1FC204603B030BD29
:100CA0000024F7E710B50446FFF7A2FF2046F8F747
:100CB0002FFB204610BD000038B504461D46FFF747
:100CC0005DFF024B20462360256438BD54C20108F5
:100CD00030B50446406C85B003689B6A9847412252
:100CE000014601A8F8F7B4FC606C01210368DB68D9
:100CF0009847606C02210368DB6C9847606C0421A4
:100D0000FEF7F4FC636C20469968FFF761FF606CA6
:100D10000294036844F62061DD6A054B039304AB3B
:100D200013E90C00A84701A8F8F798FC05B030BDFE
:100D3000750E010873B50C4B04461B685D682B6883
:100D40001E68FFF733FF002304220146CDE900327D
:100D500028462822054BB047606418B12046FFF7AB
:100D6000B7FF012002B070BD9C0D0020801A060064
:100D70002DE9FF4104220446406C036800920022E2
:100D80001D69114602ABA847002850D0029E36BA12
:100D9000B30F4CD1300CF5F777FE4FF08C41F5F7DF
:100DA000C1FD4FF06251F5F7C7FE276C05462C498F
:100DB0003846F5F7C1FE01462846F5F7BDFE054663
:100DC00001463846F6F756F888BB294607F1004039
:100DD000F6F76EF858BBC6F34A10F5F755FE2149F1
:100DE000F5F7AAFE2049F5F79DFD211D7E22074655
:100DF00003A8F8F711FCFEF7E1FBD4F828800646BB
:100E000000214046F6F72CF8A0B939464046F5F7E0
:100E100089FD164920F00040F6F74AF850B1E36B1F
:100E2000F31AB3F5FA6F05D203A8F8F717FC04B06C
:100E3000BDE8F0810E492846F5F77EFE0146206B9D
:100E4000F5F772FD39462063E06AF5F76DFDA36B97
:100E5000E0620133A363636BE66301336363E3E73B
:100E6000000020400319C83D000048420000204116
:100E70000AD77843FFF77CBF7047000010B5054BD9
:100E800004460360406C10B103685B6898472046D5
:100E900010BD00BF7CC2010837B50446F8220D46DC
:100EA000011D01A8F8F7B8FBFEF788FBE36BC01A39
:100EB000642815D8206B50B1F5F7E6FD0146A06A0D
:100EC000F5F7EEFE002323630023A063A362A36B68
:100ED00001242B6001A8F8F7C1FB204603B030BD08
:100EE0000024F7E737B5044640F20B120D46011D0A
:100EF00001A8F8F791FBFEF761FBE36BC01A6428C9
:100F000015D8E06A50B1F5F7BFFD0146606AF5F704
:100F1000C7FE0023E362002360636362636B012406
:100F20002B6001A8F8F79AFB204603B030BD0024DF
:100F3000F7E7000010B50446FFF7A0FF2046F8F7DA
:100F4000E7F9204610BD0000002330B5036485B0EA
:100F50000446406C8DF80F300268009315690DF15E
:100F60000F010122A84710B1FEF728FB206405B04D
:100F700030BD000038B50D46FFF710FE0446284688
:100F8000F5F786FD0B49F5F7CDFC214605462046D1
:100F9000F5F7CAFC01462846F5F7CEFD0649F5F7F8
:100FA0007FFE2146F5F7BEFC044900F10040F5F74D
:100FB000C3FD38BD9AC9CC449AC94C460E76D74574
:100FC00070B5124B14461B680D46186903689B6880
:100FD00098470F49F5F7A6FCE1234FF07C520D49E5
:100FE000F8F712FF0C490646F5F7A6FD01462868FA
:100FF000F5F798FC094928603046F5F79DFD014654
:101000002068F5F78FFC206070BD00BF9C0D0020AC
:101010000000A040333333BF000082426F12633FB1
:10102000F0B50025042605640446406C8BB00368C7
:1010300000961F692A46294603ABB847002800F0EE
:10104000A680606C2A46036800961E69294604AB98
:10105000B047002800F09B809DF80C209309023BCC
:10106000012B40F294809DF80D1001EB022143F614
:10107000FF72C1F30D01914200F08980002900F058
:1010800086809DF80E309DF80F6006EB032640F237
:10109000FF73C6F34A169E4279D0002E77D09DF892
:1010A00010009DF8117007EB0027C7F30D0797425A
:1010B0006DD0002F6BD09DF812209DF8135005EBDA
:1010C0000225C5F34A159D4261D0002D5FD0CB1B90
:1010D000002BB8BF5B42FF2B59DC731B002BB8BF42
:1010E0005B42FF2B53DC2046FFF744FF3946059057
:1010F0002046FFF73FFF06903046F5F7C9FC25492B
:10110000F5F71AFD2449F5F7CBFD2449F5F70AFC5C
:1011100007902846F5F7BCFC1E49F5F70DFD1E4962
:10112000F5F7BEFD1D49F5F7FDFBE36908905B6827
:101130005B0709D4204607AA05A9FFF741FF20460F
:1011400008AA06A9FFF73CFFC622211D09A8F8F747
:1011500063FA06990598F5F7E7FB0146A06AF5F7EB
:10116000E3FB0899A0620798F5F7DEFB0146606A89
:10117000F5F7DAFB236B606202332363E36A023321
:10118000E362FEF71BFAE06309A8F8F767FA0BB011
:10119000F0BD00BF0000484300E0FF4400004842AB
:1011A0007FB54FF0040C0026174B04461D68686895
:1011B0000368CDE9006C1E68144BB047606408B347
:1011C00003689B6A98472C22014603A8F8F740FA67
:1011D000606C0A210368DB6C98472046FFF7B4FE79
:1011E000A86A0A2103685B6898472046FFF718FF42
:1011F000E46B03A8003C18BF0124F8F72FFA20463F
:1012000004B070BD0446FAE79C0D0020801A060069
:101210002DE9F74F0446FFF7D1FC054698B10325A9
:10122000364E204616F8017BFFF7C0FC3A460146D1
:101230002046FFF7B5FF002844D1013DF1D1002041
:1012400003B0BDE8F08F2E4B4FF0010AD3F80080B9
:10125000D8F8040003689B68984706460AFA05F325
:1012600033420DD00327DFF894905FFA85FB59468F
:10127000204619F8012BFFF793FF18BB013FF6D169
:101280000135202DEAD1D8F80400002503684FF07D
:101290000109DB689847064609FA05F333420DD089
:1012A0000327DFF858805FFA85FA5146204618F880
:1012B000012BFFF775FF28B9013FF6D10135202D2D
:1012C000EAD1BCE70221606CFEF710FA636C20469D
:1012D0009968FFF77DFC606C02210368DB6C98471E
:1012E000606C0094036844F62061DD6A054B01934D
:1012F00002AB13E90C00A8470120A1E79CC201083A
:101300009C0D00203113010810B5036C04461BB975
:10131000BDE81040FFF718BEFEF750F9236CC01A65
:101320000A2804D92046FFF77BFE2046F0E710BDCF
:10133000FFF7EABF10B5054B04460360406E10B1DD
:1013400003685B689847204610BD00BFCCC2010807
:1013500037B5044640F20D120D46011D01A8F8F7FD
:101360005BF9FEF72BF9E36BC01A642815D8A06B64
:1013700050B1F5F789FB0146206BF5F791FC00238E
:10138000A363002360622363636A01242B6001A8C6
:10139000F8F764F9204603B030BD0024F7E70000F9
:1013A00037B504464FF490720D46011D01A8F8F7B9
:1013B00033F9FEF703F9E36BC01A642815D8606BA4
:1013C00050B1F5F761FB0146E06AF5F769FC0023CF
:1013D00063630023A062E362A36A01242B6001A877
:1013E000F8F73CF9204603B030BD0024F7E70000D1
:1013F00010B50446FFF79EFF2046F7F789FF204609
:1014000010BD000038B504461D46FFF7B7FB034B7F
:101410002046236084F8625038BD00BFCCC201086A
:101420002DE9FF411E238DF80D3000230546406E47
:101430000DF10D010268009314690122A0470446D2
:1014400018B9002004B0BDE8F0811D4B05211B68D0
:1014500005F14008986AA026036847465B689847EC
:1014600002233146686E0DF10E02FEF7A1F9002845
:10147000E8D0BDF80E3002365BBA9AB2002AF6B256
:1014800018BF0024B02E28F8023BE9D1002CD8D197
:10149000B5F84E30384603F00F0423F0FF03A5F8EB
:1014A0004E3002F0CDF88442054604D00246214673
:1014B0000448FDF7E7FA631B58425841C2E700BFF2
:1014C0009C0D0020A0C2010847F276732DE9F04F71
:1014D0000446002789B0DFF8F490DFF8F4B0ADF8E7
:1014E00010300DF1100A94F86230FF2B01D0BB428E
:1014F0002AD1D9F8003020465D684FF000082B68EB
:101500001E68FFF753FB0423CDE9008301465B46C9
:1015100028461AF80720B0476066A8B1036806AEEF
:101520009B6A98474D2201463046F8F791F8606E65
:1015300005210368DB6C98472046FFF771FF0546DD
:10154000304635B9F8F78AF80FB100253AE001279F
:10155000C9E7F8F783F8606E03689B6A98475F22D3
:10156000014605A8F8F774F85423606E8DF80F3023
:101570000368CDF8008001221F690DF10F01434679
:10158000B84784F85080FEF717F80321E065606ED5
:10159000FEF7ACF8636E20469968FFF719FB606EA2
:1015A00002210368DB6C9847606E43F2D401036844
:1015B000DF6A084B0694079396E80C00B84705A825
:1015C000F8F74CF8284609B0BDE8F08F9C0D0020D4
:1015D000801A0600D117010807B503230021406EC9
:1015E00001AAFEF7E5F848B19DF805009DF8043022
:1015F000000240EA03409DF80630184303B05DF84E
:1016000004FB00002DE9F3410446806DF5F740FA34
:1016100000270546B4F84A003946C001F5F74EFAEE
:1016200001462846F5F77EF905463946B4F84600E6
:10163000F5F744FA2946F5F77FFA4FF07051F5F7C0
:101640007BFA0646B4F842003946C003F5F736FA8D
:1016500001463046F5F768F90646606DF5F718FA69
:1016600001463046F5F768FA4FF05451F5F764FA41
:1016700039460646B4F84800F5F720FA2946F5F74A
:101680005BFA4FF07451F5F757FAB4F844108046FE
:101690004804C90BF5F712FA01464046F5F744F93C
:1016A00001463046F5F73EF94FF06051F5F744FA40
:1016B0001A49F5F741FA39460646B4F84C00F5F7F1
:1016C000FDF92946F5F738FA4FF05451F5F734FA99
:1016D0001349F5F729F91349F5F72EFACC220546F7
:1016E000211D01A8F7F798FF206B3146F5F71CF98B
:1016F00029462063E06AF5F717F9A36BE06201332E
:10170000A363636B01336363FDF758FFE06301A8D4
:10171000F7F7A4FF02B0BDE8F08100BF7A81303F47
:101720000000FA440AD7233C73B50446FDF744FF92
:10173000E36DC01A42F20F73984214D92046FFF7A6
:101740004BFF04F16105034678B9606E29460268D3
:10175000009316690122B04710B1FDF72DFFE06537
:10176000012384F8603002B070BD94F8602022B983
:1017700094F86120542A23D1A065002394F85020C6
:10178000606E9A420CBF5422442284F8603084F880
:10179000612002680093166929460122B04700289B
:1017A000DED0FDF709FF052294F85030E0650133E3
:1017B000B3FBF2F202EB82029B1A84F85030D2E7BC
:1017C000442ADAD160652046FFF71CFFD5E7000008
:1017D000FFF7AABF10B5054B04460360006C10B1BB
:1017E00003685B689847204610BD00BFF8C2010837
:1017F00037B5044640F233120D46011D01A8F7F734
:101800000BFFFDF7DBFEA36BC01A642815D8A08D73
:1018100050B1F5F73DF90146206BF5F741FA002389
:10182000A385002360622363636A01242B6001A8FF
:10183000F7F714FF204603B030BD0024F7E700009F
:1018400010B50446FFF7C6FF2046F7F761FD2046B6
:1018500010BD00001FB50B0A8DF80C300023006C82
:101860008DF80D1002680093146903A90222A047A5
:1018700004B010BDF7B50C46054600212046F5F72B
:10188000F9FA002800F091804B4E04F10044002149
:101890002046F5F7F9FA002840F08C80474B1B688A
:1018A000002B00F085801A7C002A00F08180242122
:1018B0005A7C01FB02335F6A2B6828461B6901A929
:1018C000984708B93E4B01933E490198F5F72CF82B
:1018D0003D49F5F731F901463846F5F7E1F94FF0A2
:1018E00050510546F5F7DAFA00285BD03749204613
:1018F00005F072F93649F5F71FF94FF07E51F5F70B
:1019000013F801463348F5F7CBF901463248F5F7AD
:1019100009F83249F5F710F92946F5F7C1F9002120
:101920000546F5F7A7FA00B100252D492846F5F739
:10193000B7F92C4905F050F94FF07E51F4F7F4FF58
:1019400001464FF07E50F5F7ABF901464FF07E505F
:10195000F4F7E8FF2449F5F7EFF82146F4F7E4FF40
:101960002249F5F79DF901460446F4F7DDFF05F03D
:10197000BFF907461E492846F5F7DEF83946F4F761
:10198000D3FF0146F5F7D8F84FF07C51F5F7D4F8BE
:101990002146F4F7C7FF2146F4F7C6FF3146F5F7B5
:1019A000CBF80446204603B0F0BD4FF07E566EE7FC
:1019B000104F81E70024F5E7000080BF34290020A4
:1019C0000000C8413393884348A18F43ECDD2F3F8B
:1019D0000494613B627096430A679643B81EA53F24
:1019E000366E994A9D2C9D3FB3E0D94BCDCC9C3FA0
:1019F000E5D0073D82E6C54737B504464FF49072FF
:101A00000D46011D01A8F7F707FEFDF7D7FDA36BF3
:101A1000C01A642818D8E08D50B1F5F739F801469E
:101A2000606BF5F73DF90023E3850023A062636353
:101A30002046A16AFFF71EFF0124286001A8F7F7DE
:101A40000DFE204603B030BD0024F7E730B5FF247B
:101A50000A448A4211D0082511F8010B444014F0C1
:101A6000800F05F1FF354FEA440418BF84F03104BC
:101A700015F0FF05E4B2F2D1EBE7E31A5842584102
:101A800030BD00000622F0B50446006C87B0036844
:101A9000009200221D69114604ABA8470646FDF7D7
:101AA0008DFD054656B9A06B281AC82804D943F203
:101AB00015612046FFF7CEFE07B0F0BD022220469A
:101AC0009DF8123004A9FFF7C1FF0028F4D00222CC
:101AD00020469DF815300DF11301FFF7B7FF0028E0
:101AE000EAD0BDF81000C0BAF4F7D2FF0646A08FC6
:101AF000F4F7CAFF01463046F5F7D2F80746BDF8BD
:101B00001300C0BAF4F7C4FF0E49F5F7C9F8B222C2
:101B10000646211D03A8F7F77FFD3946606BF4F7F1
:101B200003FF31466063206BF4F7FEFEE38D206314
:101B30000133E385A38DA5630133A38503A8F7F7DC
:101B40008DFDB9E700004843FFF79CBF2DE9F04F3A
:101B5000044603254FF0040B6F4B89B01A889B781D
:101B6000DFF8B8A18DF812306D4BADF810201F686A
:101B700004AED7F804902046D9F800304FF00008A2
:101B80001B680393FFF712F8CDF804B0CDF800807E
:101B900001465346484616F8012BDDF80CC0E047D5
:101BA0002064C8B103689B6A984703689B6898479C
:101BB000206C0A210368DB6C984743F6F9712046D4
:101BC000FFF748FE0346206C002B2CD103689B6A6C
:101BD00098470368DB6898474FF000088EE0B8F13B
:101BE000000FC6D0012594F82020E369062103EBFD
:101BF00082139D64206CFDF779FD236C2046996863
:101C0000FEF7E6FF206C02210368A846DB6C9847CC
:101C1000206C2246036844F62061DE6A414B05943D
:101C20000693B04773E003689B6A98470368DB68D4
:101C30009847B86A44F6206103689B689847206C0F
:101C400003689B6A984703689B68984743F215614D
:101C50002046FFF7FFFD0346206C002BB6D003683B
:101C60009B6A98470368DB689847B86A44F6206126
:101C700003689B689847206C03689B6A98470368D1
:101C80009B6898470922206C414603680092D3F86C
:101C90001090424605ABC847D4F8409020B9D9F817
:101CA000003048469B6A93E7022220469DF8163092
:101CB00005A9FFF7CBFE0028F1D0022220469DF8AF
:101CC00019300DF11701FFF7C1FE0028E7D00222FD
:101CD00020469DF81C300DF11A01FFF7B7FE804633
:101CE0000028DCD0BDF81A3048465BBAA387D9F883
:101CF00000309B6A98470368DB689847013D15F000
:101D0000FF057FF46CAFB8F1000F7FF46BAF404676
:101D100009B0BDE8F08F00BFECC20108801A0600D0
:101D20009C0D0020491B01082DE9F74305462C4E68
:101D3000071DFDF745FC804689462C6AFCB1D4E9B5
:101D40000423904579EB030317D3D4E904128845A3
:101D500079EB020306D3E3685B1842F10002C4E9A1
:101D60000432F2E74522394601A8F7F755FCD4E9D9
:101D70000103984701A8F7F771FC2468DEE7FDF737
:101D80001FFC23460A46296A91B1D1E904EC54EAC2
:101D9000030803D0A6457CEB030807D2704572EB1D
:101DA0000C08044613463CBF744663460968EBE7DB
:101DB000844273EB02014CF250310AD3241A63EBD4
:101DC00002038C4273F1000303D2642C214638BF16
:101DD0006421336889B2986A03689B689847A8E7CA
:101DE0009C0D002038B504460D460430FCF75AFC23
:101DF00004F1340000220A2184F8245004F07AFA15
:101E000004F1380000220A2104F074FA204638BD9B
:101E10002DE9FF4102AF87E80C0090F82C30054611
:101E20000E46DDF828804BBB0123C0F8308080F8D7
:101E30002C30072004F006F90446A0B398F80830C7
:101E400003F00702012A10D0022A14D021464FF4D1
:101E5000F070174B95F82420009504F04DF9A86216
:101E600060B921461348FDF781FB134ADB080721BF
:101E7000FCF7B0FDEAE7114ADB08F8E71820F7F7AE
:101E80003FFA044678B1031D97E8030083E8030096
:101E9000E660FDF795FB361841F100012B6AC4E9B5
:101EA000046123602C62204604B0BDE8F08100BFCD
:101EB000291D010824C3010818C301081EC3010815
:101EC00038B50A4B1446DB68826A0D469A420AD13D
:101ED000CC60FDF775FB24184FF0010041F10001C3
:101EE000C5E9044138BD0020FCE700BF802E00207A
:101EF000F8B51E461B6805460C4617461BB92368F5
:101F000063B9012408E03146BDF81820806B04F065
:101F100009FA0028F3D100242046F8BD21463A46AC
:101F2000686B04F039FA04460028EAD13368002BC4
:101F3000F1D0A86B04F068FAEEE7000038B50D4662
:101F4000114604461A4611B1806B04F017FA2DB100
:101F50002946606BBDE8384004F04EBA38BD000039
:101F60007047000000207047B0F94C007047000037
:101F7000B0F94E0070470000012380F854307047DC
:101F800080F8551070470000034690F8540008B1DF
:101F900093F830007047000037B590F8543004468D
:101FA0000D46ABB190F83030122BA8BF12239942E6
:101FB0000EDA00F13401612201A8F7F72DFB04EBE2
:101FC000450401A8A488F7F749FB204603B030BDBB
:101FD0000024FAE737B590F854500446A5B100F153
:101FE00034014A2201A8F7F717FBD4E90A5100236C
:101FF000226D01A8994208BF9542C4E90A2314BF83
:1020000001250025F7F72AFB284603B030BD000064
:1020100073B590F8544005460E468CB1122A28BF7D
:102020001222144600F13401712201A8F7F7F4FAE4
:1020300030466200291D05F057FB01A8F7F70EFB9B
:10204000204602B070BD0000407B704701617047C0
:1020500038B504460C4B0D4ADB68DA612368A27B75
:102060009B6862B10A4D236820464FF47A719B68E1
:1020700098472B68586903681B699847F3E742F251
:10208000107120469847E9E7802E00203BBF0108E9
:102090009C0D002013B504460121C83003F0A4FCB8
:1020A00004F1D400012103F09FFC3A224FF40471A3
:1020B000094B0094094803F05DFD3B22C4F8BC00C5
:1020C0004FF40471064B0094064803F053FDC4F826
:1020D000C00002B010BD00BF15250108E02400209B
:1020E00051200108F026002070B5437D04460D46BE
:1020F0004BB903681B6C984728B1B620FCF76CFEFF
:1021000040F20113A382236829462046BDE87040AF
:102110009B68184708B5FCF7E3FE034BDB681B1A06
:102120005842584108BD00BF802E00202DE9F047DD
:1021300004460D46FDF744FA06460F46DFF8649064
:10214000FDF73EFA801B4FF0000361EB07014FF4EF
:102150007A72F4F7F3FEA84271F1000320D22368EB
:102160004FF47A719B6820469847A388AB42E7D822
:10217000236820461B6C98470028E1D0FC22D9F840
:1021800000802046D8F82C3093F94CA083F84C20DE
:102190002368DB6C9847D8F82C3083F84CA0CFE745
:1021A000BDE8F0879C0D0020302208B582F311882D
:1021B0008368002B01DC03F03DFC03F009FC0023E5
:1021C00083F3118808BD0000F7B504466D4600F1A1
:1021D000C806304685E8060003F022FCDDE900076A
:1021E000224694F8643004EBC3018A420FD0D2F83F
:1021F00024C0844509D1D2F828C0BC4505D1304659
:1022000003B0BDE8F040FFF7CFBF0832EDE7072B82
:102210000AD895E8030004EBC3022432013382E8B4
:10222000030084F86430EAE7034B04491B689869AB
:1022300003681B689847E2E79C0D002074C30108FF
:102240000C4608B50D4B1B68586A0368DB6C984751
:102250000B4B0C48002C08BF184604F039F872B636
:10226000BFF34F8F0849094BCA6802F4E062134379
:10227000CB60BFF34F8F00BFFDE700BF9C0D002078
:10228000020007B0010007B000ED00E00400FA050D
:1022900010B5836904461BB9BDE8104003F0C0BE09
:1022A000FDF78CF9A369C01AE3699842F4D80120BC
:1022B00010BD000008B5437B13B10348FDF756F984
:1022C0000123437308BD00BF8CC3010803F0EEBBBC
:1022D000084603F0F5BB000038B50C4669B14FF471
:1022E0007A75002105480023E5FB0401044AF4F750
:1022F00025FEBDE8384003F0A9BC38BD3F420F00C1
:1023000040420F0010B5036804461B6C984740B16B
:10231000637D33B10023B4206375BDE81040FCF742
:102320005BBD10BDF7B504466D4600F1D4063046DE
:1023300085E8060003F074FBDDE90007224694F807
:10234000A83004EBC3018A420FD0D2F868C084459C
:1023500009D1D2F86CC0BC4505D1304603B0BDE808
:10236000F040FFF721BF0832EDE7072B0BD895E8C7
:10237000030003F10D0204EBC202013382E8030003
:1023800084F8A830E9E7044B04491B68986903689E
:102390001B689847E1E700BF9C0D0020CCC30108F3
:1023A00038B540250446074B2A4640F8243B002117
:1023B00005F0A8F92A46002104F1680005F0A2F909
:1023C000204638BDF0C301081046002310B50A4C62
:1023D00014F813208A4209D104EB43035B78FF22EF
:1023E00002211844F7F73AFDC0B210BD01330E2B9D
:1023F000EED13A20F9E700BF44C40108F0B585B03A
:10240000074602AD08201E4685E8060003F01AFEC6
:102410000446D0B195E803009DF9302084E803001C
:102420009DF82C103846FFF7CFFF0A9D0246E7358E
:1024300025F007003146074B009403F05DFE05468A
:1024400028B9204603F046FE284605B0F0BD01201D
:10245000FBE700BF5125010810B5044603F0ECFF6F
:10246000FDF7ACF8C4F8AC0010BD000070B503680F
:1024700004461B6C0D46984738B12046FFF7ECFF29
:102480004DB9236A13B90023A36170BD013B2362D8
:10249000002BFAD1F7E7FDF791F8A36943B1E269A0
:1024A000C11A8A4204D913441B1A9D4238BF1D46E3
:1024B000236AC4E906050133236223682046BDE888
:1024C00070409B691847000009C81847F8B590F894
:1024D000A930044603F0FF05DBB9012300F1D4065F
:1024E00080F8A930304603F09BFA304694F8A87083
:1024F000FFF75AFE04F16806AF4207DD736813B1B7
:102500003046FFF7E1FF01350836F5E7002384F890
:10251000A930F8BD10B504460B4B0C4ADB68DA61F4
:102520002368A27B9B6822B94FF47A7120469847B2
:10253000F6E7236820464FF47A719B689847204657
:10254000FFF7C4FFF5E700BF802E0020E4C30108B9
:1025500010B50446FFF7B8FF2046BDE8104003F071
:10256000B9BD000090F8E1007047000003695B7995
:1025700023B90A23406BB0FBF3F070474FF44830A7
:1025800070470000406B70470346007D00B1587DE6
:102590007047000010B5054B0A461B689B69196817
:1025A0004C6801461846A047012010BD9C0D002034
:1025B00090F8CD20034602F0FF0012B193F8CC0052
:1025C000C0B270470020704700207047F8B590F8FF
:1025D000E030476B1A330C4600EBC30150F8335020
:1025E0004E6877B103695B795BB903685B699847AB
:1025F000054B2044B3FBF7F35843281A054666F110
:10260000000628463146F8BD80969800C08970477C
:1026100008B56C30FDF7C2F9003818BF012008BDBD
:1026200090F8CC303BB1054BC26CDB689A4202D1CA
:102630005830FDF7B3B90020704700BF802E00204E
:1026400013B5044600F1B40140F27F226846F6F764
:10265000E3FF4FF4207204F19C0101A8F6F7DCFFC0
:10266000002384F8CC3084F8CD3023695A7912B92C
:10267000186802F091FE002104F15800FDF748F9B6
:10268000002104F16C00FDF743F901A8F6F7E6FF1D
:102690006846F6F7E3FF02B010BD000008B580F809
:1026A00024110821806A02F0EBFF012008BD000020
:1026B00090F8CD20034602F0FF001AB103F16C0040
:1026C000FDF784B9704700002DE9F04790460446B5
:1026D0000E46FCF773FF0746DFF868A000EB080919
:1026E000236820465B699847B04221D24FF480604E
:1026F00002F09AFFDAF80C30A4F854602365FCF776
:102700005DFFC31B434513D24FF47A7CA9EB000550
:10271000002140F2E7304FF47A720023E5FB0C0110
:10272000F4F70CFC01464FF4806002F0C9FFD7E7D4
:10273000236820465B69984786428CBF00200120B1
:10274000BDE8F087802E002070B5036904465A79F1
:10275000002A45D11D68036A002B08BF00210368C9
:1027600080F8E110DB6A9847002839D094F8E1300E
:10277000032B35D8DFE803F002383568206A80B1D2
:10278000012600F00F01324606FA01F120F00F0099
:1027900001F0A2FF236A23F00F0203F00F039E4013
:1027A0005661012384F8E230302383F31188D5F891
:1027B00054345A6912F4407F0FD0DA6822F4005280
:1027C000DA60D5F85424536923F440735361D5F883
:1027D0005424D36843F40053D360002383F3118857
:1027E00070BD0023C4E939330126206A324600F067
:1027F0000F0106FA01F120F00F0001F06DFF236ACE
:1028000023F00F0203F00F0306FA03F353613023A2
:1028100084F8E26083F31188D5F854345A6902F4DD
:102820004072B2F5007FD8D0DA6822F40052DA6044
:10283000D5F85424536943F400735361D5F85424F4
:10284000536923F48073C1E723682046BDE87040D4
:102850000021DB6B1847000010B50446C06940B189
:10286000012100F00F030222994020F00F0001F037
:1028700033FFA06950B1BDE81040012100F00F0303
:102880000222994020F00F0001F026BF10BD000089
:1028900070B5036904465A790D46002A39D101738F
:1028A000186802F079FD012D29D0022D2BD01DB919
:1028B000A38F23F4B053A387236904F13801186868
:1028C00002F05CFD94F83C3133B1236904F5947156
:1028D0001868043002F08EFE002D14BF012300237F
:1028E00084F83C3115D0236904F5947118684FF4CD
:1028F0000062BDE870402023043002F067BEA38F61
:1029000043F4B053D7E7A38F23F4007343F4A053E9
:10291000D1E770BD2DE9F84303690D4659790446A6
:1029200021B1B5FA85F04009BDE8F883C5811E687C
:10293000D868D6F85424D2F81080D2F81490D7680A
:102940001A79FCF7D9F82369E0611A7901219868AE
:10295000FCF7D2F82369A0611A7904211869FCF701
:10296000CBF8236920621A7904215869FCF7C4F86E
:1029700023686062DB6B204694F8E110984715F0FD
:10298000040FD4F8043107F4005721D043F00803B2
:10299000C4F8043194F8083149F0080563B9236993
:1029A0004FF48052186804F586711823043002F041
:1029B0000DFE012384F808310023A382D6F8543495
:1029C0001A6942450BD15A69AA4208D10120ABE7E6
:1029D00023F0080329F00805C4F80431EEE71FB11D
:1029E000DA6822F40052DA60D6F85434C3F8108062
:1029F000D6F854345D61002FE8D0D6F85424D3685B
:102A000043F40053D360E1E738B5036904465A79CB
:102A10000D46DAB9186802F0BFFC012DD4F8003178
:102A20000CD0022D0FD0D4F8003104F13801E38727
:102A300023691868BDE8384002F0A0BC23F40053B5
:102A4000C4F80031EFE743F40053F9E738BD000064
:102A500003695B791BB90421806A02F011BE7047DB
:102A6000F7B590F8CD3004460E46174603F0FF0543
:102A7000BBB100F184014FF4427201A8F6F7CCFD1E
:102A80003A46314604F16C00FDF716F894F824310B
:102A900005461BB10421A06A02F0F2FD01A8F6F779
:102AA000DDFD284603B0F0BD70B590F8E130054675
:102AB0000C46D3B9406AB8B1012600F00F01324686
:102AC00006FA01F120F00F0001F006FE686A84EAC0
:102AD000060300F00F0101F1100293408C4020F03A
:102AE0000F001C430461304670BD0020FCE700006D
:102AF00070B590F8E13005460C46D3B9006AB8B11C
:102B0000012600F00F01324606FA01F120F00F0015
:102B100001F0E2FD286A84EA060300F00F0101F1EA
:102B2000100293408C4020F00F001C43046130469B
:102B300070BD0020FCE70000154B10B50360154B7D
:102B4000044603EB411303614FF4614380F83210F4
:102B5000436300215830FCF7BFFE002104F16C00F4
:102B6000FCF7BAFE04F18400FBF79CFD04F19C0025
:102B7000FBF798FD04F1B400FBF794FD002394F8F3
:102B8000322084F8E130044B204643F8224010BD47
:102B900068C50108E0C401080029002013B5094CEC
:102BA00023686BB900933C22074B4FF478700749B8
:102BB00003F0A2FA2060236813B90548FCF7D6FC9D
:102BC00002B010BD2C2900201931010860C4010891
:102BD00068C4010837B5836A04462BBB134B2269CE
:102BE0001B685179D86A1379114A0093114B04F18B
:102BF0002C05002908BF134606222946F6F74CFE8D
:102C000094F824312946002B18BFB5220A4B08BF7F
:102C10003C224FF4F070009403F06EFAA062A36AB5
:102C200013B90648FCF7A2FC03B030BD9C0D002090
:102C30008FC4010888C40108A132010897C40108A3
:102C40002DE9F341044690461F460D4671B957EAF7
:102C500002030BD190F8CD3043B190F8CC302BB1BA
:102C6000514BDB68C36402B0BDE8F081FFF796FF0B
:102C700023691A68002AF6D04FF4C870B5FBF0F04B
:102C80005B79802838BF8020002B0CBF80234FF455
:102C9000807386B29F4238BF1F46464538BF4646BE
:102CA0004FF49472684604F1B401F6F7B5FCE36D95
:102CB0009E4207D00023314684F8CC3004F15800FE
:102CC000FCF74AFEE36D1B09C4F88030B5B1636BB5
:102CD000AB4266D0354B1B689B696563A34260D0ED
:102CE00004F158052846FCF759FED4F8F83003449F
:102CF000C4F8F8302846FCF73FFE012540F2671281
:102D000004F19C0101A8F6F787FC236F9F4207D0CE
:102D10000023394684F8CD3004F16C00FCF71CFE2A
:102D20001DB104F16C00FCF727FE23695A7992B9B2
:102D3000626B82B1A263D4F8FC20A464A287D4F8A9
:102D4000002104F13801E287D4F80421A4F84020DE
:102D5000186802F013FB236F13B1012384F8CD3000
:102D6000E36D13B1012384F8CC300F4B2046DB68B0
:102D7000E364FFF72FFF23682046DB6B94F8E11034
:102D8000984794F832302BB994F8CD3013B1084BF2
:102D9000084A1A6001A8F6F761FC6846F6F75EFC7F
:102DA00061E70025AAE700BF802E00209C0D0020CF
:102DB000100D00209525010838B5D0F820310446C3
:102DC000C3B900F5867002F039FC1823C4F820312D
:102DD00023691D68284602F0DFFAB4F8403028461F
:102DE00023F00803A4F8403004F13801BDE838406E
:102DF00002F0C4BA38BD00002DE9F047044686B0A1
:102E00000D4640F2CA3200F1840101A8F6F704FC35
:102E100094F8083123B1012D02D92046FFF7CCFFE9
:102E200004F16C092A46484602A9FCF77FFE4FF0E0
:102E300000088246474602ADC2451FDD226953792C
:102E4000D3B910680268D669D5E90012B047061EEA
:102E500014DB05D0FCF7B0FB3744C4F8E400BFB284
:102E6000314648460835FCF7CBFD55F8043C9E42F8
:102E700004D108F10108DFE70026F1E7D4F8EC30CF
:102E800001A83B44C4F8EC30D4F8F0303B44C4F81B
:102E9000F030F6F7E3FB06B0BDE8F08770B5044606
:102EA0006C30FCF77BFD0146F0B12046FFF7A4FF34
:102EB00094F8E130022B17D1D4F8E8501DB9FCF793
:102EC0007BFBC4E93A0523691B689A6BD4F8EC30A4
:102ED000C2F50071994208D2A3F500731344082B80
:102EE00003D9012384F8E13070BDFCF765FBD4F809
:102EF000E830C01A0A4B9842F6D90A4B22691B687F
:102F000009499869094BD21A0368C2F347121B6832
:102F1000984723682046BDE870400021DB6B1847C6
:102F200020A107009C0D0020B8C40108E0C40108DE
:102F300010B5036A0446E3B190F8E110F6F730FCEF
:102F4000B8B104F15800FCF741FD94F8E220D4F840
:102F5000803080B272B198420BD20023012284F8F3
:102F6000E230236A23F00F0103F00F0302FA03F3A8
:102F70000B6110BD10339842FBD90123226A84F8FB
:102F8000E23022F00F0102F00F0293404B61F0E7B4
:102F900070B5124BC26CDB6804469A4219D190F8A6
:102FA000CC3003F0FF0593B100F158063046FCF732
:102FB000F5FCD4F8F8300344C4F8F8303046FCF798
:102FC000DBFC94F8E23033B92046FFF7B1FF284626
:102FD00070BD0025FBE71D46F9E700BF802E0020ED
:102FE00038B50D4B0546DB68C06C984210D195F89A
:102FF000CC306BB105F15800FCF7DCFD044628B17C
:1030000095F8E23013B92846FFF792FF204601E019
:103010004FF0FF3038BD00BF802E002038B5044689
:1030200090F8E050FCF7CCFA85F0010504EBC505FB
:10303000C5E9340194F8E03083F0010384F8E0300E
:1030400038BD00002DE9FF4700F15808044640460E
:10305000FCF7BCFC694602464046FCF7EBFC6E46BA
:103060008146002704F5947AB9450ADD226953792F
:1030700053B910680268156AD6E90012A847051E00
:1030800003DA04B0BDE8F087002594F83C313BB189
:10309000504602F0D3FA10F0200F18BF4FF0FF3562
:1030A000D4F820315BB929464046FCF7EBFCD4F854
:1030B000F43020462B44C4F8F430FFF7AFFF7368B8
:1030C0000836AB42DDD80137CEE7000013B590F8E3
:1030D000CC300446F3B190F80831DBB900F1B4010B
:1030E0004FF48B6201A8F6F797FA2046FFF7AAFF84
:1030F000236D63B104F15800FCF750FCB4F8543070
:10310000984204D34FF48061206D02F0B9FA01A80F
:10311000F6F7A4FA02B010BD104B70B5104C1D6844
:10312000A86A226803689B681AB94FF47A719847B5
:10313000F6E7A86A4FF47A7103680B249B689847F6
:10314000084E56F8040B20B190F8CC300BB1FFF7C5
:10315000BDFF013C14F0FF04F3D1EAE79C0D002011
:103160002C2900200029002073B590F8CD300446AA
:10317000002B53D0D0F8203100F19C051BB340F256
:10318000D742294601A8F6F747FA04F5867002F0FF
:1031900055FAD4F8203123EA0000C4F8200178B9A8
:1031A00023691E68304602F0F7F8B4F84030304624
:1031B00043F00803A4F8403004F1380102F0DEF8CF
:1031C00001A8F6F74BFA94F80831DBB140F2F5426A
:1031D00004F1B40101A8F6F71FFA2046FFF732FF09
:1031E000236D63B104F15800FCF7D8FBB4F85430F8
:1031F000984204D34FF48061206D02F041FA01A897
:10320000F6F72CFA40F2FD42294601A8F6F704FA37
:103210002046FFF743FE01A8F6F720FA02B070BD82
:10322000F8B504461D4DA36A3BB92B684FF47A717B
:10323000986A03689B689847F5E70026012141F2E8
:103240000C0002F03DFA0546FCF7B6F9831BB3F516
:103250007A7F2ABF06460027012729070AD594F856
:103260002431C3B1E36C986B0130B52828BFB52079
:1032700002F0D4FC94F8CD30002BDFD06A0706D4DE
:103280002FB9D4F82031002BD8D0EB04D6D5204666
:10329000FFF76AFFD2E73C20EAE700BF9C0D002061
:1032A00008B5FFF7BDFF00000048704700C60108E1
:1032B00000207047014B0020197070473029002012
:1032C00070470000002070477047000002F006BF02
:1032D000084609B102F0FEBE7047000008B513466B
:1032E000127808460C2AA8BF0C2203491A7004F071
:1032F000FBF9012008BD00BFE8F7FF1F1046194683
:1033000002F096BF02F0A6BF2DE9F34742F6F8217E
:103310006846F6F767F9544801A9FAF79DF8534B48
:1033200005461C6868B9A0694F4A036850491B6884
:10333000984703246846F6F761F9204602B0BDE8D5
:10334000F087019B606B1F3323F01F030193036819
:1033500000211B689847019A01460746284604F059
:10336000B3F90346A06943B9036842491B6898470B
:103370002846FAF77BF80124DCE7002603683E497B
:103380001B689847B146019B4B4523D9606B5FFA98
:1033900086F8036841465B689847824620B928460C
:1033A000FAF764F80224C5E7A06A4FF47A7103685B
:1033B00001361B699847606B41460368DB68984794
:1033C00030B94246A0692D4903681B689847E6E773
:1033D000D144D8E7A069244A036829491E683B46BE
:1033E000B047606B012103684FF001085B699847A3
:1033F000DFF89090A06A4FF47A7103681B699847D0
:10340000606B2A46036839461E69019BB047064631
:10341000A0690368D6B942464946D3F800A00A23FA
:10342000D047A06A6421036808F101085B689847E7
:10343000B8F10B0FDED1606B314603685B699847CA
:10344000A0690A22036810491B68BFE71B680F497F
:103450009847606B0021036800245B699847284601
:10346000FAF704F866E700BFAC7F01089C0D002066
:1034700018C601082BC6010842C601084BC6010840
:103480005CC601086FC6010898C601088EC601080F
:103490002DE9F04F254B9DB093F8E8200C460F9294
:1034A00093F8E9200546109293F8EA2020491192FA
:1034B00093F8EB200026129293F8ED2093F8EC702D
:1034C000139293F8EE20149293F8EF20159293F84C
:1034D000F0B093F8F1A093F8F29093F8F38016AB64
:1034E0001722184604F066F9139A21460792149A97
:1034F000CDE909890692159A0E4B05920F9A089705
:103500000492109ACDE90BAB0392119A8DF86F607B
:103510000292129ACDE9000232222846F6F7BCF94F
:10352000012084F831601DB0BDE8F08F00F7FF1F67
:10353000797A0108B8C6010802F09EBF0846FBF779
:1035400031B900002DE9F04188B00D4604A805A965
:1035500002F0DEFD0024064614492846FCF770F808
:103560002746DFF84C80E0B286421CD9CDE90677C9
:1035700010B1049800EB441007AA06A901F0FCFF63
:103580000C226243059901348818D0E90130029079
:1035900007989B0A0190069800908A582846414651
:1035A000FCF74EF8DFE708B0BDE8F081F0C601088F
:1035B000FBC6010808460AB902F060BD012A01D124
:1035C00002F072BD022AF7D0012002F07FBD000098
:1035D00070B50C4615462AB9084602F07BFD2E460A
:1035E000304670BD104619B9BDE8704002F02ABDE2
:1035F00002F028FD06460028F2D054F8042C21469B
:10360000AA4228BF2A4604F06FF8204602F062FD65
:10361000E6E7000070B50C4615460026AE4204D21F
:10362000F6F726FCA0530236F8E7EB0704D5F6F7C9
:103630001FFC2C4404F8010C012070BDF6F7F6B80D
:1036400000221346C2F3460130F8111012F0010FA8
:103650001ABFC9B24B4083EA1123082113F4004F6B
:103660004FEA430318BF83F4405301F1FF3118BF01
:103670001BB211F0FF019BB2F0D10132102AE1D14F
:10368000180B70472DE9F041456A15B94162BDE854
:10369000F0818B68AC4623F06047C3F38A4616EA94
:1036A000230638BF3E464FEAD37EC3F380782B46CD
:1036B0009A68BEEBD27F22F060440AD0002A18DA62
:1036C000A40CB44217D19D420FD10D60DEE7134622
:1036D000EEE7A74207D102F08044C2F38072424570
:1036E0000BD054B1EFE708D2EDE7CCF800100B6037
:1036F000CDE7B44201D0B442E5D81A689C46002A0E
:10370000E5D11960C3E700002DE9F0474FF47F4988
:10371000089D01F007044FEAD508224405F007058B
:1037200000EBD100944201D1BDE8F08704F0070717
:1037300005F0070A57453E4638BF5646111BC6F1ED
:1037400008068E4228BF0E46E108415C08EBD50E04
:1037500013F80EC0B94029FA06F721FA0AF1FFB2B0
:103760008CEA010147FA0AF739408CEA010C03F8A8
:103770000EC034443544D5E7082341F2210280EAE3
:10378000012001B24000002980B203F1FF33B8BF2D
:10379000504013F0FF03F4D17047000038B50C46D9
:1037A0008D18A54200D138BD14F8011BFFF7E4FFC6
:1037B000F7E700000346406848B1026899895A60FB
:1037C0005A89013292B291425A8138BF9A81704728
:1037D00070B504460D4688B020220021684603F0EB
:1037E00091FF20460495FFF7E5FF024658B16B466E
:1037F000054608AE1C4603CCB442286069602346E7
:1038000005F10805F6D1104608B070BD082817D993
:1038100009280CD00A280CD00B280CD00C280CD06E
:103820000D280CD00E2814BF4020302070470C20EB
:1038300070471020704714207047182070472020D0
:1038400070470000082817D90C280CD910280CD96B
:1038500014280CD918280CD920280CD930288CBF52
:103860000F200E207047092070470A2070470B2058
:1038700070470C2070470D20704700002DE9F84379
:10388000078C0446072F1ED9D0E9029800254FF671
:10389000FF73C5F12006A5F1200029FA05F108FA09
:1038A00006F628FA00F031430143C9B21846FFF783
:1038B00063FF0835402D0346EBD13A46E169BDE888
:1038C000F843FFF76BBF4FF6FF70BDE8F8830000C9
:1038D00010B54B6823B9CA8A63F30902CA8210BDC6
:1038E00004691A681C600361C38A013BC3824A6091
:1038F000EFE700002DE9F84F1D46CB8A0F46C3F3D2
:1039000009010D29814692460B4630D00020AAB20B
:1039100007F11A049EB20C2E1FFA80F80FD89045BA
:1039200003F1010306D3FB8A0A4462F30903012071
:10393000FB821AE01AF800600130E654EAE790458D
:10394000F1D22423A1F10D0BBBFBF3F203FB12BB5D
:103950007C681FFA8BF6002C46D14846FFF72AFFF9
:10396000044638B978606FF00200BDE8F88F4FF078
:103970000008E6E70026066078604FF0000BADB265
:10398000454510D90AEB0803221D13F8011B08F165
:1039900001089155B1B223291FFA88F82CD045456A
:1039A00006F10106F1D8FB8AC3F30902154465F359
:1039B0000903BCE71C46013292B22368002BF9D1FF
:1039C000A5F10D030B442421B3FBF1F301339BB2AA
:1039D0009A42D2D2BBF1000FCFD14846FFF7EAFEA0
:1039E00020B9C4F800B0BEE70122E6E7C0F800B095
:1039F0005E4620600446C0E74545D4D94846FFF7F7
:103A0000D9FE08B92060AEE7C0F800B000262060FB
:103A10000446B5E72DE9F74F1C465B690746884623
:103A20000092002B00F0AE80238C2BB1E269002ABB
:103A300000F0A880072B38D807F10C00FFF7BAFE7A
:103A4000054628B96FF00206304603B0BDE8F08F96
:103A50002822002103F056FE228CE16905F11800AE
:103A600003F042FE208C48F00041013080B2FFF7A5
:103A7000E9FEFFF7CBFE013880B22084013085F8E3
:103A800020006369228C1B782A4403F01F0363F033
:103A90003F031376A960D4E90A2329463846C5E9CD
:103AA0000423FFF7EFFD0126CEE7072202339BB286
:103AB0000633B3FBF2F3C18A828A9BB2521A92B2E6
:103AC0009342BFD84FF000094FF0800ACB464E46D4
:103AD00000F10C0301930198FFF76CFE05460028E6
:103AE000B0D02822002103F00DFEBBF1000F3CD125
:103AF0000222009B2B8305F1180E1FFA82FC0CF1A9
:103B00000100BCF1060F218C80B201D88B452ED369
:103B1000FFF798FEFFF77AFE8B4508BF4FF0400A8B
:103B200062690138127880B202F01F0242EA49123B
:103B300029184AEA020A013048F0004281F818A028
:103B4000AA6085F82000D4E90A01C5E904012946E4
:103B50003846FFF797FD228C01365A454FF0000A90
:103B600036B289F00109B6D16EE70022C3E7E169F8
:103B70000BF1010311F80B101FFA83FB0EF8021072
:103B80000132BAE76FF001065EE70000F8B51546AE
:103B90000E463022002104461F4603F0B3FDB5F562
:103BA000201F38BF2822069B38BFB5FBF2F26360A6
:103BB000079B28BF4FF6FF72A3620023A760E66150
:103BC00097B204F110009A4206D800230360A7823E
:103BD000E3822383E360F8BD066001333046283674
:103BE000F1E7000003781BB94BB2002BC8BF01708E
:103BF0007047000000787047F8B50C46C969074661
:103C000011B9238C002B37D1257E1F2D34D838785D
:103C100028BB228C072A2CD8268A36F003032BD106
:103C20004FF6FF70FFF7BAFD4FF6FF7220F001006C
:103C30003602400446EA0565400C45EA4025234625
:103C400029463846FFF7E6FE002807DD626913784B
:103C50000133DBB21F2B88BF00231370F8BD218A0C
:103C60002D0645EA012505432046FFF707FE0246DB
:103C7000E5E76FF00300F1E76FF00100EEE7000009
:103C80002DE9F041D36905460C4616460BB9138C55
:103C90005BBB377E1F2F28D895F80080B8F1000F46
:103CA00026D03046FFF7EAFD3378210241EAC331DE
:103CB00041EA0801338A41EA076141EA03410246C9
:103CC0003346284641F08001FFF7A4FE00280ADDB4
:103CD0003378012B07D1726913780133DBB21F2BC4
:103CE00088BF00231370BDE8F0816FF00100FAE790
:103CF0006FF00300F7E70000406A00B1083070473A
:103D0000436A1A68426202691A600361C38A013B0E
:103D1000C38270472DE9F041D0F8208014461D463B
:103D200041460027284E21B9416A0B4661BBBDE8D8
:103D3000F081D1E90232E31A65EB02029E4277EB91
:103D400002031ED2036A8B420DD1FFF7C1FD036A45
:103D50001B68036203690B60C38A0161016A013B4E
:103D60008846C382DFE7FFF7B3FD0B68C8F8003071
:103D700003690B60C38A0161013BC382D8F800105C
:103D8000D1E788460968CEE7D1E90476A742AE417B
:103D90000A680BD2466A8E420BD1036942620B60FD
:103DA0000161416AC38A0A46013BC3820B46114640
:103DB000BCE71A6002690A60C28A0161013AC282E4
:103DC00019461A68F2E700BF80841E002DE9F04F03
:103DD0008BB00D4614469B468046DDF85090002877
:103DE00000F01C81B9F1000F00F01881531E3F2B29
:103DF00000F21481012A03D1BBF1000F40F00E81C3
:103E00000023CDE90833B8F81430B5EBC30F4FEAFF
:103E1000C30703D300200BB0BDE8F08F2B199F42DE
:103E2000D8F80C3036BF7F1B2746FFB21BB9D8F835
:103E30001030002B7DD0672D4ED8C5F16806B742F3
:103E40004FF0000334BF3E46F6B200932946324697
:103E5000D8F8080008ABFFF757FCA7EB060A354473
:103E60005FFA8AFA6821B8F8143003F100530D3B69
:103E7000DB000493D8F80C300393039B13B1BAF121
:103E8000000F2CD1D8F8100040B1BAF1000F05D0C6
:103E90005246009608AB691AFFF736FC38B2002F7D
:103EA000B8D066070AD00AAB03EBD40111F8083C7E
:103EB000624202F00702134101F8083C082C3FD986
:103EC000102C40F2B880202C40F2BA80BBF1000FD9
:103ED00000F09F80082337E0BA460026C2E7049B23
:103EE000B3F5907F28BF4FF4907306930B44AB4219
:103EF000059315D95A1B924538BF5246039828BFDF
:103F0000D2B20096691A08AB04300792FFF7FCFBA7
:103F1000079A1644AAEB020A1544F6B25FFA8AFA27
:103F2000049B069A05999B1A0493039B1B680393B1
:103F3000A3E700933A462946D8F8080008ABABE758
:103F4000BBF1000F13D00123B4EBC30F6CD0082CCE
:103F500012D89DF82030621E23FA02F2D50706D54A
:103F60004FF0FF3202FA04F423438DF820309DF81D
:103F7000203089F800304EE7102C12D8BDF82030E0
:103F8000621E23FA02F2D10706D54FF0FF3202FA81
:103F900004F42343ADF82030BDF82030A9F80030F8
:103FA00039E7202C0FD80899631E21FA03F3DA07AA
:103FB00005D54FF0FF3202FA04F40C430894089B35
:103FC000C9F8003027E7402C2BD0DDE90865611ED9
:103FD000C4F12102A4F1210326FA01F105FA02F24B
:103FE00025FA03F311431943CB0712D50122A4F19B
:103FF0002003C4F1200102FA03F322FA01F1A240E6
:10400000524243EA010363EB430332432B43CDE9BE
:104010000823DDE90823C9E90023FCE66FF001006D
:10402000F9E66FF00800F6E6082CA0D9102CB3D9F9
:10403000202CEED8C3E7BBF1000FADD0022383E7FD
:10404000BBF1000FBBD004237EE70000012A30B58E
:10405000144638BF01220025402A28BF402285B0DF
:10406000012CCDE9025517D81B788DF8083053077D
:104070000AD004AB03EBD20515F8083C544204F017
:104080000704A34005F8083C0346009102A800215C
:10409000FFF73AFB05B030BD082CE5D9102C03D84A
:1040A0001B88ADF80830E2E7202C02D81B68029389
:1040B000DDE7D3E90045CDE90245D8E710B5CB6887
:1040C0001BB98B600B618B8210BD04691A681C6080
:1040D0000361C38A013BC382CA60F0E703460A8BCF
:1040E00048699A80186018467047000020F0004325
:1040F000B3F1FF4F10B5044607D316D047F6FF7053
:10410000240C04F40044204310BD09484FF0F06132
:104110002040F2F711FD00F58050B0F1786F28BF14
:104120004FF07860C0F34F30EAE74FF4F840E7E72C
:1041300000F0FF7F03064CBFC0F3C0300220704781
:1041400008B50246FFF7F6FF022806D15306C2F370
:104150000F2001D100F0030008BDC2F30740FBE7C8
:104160002DE9F04F93B0CDE903230A6804461046C9
:10417000FFF7E0FF02280CBF0026C2F30626002A44
:104180000D46824680F2048212F0C04940F000825F
:10419000097E002900F0FC81022803D02378B34275
:1041A00040F0F981C2F304631046069302F07F03E6
:1041B0000593FFF7C5FF059B00224FEA83480023C4
:1041C00048EA0A48294448EA4668CE7BCDE90823F4
:1041D000F309834648EA0008029367D0059B02462C
:1041E000009320465346676808A9B847002800F0A6
:1041F000D581276A4FB9414604F10C00FFF7E8FA70
:10420000074690B96FF0020054E03B6998450DD025
:104210003F68002FF9D1414604F10C00FFF7D8FAAE
:1042200007460028EED0236A3B60276297F817C044
:1042300006F01F08CCF3840CACEB08001FFA80FEDC
:104240000028B8BF0EF12000A8EB0C031FFA83FE74
:10425000B8BF00B2002B0793BEBF0EF120031BB204
:104260000793D7E9022152EA010338D04FF0000C3E
:10427000039BDFF808E29A1A049B63EB0101964561
:104280007CEB01032BD36B7E97F81AE0734519D1B1
:10429000029B002B79D0012821DC7868F8B9DFF87F
:1042A000E0C1944570EB010316D337E0276A27B9C4
:1042B0006FF00C0013B0BDE8F08F3B699845B5D0A6
:1042C0003F68F4E76E4890427CEB010301D3002085
:1042D000F0E7029B002BFAD0079B0F2B17DCFA7D2F
:1042E000B30002F0030203F07C031343FB7539466D
:1042F0002046FFF7EDFA6B7EBB76029B3BB9FB7D58
:10430000C3F38402013262F38603FB75D0E76A7E51
:10431000BB7E9A42DBD1029B002B36D0B309022B25
:1043200033D0039B1422BB60049B0021FB600DA8CB
:1043300003F0E8F9039B20460A93049BADF83EB0D6
:104340000B9305F110030C932B7E8DF840A0013BDD
:10435000DBB2ADF83C30069B8DF841808DF84230E1
:10436000059B0AA98DF8433094F82C3083F00103A3
:104370008DF84430A3689847FB7DC3F38403013371
:1043800003F01F039B02FB82A1E7FB7DC6F34012F3
:10439000B2EBD31F40F00581C3F38403434540F0E3
:1043A0000381029A2B7EB609002A53D016F001062B
:1043B00068D1032B40F2FB80039B3946BB60049B12
:1043C00004F10C00FB60FB8A66F30903FB822B7E81
